:020000040000FA
:1000000000040020E90800007D050000C908000088
:1000100087050000910500009B050000000000001E
:100020000000000000000000000000000D090000BA
:10003000A505000000000000AF050000B9050000A4
:10004000C3050000CD050000D7050000E105000054
:10005000EB050000F5050000FF05000009060000A3
:10006000130600001D0600002706000031060000F0
:100070003B060000450600004F0600005906000040
:10008000630600006D060000770600008106000090
:100090008B060000950600009F060000A9060000E0
:1000A000B3060000BD060000C7060000D106000030
:1000B000DB060000E5060000EF060000F906000080
:1000C000030700000D0700001707000021070000CC
:1000D0002B070000350700003F070000490700001C
:1000E000530700005D07000067070000710700006C
:1000F0007B070000850700008F07000099070000BC
:10010000A30700001FB500F003F88DE80F001FBD26
:1001100000F0E0BB1FB56FF00100009040100390AD
:10012000029001904FF010208069000B420900F00E
:100130001F045DF822300120A04083434DF8223097
:10014000684600F045F91FBDF0B54FF6FF734FF458
:10015000B4751A466E1E11E0A94201D3344600E080
:100160000C46091B30F8027B641E3B441A44F9D14B
:100170009CB204EB134394B204EB12420029EBD17E
:1001800098B200EB134002EB124140EA0140F0BD8F
:10019000DE4992B00446D1E90001CDE91001FF2209
:1001A0004021684600F03CFB94E80F008DE80F000A
:1001B000684610A902E004C841F8042D8842FAD12B
:1001C00010216846FFF7C0FF1090AA208DF8440068
:1001D000FFF7A0FF00F0F3F84FF01024A069102201
:1001E0006946803000F002F9A069082210A900F0E9
:1001F000FDF800F0D8F84FF080510A6949690068AD
:100200004A43824201D8102070470020704710B541
:10021000D0E900214FF0805002EB8103026944696C
:100220006243934209D84FF01022536903EB8103D4
:100230000169406941438B4201D9092010BD5069D1
:10024000401C01D0002010BD0F2010BD70B501680A
:100250000446AF4D4FF01020072952D2DFE801F0DD
:10026000330419293C1E2500D4E902656468294637
:10027000304600F0CDF82A462146304600F0B6F868
:10028000AA002146304600F09FFA002800D0032043
:1002900070BD00F051FB4FF4805007E0201DFFF7C8
:1002A000AAFF0028F4D100F047FB60682860002016
:1002B00070BD241D94E80700920000F085FA002824
:1002C000F6D00E2070BD8069401C12D0201DFFF7B3
:1002D0009EFF0028F6D109E08069401C09D0201D4E
:1002E000FFF789FF0028EDD1606820B12046FFF7B5
:1002F0004FFF042070BDFFF70DFF00F060F800F025
:1003000052F8072070BD10B50C46182802D0012005
:10031000086010BD2068FFF799FF206010BD4FF006
:100320001024A069401C05D0A569A66980353079E4
:10033000AA2808D06069401C2DD060690068401C64
:1003400029D060692CE010212846FFF7FDFE3168B6
:1003500081421CD1A16901F18002C03105E030B1B8
:1003600008CA51F8040D984201D1012000E0002094
:100370008A42F4D158B1286810B1042803D0FEE7AE
:10038000284600F057F862496868086008E000F005
:1003900016F800F008F84FF480500168491C01D0AD
:1003A00000F0A4FAFEE7BFF34F8F5A4801685A4A9B
:1003B00001F4E06111430160BFF34F8FFEE74FF09E
:1003C00010208169491C02D0806900F0AEB87047E6
:1003D000524A01681160121D416811604F4A8168DC
:1003E00010321160111DC068086070472DE9F0419E
:1003F00017460D460646002406E03046296800F000
:10040000A7F8641C2D1D361DBC42F6D3BDE8F08153
:1004100070B50C4605464FF4806608E0284600F0AB
:1004200084F8B44205D3A4F5806405F58055002C0A
:10043000F4D170BD4168044609B1012500E00025F2
:100440004FF010267069A268920000F0BDF9C8B1A3
:10045000204600F01AF89DB17669A56864684FF4EB
:10046000002084420AD2854208D229463046FFF74E
:10047000CFFF2A4621463046FFF7B8FFFFF79FFF20
:10048000FFF791FFFFF746FEF8E72DE9FF414FF038
:100490001024616980680D0B01EB800000F6FF708D
:1004A000010B0020009001900290024603906846E4
:1004B00001230BE0560902F01F0C50F8267003FAD6
:1004C0000CFC47EA0C0740F82670521CAA42F1D3F4
:1004D0000AE04A0901F01F0650F8225003FA06F616
:1004E000354340F82250491C8029F2D3A169090BF9
:1004F0004A0901F01F0150F822408B409C4340F80C
:100500002240FFF765FFBDE8FF8100005C090000A5
:10051000000000200CED00E00400FA050006004099
:10052000144801680029FCD07047134A0221116069
:1005300010490B68002BFCD00F4B1B1D186008687E
:100540000028FCD00020106008680028FCD070470C
:10055000094B10B501221A60064A1468002CFCD021
:10056000016010680028FCD0002018601068002886
:10057000FCD010BD00E4014004E5014008208F4993
:1005800009680958084710208C4909680958084724
:1005900014208A49096809580847182087490968BA
:1005A0000958084730208549096809580847382004
:1005B00082490968095808473C2080490968095858
:1005C000084740207D4909680958084744207B496D
:1005D00009680958084748207849096809580847B0
:1005E0004C20764909680958084750207349096822
:1005F0000958084754207149096809580847582084
:100600006E490968095808475C206C49096809580F
:100610000847602069490968095808476420674904
:100620000968095808476820644909680958084753
:100630006C20624909680958084770205F490968B9
:100640000958084774205D49096809580847782007
:100650005A490968095808477C20584909680958C7
:10066000084780205549096809580847842053499C
:1006700009680958084788205049096809580847F7
:100680008C204E4909680958084790204B49096851
:10069000095808479420494909680958084798208B
:1006A00046490968095808479C204449096809587F
:1006B0000847A0204149096809580847A4203F4934
:1006C000096809580847A8203C490968095808479B
:1006D000AC203A49096809580847B02037490968E9
:1006E00009580847B4203549096809580847B8200F
:1006F0003249096809580847BC2030490968095837
:100700000847C0202D49096809580847C4202B49CB
:10071000096809580847C82028490968095808473E
:10072000CC202649096809580847D0202349096880
:1007300009580847D4202149096809580847D82092
:100740001E49096809580847DC201C4909680958EE
:100750000847E0201949096809580847E420174963
:10076000096809580847E8201449096809580847E2
:10077000EC201249096809580847F0200F49096818
:1007800009580847F4200D49096809580847F82016
:100790000A49096809580847FC20084909680958A6
:1007A00008475FF480700549096809580847000048
:1007B00003480449024A034B704700000000002030
:1007C000680900006809000040EA010310B59B07B2
:1007D0000FD1042A0DD310C808C9121F9C42F8D0AB
:1007E00020BA19BA884201D9012010BD4FF0FF305C
:1007F00010BD1AB1D30703D0521C07E0002010BD72
:1008000010F8013B11F8014B1B1B07D110F8013BFD
:1008100011F8014B1B1B01D1921EF1D1184610BDDE
:1008200002F0FF0343EA032242EA024200F005B865
:100830007047704770474FF000020429C0F01280E3
:1008400010F0030C00F01B80CCF1040CBCF1020F83
:1008500018BF00F8012BA8BF20F8022BA1EB0C0158
:1008600000F00DB85FEAC17C24BF00F8012B00F84E
:10087000012B48BF00F8012B70474FF0000200B574
:10088000134694469646203922BFA0E80C50A0E8B3
:100890000C50B1F12001BFF4F7AF090728BFA0E861
:1008A0000C5048BF0CC05DF804EB890028BF40F82D
:1008B000042B08BF704748BF20F8022B11F0804F6F
:1008C00018BF00F8012B7047014B1B68DB68184705
:1008D0000000002009480A497047FFF7FBFFFFF7B7
:1008E00011FC00BD20BFFDE7064B1847064A10600B
:1008F000016881F30888406800470000680900002B
:10090000680900001F030000000000201EF0040F13
:100910000CBFEFF30881EFF3098188690238007892
:10092000182803D100E00000074A1047074A126860
:100930002C3212681047000000B5054B1B68054AB1
:100940009B58984700BD00000703000000000020EE
:100950005809000004000000001000000000000022
:0809600000FFFFFF0090D0032F
:10100000E0120020D1430200192F000043430200E8
:10101000192F0000192F0000192F000000000000F8
:101020000000000000000000000000002944020051
:10103000192F000000000000192F0000192F0000D8
:101040009144020097440200192F0000192F00005C
:10105000192F0000192F0000192F0000192F000070
:101060009D440200192F0000192F0000A344020024
:10107000192F0000A9440200AF440200B544020049
:10108000192F0000192F0000192F0000192F000040
:10109000192F0000192F0000192F0000192F000030
:1010A000192F0000BB440200192F0000192F000067
:1010B000192F0000192F0000192F0000192F000010
:1010C000C1440200192F0000192F0000192F000041
:1010D000192F0000192F0000192F0000192F0000F0
:1010E000192F0000192F0000192F0000192F0000E0
:1010F000192F0000192F0000192F0000192F0000D0
:10110000192F0000192F000000F002F823F04DF90C
:101110000AA090E8000C82448344AAF10107DA4552
:1011200001D123F042F9AFF2090EBAE80F0013F033
:10113000010F18BFFB1A43F0010318479038020053
:10114000B03802000A444FF0000C10F8013B13F0D5
:10115000070408BF10F8014B1D1108BF10F8015B10
:10116000641E05D010F8016B641E01F8016BF9D103
:1011700013F0080F1EBF10F8014BAD1C0C1B09D15A
:101180006D1E58BF01F801CBFAD505E014F8016BCC
:1011900001F8016B6D1EF9D59142D6D3704700005E
:1011A0000023002400250026103A28BF78C1FBD870
:1011B000520728BF30C148BF0B6070471FB500F011
:1011C0003DF88DE80F001FBD1EF0040F0CBFEFF3BC
:1011D0000880EFF30980014A10470000752E0000D7
:1011E0008269034981614FF001001044704700009B
:1011F000F511000001B41EB400B512F00FFE01B4E9
:101200000198864601BC01B01EBD0000F0B4404606
:10121000494652465B460FB402A0013001B506486C
:10122000004700BF01BC86460FBC804689469246F7
:101230009B46F0BC704700000911000023F0B2B8D3
:1012400070B51A4C054609202070A01C00F05FF80C
:101250005920A08029462046BDE8704008F05CB8BF
:1012600008F065B870B50C461149097829B1A0F1AC
:1012700060015E2908D3012013E0602804D06928AA
:1012800002D043F201000CE020CC0A4E94E80E009C
:1012900006EB8000A0F58050241FD0F8806E284611
:1012A000B047206070BD012070470000080000209A
:1012B0001C0000202845020010B504460021012032
:1012C00000F03DF800210B2000F039F8042119202E
:1012D00000F035F804210D2000F031F804210E2033
:1012E00000F02DF804210F2000F029F80421C84354
:1012F00000F025F80621162000F021F8062115201F
:1013000000F01DF82046FFF79BFF002010BDA8212C
:1013100001807047FFF7A4BF11487047104870471D
:10132000104A10B514680F4B0F4A08331A60FFF7C4
:1013300099FF0C48001D046010BD704770474907B5
:10134000090E002806DA00F00F0000F1E02080F816
:10135000141D704700F1E02080F800147047000071
:1013600003F900421005024001000001FE4800217F
:1013700001604160018170472DE9F743044692B056
:101380009146406813F00EF840B1606813F013F80E
:1013900020B9607800F00300022801D0012000E0AD
:1013A0000020F14E3072484612F0B8FF18B11020FC
:1013B00015B0BDE8F0834946012001F018FF002870
:1013C000F6D101258DF842504FF4C050ADF84000E1
:1013D000002210A9284606F047FC0028E8D18DF825
:1013E00042504FF428504FF00008ADF840004746F7
:1013F0001C216846CDF81C8022F07BFF9DF81C0064
:1014000008AA20F00F00401C20F0F00010308DF8EA
:101410001C0020788DF81D0061789DF81E0061F396
:10142000420040F001008DF81E009DF800000AA95E
:1014300040F002008DF800002089ADF83000ADF8D2
:101440003270608907AFADF834000B97606810AC5C
:101450000E900A94684606F0FCF90028A8D1BDF861
:10146000200030808DF8425042F60120ADF8400057
:101470009DF81E0008AA20F00600801C20F0010044
:101480008DF81E000220ADF83000ADF8340013A82E
:101490000E900AA9684606F0DCF9002888D1BDF84C
:1014A00020007080311D484600F033F9002887D1B4
:1014B0008DF8425042F6A620ADF840001C21684647
:1014C000CDF81C8022F015FF9DF81C00ADF83450BB
:1014D00020F00F00401C20F0F00010308DF81C00B0
:1014E0009DF81D0008AA20F0FF008DF81D009DF852
:1014F0001E000AA920F0060040F00100801C8DF8B3
:101500001E009DF800008DF8445040F002008DF858
:101510000000CDE90A4711A80E90ADF8305068469A
:1015200006F097F9002899D1BDF82000F08000203E
:101530003EE73EB504460820ADF80000204612F014
:10154000EDFE08B110203EBD2146012001F04FFE06
:101550000028F8D12088ADF804006088ADF80600B6
:10156000A088ADF80800E088ADF80A007E4801AB1D
:101570006A468088002106F071FDBDF80010082938
:10158000E1D003203EBD1FB5044600200290082094
:10159000ADF80800CDF80CD0204612F0BFFE10B117
:1015A000102004B010BD704802AA81884FF6FF7069
:1015B00006F096FF0028F4D1BDF80810082901D0E4
:1015C0000320EEE7BDF800102180BDF80210618015
:1015D000BDF80410A180BDF80610E180E1E701B577
:1015E00082B00220ADF800005F4802AB6A46408836
:1015F000002106F033FDBDF80010022900D00320C1
:101600000EBD1CB5002100910221ADF80010019023
:1016100012F0AAFE08B110201CBD53486A4641884A
:101620004FF6FF7006F05CFFBDF800100229F3D002
:1016300003201CBDFEB54C4C06461546207A0F46CD
:10164000C00705D0084612F069FE18B11020FEBD93
:101650000F20FEBDF82D01D90C20FEBD304612F042
:101660005DFE18BB208801A905F03CFE0028F4D1DE
:1016700030788DF80500208801A906F0CEFC0028FE
:10168000EBD100909DF800009DF8051040F002009D
:101690008DF80000090703D040F008008DF8000025
:1016A0002088694606F056FC0028D6D1ADF80850CF
:1016B00020883B4602AA002106F0D0FCBDF80810A5
:1016C000A942CAD00320FEBD7CB50546002000908B
:1016D00001900888ADF800000C462846019512F0EC
:1016E00061FE18B9204612F03FFE08B110207CBD03
:1016F00015B1BDF8000050B11B486A4601884FF68D
:10170000FF7006F0EDFEBDF8001021807CBD0C20BE
:101710007CBD30B593B0044600200D4600901421E6
:1017200001A822F0E6FD1C2108A822F0E2FD9DF8A8
:101730000000CDF808D020F00F00401C20F0F00091
:1017400010308DF800009DF8010020F0FF008DF8AA
:1017500001009DF8200040F002008DF820000120DB
:101760008DF8460002E000000C02002042F6042042
:10177000ADF8440011A801902088ADF83C006088C5
:10178000ADF83E00A088ADF84000E088ADF842001A
:101790009DF8020006AA20F00600801C20F001003F
:1017A0008DF802000820ADF80C00ADF810000FA86D
:1017B000059001A908A806F04CF8002803D1BDF84F
:1017C00018002880002013B030BD0000F0B5007B69
:1017D000059F1E4614460D46012800D0FFDF0C2051
:1017E00030803A203880002C08D0287A032806D090
:1017F000287B012800D0FFDF17206081F0BDA88979
:10180000FBE72DE9F04786B0144691F80C900E9A4C
:101810000D46B9F1010F0BD01021007B2E8A8846AE
:10182000052807D0062833D0FFDF06B0BDE8F087D3
:101830000221F2E7E8890C2100EB400001EB4000B7
:10184000188033201080002CEFD0E88960810027B9
:101850001AE00096688808F1020301AA696900F09D
:1018600084FF06EB0800801C07EB470186B204EBFF
:101870004102BDF8040090810DF1060140460E3290
:1018800010F018FE7F1CBFB26089B842E1D8CCE7E7
:1018900034201080E889B9F1010F11D0122148439A
:1018A0000E301880002CC0D0E88960814846B9F11C
:1018B000010F00D00220207300270DF1040A1FE061
:1018C0000621ECE70096688808F1020301AA69691D
:1018D00000F04BFF06EB0800801C86B2B9F1010F47
:1018E00012D007EBC70004EB4000BDF80410C18123
:1018F00010220AF10201103022F05AFC7F1CBFB204
:101900006089B842DED890E707EB470104EB41025B
:10191000BDF80400D0810AF102014046103210F0F7
:10192000C9FDEBE72DE9F0470E4688B090F80CC0F2
:1019300096F80C80378AF5890C20109902F10C0476
:101940004FF0000ABCF1030F08D0BCF1040F3ED0E9
:10195000BCF1070F7DD0FFDF08B067E705EB850C12
:1019600000EB4C00188031200880002AF4D0A8F148
:10197000060000F0FF09558125E0182101A822F09A
:10198000B8FC00977088434601AA716900F0EDFE2B
:10199000BDF804002080BDF80600E080BDF8080016
:1019A0002081A21C0DF10A01484610F083FDB9F117
:1019B000000F00D018B184F804A0A4F802A007EB2F
:1019C000080087B20A346D1EADB2D6D2C4E705EB6B
:1019D000850C00EB4C00188032200880002ABBD018
:1019E000A8F1050000F0FF09558137E000977088E5
:1019F000434601AA716900F0B8FE9DF80600BDF8E3
:101A00000410E1802179420860F3000162F3410192
:101A1000820862F38201C20862F3C301020962F321
:101A20000411420962F34511820962F386112171A2
:101A3000C0096071BDF80700208122460DF109013F
:101A4000484610F037FD18B184F802A0A4F800A0B1
:101A500000E007E007EB080087B20A346D1EADB264
:101A6000C4D279E7A8F1020084B205FB08F000F1C6
:101A70000E0CA3F800C035230B80002AA6D0558198
:101A80009481009783B270880E32716900F06DFE08
:101A900062E72DE9F84F1E460A9D0C4681462AB1A1
:101AA000607A00F58070D080E089108199F80C0090
:101AB0000C274FF000084FF00E0A0D2873D2DFE814
:101AC00000F09E070E1C28303846556A7373730069
:101AD000214648460095FFF779FEBDE8F88F207B48
:101AE0009146082802D0032800D0FFDF378030203D
:101AF0000AE000BFA9F80A80EFE7207B914604289E
:101B000000D0FFDF378031202880B9F1000FF1D1FC
:101B1000E3E7207B9146042800D0FFDF37803220A6
:101B2000F2E7207B9146022800D0FFDF3780332088
:101B3000EAE7207B1746022800D0FFDF3420A6F812
:101B400000A02880002FC8D0A7F80A80C5E7207B16
:101B50001746042800D0FFDF3520A6F800A0288013
:101B6000002FBAD04046A7F80A8012E0207B174623
:101B7000052802D0062800D0FFDF10203080362054
:101B80002880002FA9D0E0897881A7F80E80B9F8C5
:101B90000E00B881A1E7207B9146072800D0FFDF27
:101BA00037803720B0E72AE04FF0120018804FF05E
:101BB00038001700288090D0E0897881A7F80E803F
:101BC000A7F8108099F80C000A2805D00B2809D036
:101BD0000C280DD0FFDF80E7207B0A2800D0FFDF34
:101BE00001200AE0207B0B2800D0FFDF042004E066
:101BF000207B0C2800D0FFDF052038736DE7FFDF66
:101C00006BE770B50C46054601F025FC20B1007865
:101C1000222804D2082070BD43F2020070BD0521C5
:101C200028460EF0C5FE206008B1002070BD0320DC
:101C300070BD30B44880087820F00F00C01C20F040
:101C4000F000903001F8080B1DCA81E81D0030BC7F
:101C500007F0E3BB2DE9FF4784B0002782460297D7
:101C600007989046894612300AF014F9401D20F07A
:101C70000306079828B907A95046FFF7C2FF0028B6
:101C800054D1B9F1000F05D00798017B19BB052588
:101C900004681BE098F80000092803D00D2812D032
:101CA000FFDF46E0079903254868B0B3497B4288C7
:101CB0007143914239D98AB2B3B2011D0EF0EBFCE7
:101CC0000446078002E0079C042508340CB12088F4
:101CD00010B1032D29D02CE00798012112300AF011
:101CE0000BF9ADF80C00024602AB2946504608F04D
:101CF000F0F9070001D1A01C029007983A46123073
:101D0000C8F80400A8F802A003A94046029B0AF004
:101D100000F9D8B10A2817D200E006E0DFE800F0A9
:101D200007091414100B0D141412132014E60020CC
:101D300012E6112010E608200EE643F203000BE63F
:101D4000072009E60D2007E6032005E6BDF80C0094
:101D50002346CDE900702A465046079900F015FD4C
:101D600057B9032D08D10798B3B2417B406871433E
:101D70008AB2011D0EF0A3FCB9F1000FD7D007996C
:101D800081F80C90D3E72DE9FE4F91461A881C4646
:101D90008A468046FAB102AB494608F09AF9050036
:101DA00019D04046A61C27880EF046FF324607266B
:101DB00029463B4600960EF054FB20882346CDE989
:101DC00000504A465146404600F0DFFC002020808B
:101DD0000120BDE8FE8F0020FBE710B586B01C4651
:101DE000AAB104238DF800301388ADF8083052886A
:101DF000ADF80A208A788DF80E200988ADF80C100D
:101E000000236A462146FFF725FF06B010BD1020CB
:101E1000FBE770B50D4605210EF0CAFD040000D1A8
:101E2000FFDF294604F11200BDE870400AF04DB80A
:101E30002DE9F8430D468046002607F0EBFA0446EC
:101E40002878102878D2DFE800F0773B345331311E
:101E5000123131310831313131312879001FC0B2AE
:101E6000022801D0102810D114BBFFDF35E004B9DF
:101E7000FFDF052140460EF09BFD007B032806D0C6
:101E800004280BD0072828D0FFDF072655E0287943
:101E9000801FC0B2022820D050B1F6E72879401F39
:101EA000C0B2022819D0102817D0EEE704B9FFDF1E
:101EB00013E004B9FFDF287901280ED1172137E09C
:101EC000052140460EF074FD070000D1FFDF07F149
:101ED0001201404609F0D6FF2CB12A462146404661
:101EE000FFF7A7FE29E01321404602F0A7FD24E0FA
:101EF00004B9FFDF052140460EF05AFD060000D16F
:101F0000FFDF694606F1120009F0C6FF060000D0A7
:101F1000FFDFA988172901D2172200E00A46BDF881
:101F20000000824202D9014602E005E01729C5D32C
:101F3000404600F03AFCD0E7FFDF3046BDE8F883CA
:101F4000401D20F0030219B102FB01F0001D00E06A
:101F500000201044704713B5009848B1002468462B
:101F60000EF043FB002C02D1F74A009911601CBD12
:101F700001240020F4E72DE9F0470C461546242102
:101F8000204622F0B6F905B9FFDFA87860732888EB
:101F9000DFF8B4A3401D20F00301AF788946DAF8DA
:101FA00000000EF040FB060000D1FFDF4FF00008FC
:101FB0002660A6F8008077B109FB07F1091D0AD059
:101FC000DAF800000EF02FFB060000D1FFDF66609C
:101FD000C6F8008001E0C4F80480298804F11200EA
:101FE000BDE8F04709F040BF2DE9F047804601F118
:101FF00012000D46814609F04DFF401DD24F20F0E2
:1020000003026E7B1446296838680EF037FB3EB138
:1020100004FB06F2121D03D0696838680EF02EFB2F
:1020200005200EF06DFC044605200EF071FC201A10
:10203000012802D138680EF0EBFA49464046BDE867
:10204000F04709F026BF70B5054605210EF0B0FC3B
:10205000040000D1FFDF04F112012846BDE8704002
:1020600009F010BF2DE9F04F91B04FF0000BADF823
:1020700034B0ADF804B047880C46054692460521B9
:1020800038460EF095FC060000D1FFDF24B1A78092
:10209000A4F806B0A4F808B0297809220B20B2EB06
:1020A000111F7DD12A7A04F1100138274FF00C0856
:1020B0004FF001090391102A73D2DFE802F072F2A7
:1020C000F1F07F08D2888D9F3DDBF3EEB6B6307B12
:1020D000022800D0FFDFA88908EBC001ADF804108A
:1020E0003021ADF83410002C25D06081B5F80E9069
:1020F00000271DE004EBC708317C88F80E10F18939
:10210000A8F80C10CDF800906888042304AA296967
:1021100000F02BFBBDF81010A8F8101009F1040016
:10212000BDF812107F1C1FFA80F9A8F81210BFB278
:102130006089B842DED80DE1307B022800D0FFDF95
:10214000E98908EBC100ADF804003020ADF8340097
:10215000287B0A90001FC0B20F90002CEBD0618149
:10216000B5F81090002725E0CDF8009068886969DF
:1021700003AA0A9B00F0F9FA0A9804EBC70848443E
:102180001FFA80F908F10C0204A90F9810F092F9D7
:1021900018B188F80EB0A8F80CB0BDF80C1001E02A
:1021A000D4E0CFE0A8F81010BDF80E107F1CA8F8FE
:1021B0001210BFB26089B842D6D8CBE00DA800900B
:1021C00001AB224629463046FFF71BFBC2E0307BBD
:1021D000082805D0FFDF03E0307B082800D0FFDFB0
:1021E000E8891030ADF804003620ADF83400002C3A
:1021F0003FD0A9896181F189A18127E0307B09283D
:1022000000D0FFDFA88900F10C01ADF804103721E0
:10221000ADF83410002C2CD06081E8890090AB8997
:10222000688804F10C02296956E0E88939211030E8
:1022300080B2ADF80400ADF83410002C74D0A98938
:102240006181287A0E280AD002212173E989E1816F
:10225000288A0090EB8968886969039A3CE001212B
:10226000F3E70DA8009001AB224629463046FFF760
:1022700059FB6FE0307B0A2800D0FFDF1220ADF859
:102280000400ADF834704CB3A9896181A4F810B092
:10229000A4F80EB084F80C905CE020E002E031E09D
:1022A00039E042E0307B0B2800D0FFDF288AADF810
:1022B00034701230ADF8040084B104212173A9896F
:1022C0006181E989E181298A2182688A00902B8ACB
:1022D000688804F11202696900F047FA3AE0307B3D
:1022E0000C2800D0FFDF1220ADF80400ADF83470E8
:1022F0003CB305212173A4F80AB0A4F80EB0A4F8E9
:1023000010B027E00DA8009001AB224629463046C8
:10231000FFF75CFA1EE00DA8009001AB22462946AB
:102320003046FFF7B6FB15E034E03B21ADF8040082
:10233000ADF8341074B3A4F80690A4F808B084F88B
:102340000AB007E0FFDF05E010000020297A01292C
:1023500017D0FFDFBDF80400AAF800006CB1BDF88B
:1023600034002080BDF804006080BDF834003928B6
:1023700003D03C2801D086F80CB011B00020BDE895
:10238000F08F3C21ADF80400ADF8341014B1697A37
:10239000A172DFE7AAF80000EFE72DE9F8435688BD
:1023A0000F4680461546052130460EF001FB04001D
:1023B00000D1FFDF123400943B46414630466A6844
:1023C00009F0DBFEBAE570B50D4605210EF0F0FA16
:1023D000040000D1FFDF294604F11200BDE870407F
:1023E00009F065BD70B50D4605210EF0E1FA040057
:1023F00000D1FFDF294604F11200BDE8704009F06A
:1024000083BD70B5054605210EF0D2FA040000D157
:10241000FFDF04F1080321462846BDE8704004228E
:10242000B1E470B5054605210EF0C2FA040000D1F2
:10243000FFDF214628462368BDE870400522A2E45C
:1024400070B5064605210EF0B3FA040000D1FFDF97
:1024500004F1120009F01EFD401D20F0030511E0FB
:10246000011D00880322431821463046FFF78BFCEC
:1024700000280BD0607BABB2684382B26068011D5C
:102480000EF053F9606841880029E9D170BD70B53C
:102490000E46054606F0BEFF040000D1FFDF012016
:1024A000207266726580207820F00F00C01C20F03A
:1024B000F00030302070BDE8704006F0AEBF2DE96E
:1024C000F0438BB00D461446814606A9FFF799FBF1
:1024D000002814D14FF6FF7601274FF420588CB115
:1024E00003208DF800001020ADF8100007A805901B
:1024F00007AA204604A90FF0FCFF78B107200BB013
:10250000BDE8F0830820ADF808508DF80E708DF806
:102510000000ADF80A60ADF80C800CE00698A178D8
:1025200001742188C1818DF80E70ADF80850ADF8A6
:102530000C80ADF80A606A4602214846069BFFF708
:1025400089FBDCE708B501228DF8022042F6020281
:10255000ADF800200A4603236946FFF73EFC08BD9C
:1025600008B501228DF8022042F60302ADF80020E2
:102570000A4604236946FFF730FC08BD00B587B062
:1025800079B102228DF800200A88ADF80820498828
:10259000ADF80A1000236A460521FFF75BFB07B080
:1025A00000BD1020FBE709B1072316E407207047A0
:1025B00070B588B00D461446064606A9FFF721FB04
:1025C00000280ED17CB10620ADF808508DF800002F
:1025D000ADF80A40069B6A460821DC813046FFF7C9
:1025E00039FB08B070BD05208DF80000ADF808502B
:1025F000F0E700B587B059B107238DF80030ADF88A
:102600000820039100236A460921FFF723FBC6E750
:102610001020C4E770B588B00C460646002506A910
:10262000FFF7EFFA0028DCD106980121123009F0FB
:1026300063FC9CB12178062921D2DFE801F0200556
:1026400005160318801E80B2C01EE28880B20AB14F
:10265000A3681BB1824203D90C20C2E71020C0E757
:10266000042904D0A08850B901E00620B9E7012967
:1026700013D0022905D004291CD005292AD007200F
:10268000AFE709208DF800006088ADF80800E08809
:10269000ADF80A00A068039023E00A208DF800003E
:1026A0006088ADF80800E088ADF80A00A0680A2547
:1026B000039016E00B208DF800006088ADF808004C
:1026C000A088ADF80A00E088ADF80C00A0680B25E2
:1026D000049006E00C208DF8000060788DF808006A
:1026E0000C256A4629463046069BFFF7B3FA78E781
:1026F00000B587B00D228DF80020ADF8081000233A
:102700006A461946FFF7A6FA49E700B587B071B1E6
:1027100002228DF800200A88ADF808204988ADF81B
:102720000A1000236A460621FFF794FA37E71020C3
:1027300035E770B586B0064601200D46ADF80810A5
:102740008DF80000014600236A463046FFF782FA02
:10275000040008D12946304605F09AFC0021304695
:1027600005F0B4FC204606B070BDF8B51C46154611
:102770000E46069F0EF04EFA2346FF1DBCB23146B0
:102780002A4600940DF039FEF8BD30B41146DDE95B
:1027900002423CB1032903D0002330BC08F022BB25
:1027A0000123FAE71A8030BC704770B50C46054625
:1027B000FFF72FFB2146284605F079FC2846BDE8A7
:1027C0007040012105F082BC4FF0E0224FF400413F
:1027D0000020C2F88011204908702049900208604A
:1027E000704730B51C4D04462878A04218BF002C15
:1027F00002D0002818BFFFDF2878A04208BF30BDF4
:102800002C701749154A0020ECB1164DDFF858C05E
:10281000131F012C0DD0022C1CBFFFDF30BD086040
:1028200003200860CCF800504FF4000010601860DE
:1028300030BD086002200860CCF800504FF04070B6
:102840001060186030BD086008604FF06070106064
:1028500030BD00B5FFDF00BD1800002008F50140C5
:1028600000F500408C02002014F5004070B50B20EC
:1028700000F0B5F9082000F0B2F900210B2000F0BB
:10288000C4F90021082000F0C0F9EC4C0125656076
:10289000A5600020C4F84001C4F84401C4F8480110
:1028A0000B2000F0A7F9082000F0A4F90B2000F09D
:1028B0008BF9256070BD10B50B2000F090F9082051
:1028C00000F08DF9DD48012141608160DC490A6832
:1028D000002AFCD10021C0F84011C0F84411C0F812
:1028E00048110B2000F086F9BDE81040082000F0E8
:1028F00081B910B50B2000F07DF9BDE8104008202B
:1029000000F078B900B530B1012806D0022806D011
:10291000FFDF002000BDCB4800BDCB4800BDCA484A
:10292000001D00BD70B5C9494FF000400860C84D9A
:10293000C00BC5F80803C74800240460C5F840412F
:102940000820C43500F04BF9C5F83C41C24804707A
:1029500070BD08B5B94A002128B1012811D002285C
:102960001CD0FFDF08BD4FF48030C2F80803C2F866
:102970004803B3483C300160C2F84011BDE808404C
:10298000D0E74FF40030C2F80803C2F84803AC485F
:1029900040300160C2F84411AB480CE04FF4802095
:1029A000C2F80803C2F84803A54844300160C2F8E1
:1029B0004811A548001D0068009008BD70B5164676
:1029C0000D460446022800D9FFDF00229B48012360
:1029D00004F110018B4000EB8401C1F8405526B191
:1029E000C1F84021C0F8043303E0C0F80833C1F84F
:1029F0004021C0F8443370BD2DE9F0411C46154616
:102A000030B1012834D0022839D0FFDFBDE8F08191
:102A1000891E002221F07F411046FFF7CFFF012CD5
:102A200024D000208C4E8A4F012470703C6189496B
:102A300000203C3908600220091D086085490420F7
:102A40003039086083483D350560C7F800420820EA
:102A500000F0D0F82004C7F80403082000F0B4F810
:102A60007A49E007091F08603470CFE70120D9E7F1
:102A7000012B02D00022012005E00122FBE7012BFF
:102A800004D000220220BDE8F04197E70122F9E7D7
:102A90006B480068704770B500F0C7F8674C054692
:102AA000D4F840010026012809D1D4F80803C00356
:102AB00005D54FF48030C4F80803C4F84061D4F859
:102AC000440101280CD1D4F80803800308D54FF441
:102AD0000030C4F80803C4F84461012010F0CDFCB4
:102AE000D4F8480101280CD1D4F80803400308D5D4
:102AF0004FF48020C4F80803C4F84861022010F0A5
:102B0000BCFC5648056070BD70B500F08EF8524DA3
:102B10000446287858B1FFF705FF687820B10020F7
:102B200085F8010010F0A9FC4C48046070BD03203A
:102B3000F8E74FF0E0214FF40010C1F800027047B1
:102B4000152000F057B8424901200861082000F024
:102B500051B83F494FF47C10C1F8080300200246E9
:102B600001EB8003C3F84025C3F84021401CC0B2EC
:102B70000628F5D37047410A43F609525143C0F382
:102B8000080010FB02F000F5807001EB5020704748
:102B900010B5430B48F2376463431B0C5C020C60B6
:102BA0002F4C03FB04002F4B4CF2F72443435B0DE7
:102BB00013FB04F404EB402000F580704012107009
:102BC00008681844086010BD00F01F020121914000
:102BD0004009800000F1E020C0F80011704700F0CB
:102BE0001F02012191404009800000F1E020C0F85F
:102BF0008011704700F01F020121914040098000C0
:102C000000F1E020C0F8801270474907090E002843
:102C100006DA00F00F0000F1E02080F8141D704784
:102C200000F1E02080F8001470470C48001F006895
:102C30000A4A0D49121D11607047000000B00040A3
:102C400004B500404081004044B1004008F5014017
:102C500000800040408500403800002014050240FC
:102C6000F7C2FFFF6F0C0100010000010A4810B518
:102C70000468094909480831086010F092FC0648C8
:102C8000001D046010BD0649002008604FF0E021DF
:102C90000220C1F8800270471005024001000001C7
:102CA000FC1F004010B50D2000F06FF8C4B26FF0AB
:102CB000040000F06AF8C0B2844200D0FFDF3A4955
:102CC0000120086010BD70B50D2000F048F8374CA9
:102CD0000020C4F800010125C4F804530D2000F0C1
:102CE00049F825604FF0E0216014C1F8000170BD83
:102CF00010B50D2000F033F82C480121416000216F
:102D0000C0F80011BDE810400D2000F033B828488D
:102D100010B5046826492748083108602349D1F8CE
:102D20000001012804D0FFDF2148001D046010BD10
:102D30001D48001D00680022C0B2C1F8002110F03B
:102D4000E7FFF1E710B51948D0F800110029FBD0D2
:102D5000FFF7DDFFBDE810400D2000F00BB800F0DC
:102D60001F02012191404009800000F1E020C0F8DD
:102D70008011704700F01F0201219140400980003E
:102D800000F1E020C0F880127047002806DA00F059
:102D90000F0000F1E02090F8140D03E000F1E020B6
:102DA00090F800044009704704D5004000D000406E
:102DB000100502400100000110B5202000F082F84B
:102DC000202000F08AF84A49202081F8000449496F
:102DD00000060860091D48480860FEF79DFA45494D
:102DE000C83108604548D0F8041341F00101C0F82B
:102DF0000413D0F8041341F08071C0F804133C4967
:102E000001201C39C1F8000110BD10B5202000F0D0
:102E100059F8384800210160001D0160354A481EFC
:102E2000E83A1060354AC2F80803324BC8331960DB
:102E3000C2F80001C2F8600131490860BDE81040E5
:102E4000202000F04AB82B492E48EC390860704722
:102E500028492C48E8390860704726480160001D61
:102E6000521E0260704723490120E8390860BFF311
:102E70004F8F704770B51F4A8069E83A2149116049
:102E80001E49D1F8006100231F4D1D4A5C1E1EB172
:102E9000A84206D300210FE0D1F8606186B1A842B4
:102EA00009D2C1F80031C1F860311460BDE870404A
:102EB000202000F012B81168BDE8704021F040BA3F
:102EC000FFDF70BD00F01F0201219140400980002A
:102ED00000F1E020C0F88011704700F01F020121CE
:102EE00091404009800000F1E020C0F88012704756
:102EF00020E000E000060240C41400200000024070
:102F00000004024001000001006002000F4A126844
:102F10000D498A420CD118470C4A12680A4B9A4252
:102F200006D101B510F06EFFFFF78DFFBDE801403F
:102F3000074909680958084706480749054A064BE2
:102F40007047000000000000BEBAFECAB0000020BA
:102F500004000020E0120020E012002070B50C46B2
:102F6000054609F0A7FA21462846BDE870400AF058
:102F70008CBB10B511F0B0FBFFF726FC11F04CFA3A
:102F8000BDE8104011F0FEBA0120810708607047CB
:102F9000012081074860704712480068C00700D0D0
:102FA000012070470F48001F0068C00700D00120B3
:102FB00070470C4808300068C00700D001207047F7
:102FC000084810300068704706490C310A68D2037F
:102FD00006D5096801F00301814201D10120704743
:102FE000002070470C0400407047704770477047DE
:102FF000704770477047704770470004050600002F
:103000002CFFFFFFDBE5B15100600200A800FFFFCD
:1030100084000000808D5B0016425791AD5F58BC64
:103020008E702F5A0FAA100DBCD52BFD30B5FC4D5C
:103030000446062CA9780ED2DFE804F0030E0E0E2B
:103040000509FFDF08E0022906D0FFDF04E00329BD
:1030500002D0FFDF00E0FFDFAC7030BD30B50446CA
:103060001038EF4D07280CD2DFE800F0040C060CF6
:103070000C0C0C00FFDF05E0287E112802D0FFDFDA
:1030800000E0FFDF2C7630BD2DE9F0410FF09CFB16
:10309000044610F038FD201AC5B206200DF030FCB1
:1030A000044606200DF034FC211ADD4C207E122847
:1030B00018D000200F1807200DF022FC064607202C
:1030C0000DF026FC301A3918207E13280CD0002071
:1030D0000144A078042809D000200844281AC0B26E
:1030E000BDE8F0810120E5E70120F1E70120F4E7E8
:1030F000CB4810B590F825004108C94800F12600DA
:1031000005D00BF0B6FABDE8104005F0AFBF0BF0EC
:1031100089FAF8E730B50446A1F120000D460A28E7
:103120004AD2DFE800F005070C1C2328353A3F445B
:10313000FFDF42E0207820283FD1FFDF3DE0B848A4
:103140008178052939D0007E122836D020782428AD
:1031500033D0252831D023282FD0FFDF2DE0207851
:1031600022282AD0232828D8FFDF26E0207822280A
:1031700023D0FFDF21E0207822281ED024281CD075
:1031800026281AD0272818D0292816D0FFDF14E0C7
:103190002078252811D0FFDF0FE0207825280CD0DB
:1031A000FFDF0AE02078252807D0FFDF05E0207840
:1031B000282802D0FFDF00E0FFDF257030BD10B50A
:1031C000012803D0022805D0FFDF10BDBDE8104064
:1031D00003202BE79248007E122800D0FFDF002159
:1031E000052011F04FF8BDE81040112036E71FB55B
:1031F00004466A46002001F01FFEB4B1BDF802206B
:103200004FF6FF700621824201D1ADF80210BDF8E1
:103210000420824201D1ADF80410BDF808108142AB
:1032200003D14FF44860ADF8080068460BF089FF01
:1032300005F01CFF04B010BD70B514460D460646DF
:1032400011F06CF858B90DB1A54201D90C2070BD30
:10325000002408E056F8240011F060F808B11020AE
:1032600070BD641CE4B2AC42F4D3002070BD2DE903
:10327000F04105461F4690460E460024006811F0B6
:103280009AF808B110202BE728680028A88802D0F7
:10329000B84202D84FE00028F5D0092020E728687E
:1032A000025DB2B1611C475C152F2DD03BDC3AD2D8
:1032B000DFE807F03912222228282A2A3131393949
:1032C00039393939393939392200025D32BB641C48
:1032D000A4B2A142F9D833E0022ADED1A21C805C5C
:1032E00088F80000072801D2400701D40A20F7E639
:1032F000307840F0010015E0D043C00707E0012A14
:1033000007D010E00620EBE61007A0F1805000285F
:10331000F5D01846E4E63078820701D50B20DFE6C9
:1033200040F0020030702868005D084484B2A8882C
:10333000A04202D2B1E74FF4485381B2A142AED8C5
:103340000020CDE610B5027843F202235408012292
:10335000022C12D003DC3CB1012C16D106E0032C68
:1033600010D07F2C11D112E0002011E080790324CD
:10337000B4EB901F09D10A700BE08079B2EB901F7B
:1033800003D1F8E780798009F5D0184610BDFF20F9
:103390000870002010BD224991F82E2042B191F80A
:1033A0002F10022909D0032909D043F202207047C7
:1033B00001461B48253001F092BD032100E00121A8
:1033C00001700020704738B50C460546694601F08B
:1033D00086FD00280DD19DF80010207861F347008C
:1033E000207055F8010FC4F80100A888A4F8050062
:1033F000002038BD38B51378B0B1022814D0FF28AA
:103400001BD008A46D46246800944C7905EB9414F5
:10341000247864F34703137003280AD010E00000F7
:10342000D80100200302FF0123F0FE0313700228DD
:10343000F2D1D8B240F0010005E043F0FE00107078
:10344000107820F0010010700868C2F80100888828
:10345000A2F8050038BD02210DF0AABA38B50C4615
:103460000978222901D2082038BDADF800008DF876
:10347000022068460BF044F905F0F8FD050003D181
:1034800021212046FFF746FE284638BD1CB5002006
:103490008DF80000CDF80100ADF80500FE4890F869
:1034A0002E00022801D0012000E000208DF8070046
:1034B00068460BF056FB002800D0FFDF1CBD002241
:1034C0000A80437892B263F345120A8043785B081E
:1034D00063F386120A8000780C282BD2DFE800F014
:1034E0002A06090E1116191C1F220C2742F0110082
:1034F00009E042F01D0008800020704742F01100F2
:1035000012E042F0100040F00200F4E742F0100038
:10351000F1E742F00100EEE742F0010004E042F082
:103520000200E8E742F0020040F00400E3E742F066
:103530000400E0E7072070472DE9FF478AB0002527
:10354000BDF82C6082461C4690468DF81C507007D2
:1035500003D5606810F0E2FE68B9CF4F4FF0010963
:1035600097F82E0058B197F82F00022807D160680D
:1035700010F021FF18B110200EB0BDE8F087300721
:1035800002D5A089802816D8700705D4B8F1000F9D
:1035900002D097F8240070B1E07DC0F300108DF8E0
:1035A0001B00617D072041B1012906D00229E3D02B
:1035B0000429E1D12CE00720DEE749468DF8179079
:1035C000F00609D4A27D072032B1012A04D0022AD4
:1035D00005D0042AD0D11BE08DF8191002E002209A
:1035E0008DF819008DF815806068B0B107A9FFF754
:1035F000A9FE0028C0D19DF81C00FF280AD06068F1
:1036000050F8011FCDF80F108088ADF8130008E0C6
:103610000620B1E743F20220AEE7CDF80F50ADF837
:103620001350E07B0028F3D1207C0028F0D1607C8F
:103630000028EDD1A07C0028EAD1E07CC006E7D1CB
:103640008DF800A0BDF82C00ADF80200A068019034
:10365000A068029004F10F0001F035FC8DF80C0019
:103660000DF10D00FFF797FE00B1FFDF9DF81C0084
:103670008DF80E008DF816508DF81850E07D08A9D1
:1036800000F00F008DF81A0068460BF036FF05F0C9
:10369000EDFC71E7F0B59DB000228DF868208DF843
:1036A00058208DF8602005468DF86C2012921392F8
:1036B0001492159219B10FC912AC84E80F00764C20
:1036C000A078052801D004280CD11298616888429E
:1036D00000D120B91498E168884203D110B10820C4
:1036E0001DB0F0BD1F26334618AA1AA912A8FFF76D
:1036F000BEFD0028F4D133461BAA16A914A8FFF773
:10370000B6FD0028ECD19DF85800C00701D00A2072
:10371000E6E7A08A410708D4A17D31B19DF8601089
:10372000890702D043F20120DAE79DF86010C9074B
:1037300009D0400707D4208818B144F2506188426C
:1037400001D90720CCE78DF8005003268DF80160E1
:1037500001278DF80270BDF84C208DF8032001A8D8
:10376000129920F025FD68460BF028FF05F07EFC3D
:103770000028B5D18DF824508DF825608DF826707D
:10378000BDF854208DF827200AA8149920F010FDC8
:1037900009A80BF060FF05F069FC0028A0D112AD6C
:1037A000241D95E80F0084E80F00002098E770B50D
:1037B00086B00D46040005D010F0FDFD20B11020AC
:1037C00006B070BD0820FBE72078C107A98802D0A9
:1037D000FF2902D303E01F2901D20920F0E7800767
:1037E00061D4FFF751FC38B12078C0F3C101012941
:1037F00004D0032902D005E01320E1E7264991F81F
:10380000241041B1C0074FF000054FF0010604D06D
:103810008DF80F6003E00720D2E78DF80F5068465F
:10382000FFF7B9FD00B1FFDF2078C0F3C1008DF8CC
:1038300001008DF80250607808B98DF80260607858
:10384000C00705D09DF8020040F001008DF802008D
:103850006078800705D59DF8020040F002008DF8E1
:1038600002006078400705D59DF8020040F0040092
:103870008DF802002078C0F380008DF80300608886
:10388000ADF80600A088ADF80A00207A58B9607A31
:1038900048B9A07A38B901E0D8010020E07A10B91F
:1038A000207BC00601D006208AE704F1080001F061
:1038B0000AFB8DF80E0068460BF087F905F0D6FB81
:1038C00000288BD18DF810608DF81150ADF8125092
:1038D000ADF8145004A80BF0FDF905F0C7FB002863
:1038E0008BD1E08864280AD248B1012001F001FBA5
:1038F000002891D12078C00705D0152004E064216C
:10390000B0FBF1F0F2E71320FFF7A8FB002057E728
:103910002DE9FF470220FF4E8DF804000027708E2E
:10392000ADF80600B84643F202094CE001A80CF0DD
:10393000A6FF050006D0708EA8B3A6F83280ADF8B9
:1039400006803EE0039CA07F01072DD504F12400F2
:103950000090A28EBDF80800214604F1360301F064
:1039600054FC050005D04D452AD0112D3CD0FFDF79
:103970003AE0A07F20F00801E07F420862F3C7111F
:10398000A177810861F30000E07794F8210000F04E
:103990001F0084F820002078282826D129212046DD
:1039A000FFF7B8FB21E014E040070AD5BDF8080096
:1039B00004F10E0101F0ABFA05000DD04D4510D118
:1039C00000257F1CFFB202200CF09AFF401CB84279
:1039D000ACD8052D11D008E0A07F20F00400A0771E
:1039E00003E0112D00D0FFDF0025BDF80600708632
:1039F000052D04D0284604B0BFE5A6F8328000208B
:103A0000F9E770B50646FFF726FD054605F002FD0D
:103A1000040000D1FFDF6680207820F00F00801CBA
:103A200020F0F000203020700620207295F83E0033
:103A30006072BDE8704005F0F0BC2DE9F04786B03B
:103A4000040000D1FFDF2078B24D20F00F00801C71
:103A500020F0F0007030207060680178491F1B2949
:103A600033D2DFE801F0FE32323255FD320EFDFD79
:103A700042FC32323278FCFCFB323232FCFCFAF986
:103A8000FC00C6883046FFF7E6FC0546304607F0E6
:103A9000A7F8E0B16068007A85F83E002121284649
:103AA000FFF738FB3046FEF7CEFA304603F016FE3D
:103AB0003146012010F0E6FBA87F20F01000A87727
:103AC000FFF726FF002800D0FFDF06B055E520787D
:103AD00020F0F000203020700620207266806068A0
:103AE000007A607205F099FCD8E7C5882846FFF790
:103AF000B2FC00B9FFDF60680079012800D0FFDF69
:103B00006068017A06B02846BDE8F04707F044BC7B
:103B1000C6883046FFF79FFC050000D1FFDF05F0A7
:103B20007CFC606831460089288160684089688132
:103B300060688089A881012010F0A4FB0020A8758E
:103B4000A87F00F003000228BFD1FFF7E1FE0028A4
:103B5000BBD0FFDFB9E70079022811D000B1FFDF49
:103B600005F05BFC6668B6F806A0307A361D0128C1
:103B70000CD0687E814605F0E5F9070009D107E021
:103B800006B00220BDE8F047FFF719BBE878F1E77F
:103B9000FFDF0022022150460CF001FF040000D19B
:103BA000FFDF22212046FFF7B5FA3079012800D047
:103BB0000220A17F804668F30101A177308B20812C
:103BC000708B6081B08BA08184F822908DF8088082
:103BD000B8680090F86801906A46032150460CF0DE
:103BE000DEFE00B9FFDFB888ADF81000B8788DF8B8
:103BF000120004AA052150460CF0D1FE00B9FFDFE7
:103C0000B888ADF80C00F8788DF80E0003AA0421EE
:103C100050460CF0C4FE00B9FFDF062106F1120089
:103C200001F093F938B37079800700D5FFDF71791F
:103C3000E07D61F34700E075D6F80600A061708969
:103C4000A083062106F10C0001F07FF9E8B195F898
:103C500025004108607805E032E02AE047E03FE0D7
:103C600021E035E061F347006070D5F82600C4F824
:103C70000200688D12E0E07D20F0FE00801CE075FF
:103C8000D6F81200A061F08ADAE7607820F0FE0032
:103C9000801C6070F068C4F80200308AE080404602
:103CA000FFF78DFA11E706B02046BDE8F04701F0B6
:103CB00035BD05F0B2FB15F8300F40F0020005E00D
:103CC00005F0ABFB15F8300F40F004002870FCE65F
:103CD000287E132809D01528E4D11620FFF7BEF955
:103CE00006B0BDE8F04705F098BB1420F6E7A978C8
:103CF000052909D00429D5D105F08FFB022006B093
:103D0000BDE8F047FFF792B900790028CAD0E878FB
:103D100002E00000D801002001F0BCF805F07DFBB6
:103D20000320ECE72DE9F05F054600784FF000082E
:103D30000009DFF820A891460C46464601287AD0B3
:103D400001274FF0020C4FF6FF73022874D00728AA
:103D50000BD00A2871D0FFDFA9F8006014B1A4F8D5
:103D6000008066800020BDE8F09F696804F10800CB
:103D70000A78172A70D010DC4FF0000B142A31D0CB
:103D800006DC052A6DD0092A0FD0102A7ED11FE04B
:103D9000152A7CD0162AF9D1F0E01B3A052A75D2F3
:103DA000DFE802F009C5FDDAFC00C8884FF0120810
:103DB0001026214675E14FF01C080A26D4B38888E6
:103DC000A0806868807920726868C0796072C3E7F3
:103DD0004FF01B0814266CB303202072686880889B
:103DE000A080B9E70A793C2AB6D00D1D4FF0100823
:103DF0002C26FCB16988A180298B6182298B2182C4
:103E0000698BA182A98BE1826B790246A91D1846B4
:103E1000FFF7F0FA2879012810D084F80FC0FF20AE
:103E20002076C4F81CB0C4F820B0C4F824B0C4F89C
:103E300028B091E712E013E13BE135E1E7730AF1C5
:103E4000040084F818B090E80E00DAF81000C4E915
:103E50000930C4E907127FE7A8E002E0A9F8006092
:103E600080E72C264FF01D08002CF7D00546A380D4
:103E7000887B2A880F1D60F300022A80887B400817
:103E800060F341022A80887B800801E0E6E0ADE033
:103E900060F382022A80887BB91CC00860F3C302E9
:103EA0002A80B87A0011401C60F3041202F07F00EF
:103EB00028807878AA1CFFF79DFA387D05F1090261
:103EC00007F11501FFF796FA387B01F04DF82874D9
:103ED000787B01F049F86874F87EA874787AE87401
:103EE00097F83B002875B87B6875A5F816B0DAF826
:103EF0001C00A861397ABAF82000884201D2014634
:103F000010E0B87AC0F3411002280BD0012809D084
:103F1000288820F060002880A1840A4607F11C014F
:103F2000A86998E0288820F060004030F3E7112667
:103F30004FF02008002C91D0A380686804F10A0299
:103F4000007920726868007B607269688B1D48790F
:103F50001946FFF74FFAFFE60A264FF02108002C1A
:103F6000E9D08888A0806868807920726868C07904
:103F700060729AF8301021F004018BE00B264FF0AC
:103F80002208002CD7D0C888A080686800792072E9
:103F90006868007A00F0E8FF607201E052E039E002
:103FA0006868407A00F0E0FFA072D5E61C264FF06A
:103FB0002608002CBFD0A3806868407960726868CA
:103FC000007AA0720AF1040090E80E00DAF81000FE
:103FD000C4E90530C4E90312686800793C2803D0BD
:103FE00043287DD0FFDFB7E62772B5E610264FF0F5
:103FF0002408002C9FD08888A08068688079208160
:104000006868807A608168680089A08168688089B2
:10401000E081A1E610264FF02308002C8BD0888881
:10402000A0806868C08820816868008960816868AD
:104030004089A08168688089E0819AF8301021F079
:10404000020127E030264FF02508002C88D0A380FD
:1040500069682822496820F0ABF87DE64A4677E097
:10406000287A012803D0022817D0FFDF74E6102633
:104070004FF01F08002C85D06888A080A889208177
:10408000E8896081288AA081688AE0819AF83010E6
:1040900021F001018AF830105EE64FF01208102678
:1040A000688800F03FFF57E62846BDE8F05F01F062
:1040B000BFBC287A07284DD2DFE800F04C38384AD8
:1040C0004A4A040009264FF01108002C92D06F884C
:1040D0003846FFF7C0F990F822A0A780687A00E080
:1040E0002DE02072042138460CF074FC052138467E
:1040F0000CF070FC002138460CF06CFC01213846B5
:104100000CF068FC032138460CF064FC02213846B0
:104110000CF060FC062138460CF05CFC07213846A8
:104120000CF058FC504600F0B5FE15E614264FF092
:104130001B08002C8AD0A380287A012802D084F89A
:1041400008C009E62772DAE90710C4E9031003E69C
:104150002146A9E7FFDFFFE570B5FE4D287E122856
:1041600001D0082070BD0AF0C3FF04F07FFF0400F7
:1041700002D1687E00F08EFE0021052010F082F84A
:10418000204670BD1CB5F348007E132801D20820DC
:104190001CBD00208DF8000068460AF09BFD04F06D
:1041A00065FF0028F4D10021052010F06BF81120E4
:1041B000FEF754FF00201CBD70B5012805D005286E
:1041C00025D0062800D0FFDF70BD8DB22846FFF74E
:1041D00042F9040000D1FFDF20782128F4D005F057
:1041E00019F968B1017821F00F01891C21F0F00163
:1041F000103101700221017245800020A07528E075
:1042000021462846BDE870401322FFF727B9D14860
:10421000047EA4F1120005281FD2DFE800F0060397
:1042200003030300FFF7AEFF01E0FFF795FF00284F
:10423000CAD105F0EFF80028C6D0017821F00F01AF
:10424000891C21F0F00120310170132C07D00221CC
:104250000172BDE8704005F0E0B8FFDF70BD0121DC
:10426000F6E72DE9F04116460C00804600D1FFDF4D
:10427000307820F00F00801C20F0F00010303070FB
:104280002078012804D0022818D0FFDFBDE8F08193
:104290004046FFF7E0F8050000D1FFDF0320A875D6
:1042A00005F0BBF894E80F00083686E80F00A9482F
:1042B00010F8301F41F001010170E7E74046FFF7B9
:1042C000CAF8050000D1FFDFA1884FF6FF70002774
:1042D000814202D1E288824203D0814201D1E0884A
:1042E00040B105F09AF894E80F00083686E80F0010
:1042F000AF75CBE7A87D0128C8D1782300224146BD
:104300000FF016FF0220A875C0E738B505460C4629
:10431000084610F003F818BB203D062D4AD2DFE80E
:1043200005F0031B373C4230002106200FF080FFD0
:1043300008B1112038BDA01C0AF0AFFF04F096FEB2
:10434000050038D100220823114606200FF0F0FEA8
:10435000062830D0FFDF2EE0606810F023F808B1A7
:10436000102038BD618820886A460BF05FFB04F09E
:104370007DFE05001FD16068E8B1BDF80010018026
:1043800019E0A07800F0010120880BF085FB0EE019
:10439000206801F0FBFD05460DE0207800F00100EB
:1043A0000AF033F903E0618820880BF0C4FA04F0C6
:1043B0005DFEF0E70725284638BD70B505460C467A
:1043C00008460FF0D1FF08B1102070BD202D07D096
:1043D000212D0DD0222D0BD0252D09D0072070BD09
:1043E0002088A11C0AF006FABDE8704004F03EBE29
:1043F000062070BD57482530704708B53421554810
:104400001FF077FF0120FEF711FE1120FEF726FEB8
:1044100050496846263104F093FF4E489DF800202D
:1044200010F8251F62F3470121F0010101700021FE
:1044300041724FF46171A0F8071002218172FEF7FA
:1044400057FE00B1FFDFFCF791FF01F032F908BD24
:1044500010B50C46402120461FF029FFA07F20F018
:104460000300A077202020700020A07584F823008E
:1044700010BD70472DE9FC4107460FF04FFF10B10A
:104480001020BDE8FC81334E06F12501D6F8250049
:104490000090B6F82950ADF8045096F82B408DF8EE
:1044A00006403846FEF78FFF0028EAD1FEF720FECF
:1044B0000028E6D0009946F8251FB580B471E0E7E2
:1044C00010B504460FF050FF08B1102010BD214870
:1044D0002049224690F8250026314008FEF78AFF41
:1044E000002010BDFEB50D4604004FF0000712D0AD
:1044F0000822FEF7A1FE002812D1002609E000BF25
:1045000054F826006946FEF71DFF002808D1761CE6
:10451000F6B2AE42F4D309F07CFF10B143F20320AF
:10452000FEBD0C4E86F8247024B300271EE000BFA9
:1045300054F8270002A9FEF705FF00B1FFDF9DF840
:1045400008008DF8000054F8270050F8011FCDF83E
:10455000011001E0D80100208088ADF80500684610
:1045600009F0A1FF00B1FFDF7F1CFFB2AF42DFD334
:1045700086F824500020FEBD2DE9F0478AB015468C
:10458000894604001ED00F4608222946FEF754FE35
:10459000002810D1002613E054F826006946103098
:1045A00000F09DFC002806D147B157F826000FF017
:1045B000B5FE18B110200AB0BDE8F087761CF6B23F
:1045C000AE42E9D30026A5F101081BE006F1010A7D
:1045D0000AF0FF0712E000BF54F82600017C4A08E9
:1045E00054F827100B7CB2EB530F05D10622113083
:1045F00011311FF0B1FD58B17F1CFFB2AF42EBD3B8
:104600000AF0FF064645E1DB4E4624B1012003E0F7
:1046100043F20520CFE7002009F076FF10B909F03A
:1046200087FF10B143F20420C5E75CB300270DF10A
:10463000170825E054F827006946103000F04FFCB9
:1046400000B1FFDF54F82700102250F8111FCDF8F9
:1046500001108088ADF8050054F827100DF107000F
:104660001FF0A6FD96B156F82710102240461FF005
:104670009FFD684609F0F0FE00B1FFDF7F1CFFB22E
:10468000AF42D7D3FEF702FF002094E7404601F087
:1046900071FCEEE730B585B004460FF03FFE18B967
:1046A00060680FF088FE10B1102005B030BD608842
:1046B0004AF2B811884206D82078FB4D28B101286B
:1046C00006D0022804D00720EFE7FEF711FD18E01E
:1046D0006078022804D0032802D043F20220E4E7E5
:1046E00085F82F00C1B200200090ADF80400022927
:1046F0002CD0032927D0FFDF684609F0BAFF04F069
:10470000B5FC0028D1D1606801F027FC207858B1B1
:1047100001208DF800000DF1010001F02BFC68462E
:104720000BF018FA00B1FFDF207885F82E00FEF7B5
:10473000ADFE608860B1A88580B209F0DDFE00B1F1
:10474000FFDF0020B1E78DF80500D5E74020FAE74C
:104750004FF46170EFE710B504460FF005FE20B985
:10476000606838B10FF01EFE08B1102010BD6068FF
:1047700001F000FCCC4830F82C1F6180C1786170DA
:1047800080782070002010BD2DE9F843144689463A
:1047900006460FF0E9FDA0B948460FF00CFE80B9BF
:1047A00020460FF008FE60B9BF4DA878012800D15F
:1047B0003CB13178FF2906D049B143F20400BDE88D
:1047C000F8831020FBE7012801D00420F7E74FF021
:1047D0000008A4B3052811D004280FD0694620464C
:1047E000FEF76DFE0028EAD1207D48B1012809D0EE
:1047F000022809D0032809D00720E0E70820DEE7D7
:10480000424604E0012202E0022200E003222346A5
:10481000174600200099FEF78FFE0028CFD1A0890F
:104820002880A07BE875BDF80000A882AF75BDF8B0
:104830000000000701D5A08988B1A08928804946D9
:104840000020FEF727FF0028B9D1A87805280BD053
:10485000042809D0287DC00703D0032002E080206F
:10486000ECE70220FEF7E2FB86F800800020A6E7D6
:104870007CB58D4C05460E46A078022803D003284F
:1048800001D008207CBD15B143F204007CBD072097
:104890000CF03EF810B9A078032806D0FEF7F4FB20
:1048A00028B1A078032804D009E012207CBD132091
:1048B0007CBD304600F0CDFA0028F9D1E670012029
:1048C0008DF800008DF801008DF802502088ADF8B9
:1048D0000400E07D8DF8060068460AF0EAFF04F067
:1048E000C5FB0028E4D1A078032805D05FF00400C0
:1048F000FEF79CFB00207CBDE07800F0BAFA0520B2
:10490000F6E71CB510B143F204001CBD664CA0785C
:10491000042803D0052801D008201CBD00208DF8F4
:10492000000001218DF801108DF8020068460AF0A0
:10493000C0FF04F09BFB0028EFD1A078052805D02C
:104940005FF00200FEF772FB00201CBDE07800F073
:10495000A1FA0320F6E72DE9FC4180460E46032527
:1049600008460FF028FD002866D14046FEF773FD8B
:10497000040004D02078222804D2082081E543F2E4
:1049800002007EE5A07F00F003073EB1012F0CD0AE
:1049900000203146FEF72BFC0500EFD1012F06D099
:1049A000022F1AD0FFDF28466BE50120F1E7A07D3A
:1049B0003146022801D011B107E0112061E56846B7
:1049C000FCF7E1FD0028D9D16946404606F0A7FC76
:1049D0000500E8D10120A075E5E7A07D032804D1FA
:1049E000314890F83000C00701D02EB30EE026B158
:1049F000A07F40071ED4002100E00121404606F0C0
:104A0000AEFC0500CFD1A075002ECCD0314640467B
:104A100000F07DFA05461128C5D1A07F4107C2D418
:104A2000316844F80E1F7168616040F00400207422
:104A30000025B8E71125B6E7102022E570B50C4631
:104A40000546FEF708FD010005D022462846BDE8D0
:104A50007040FEF703BD43F2020070BD10B501289F
:104A600007D1114B9B78012B00D011B143F2040008
:104A700010BD09F084FDBDE8104004F0F7BA012331
:104A800000F012BA00231A46194600F00DBA70B5AC
:104A900006460C4608460FF041FC18B920680FF096
:104AA00063FC18B1102070BDD8010020F74D2A7E9C
:104AB000112A04D0132A00D33EB10820F3E721467F
:104AC0003046FEF774FE60B1EDE70920132A0DD0E1
:104AD000142A0BD0A188FF29E5D31520FEF7BEFAD2
:104AE0000020D4E90012C5E90712DCE7A1881F29DC
:104AF000D9D31320F2E72DE9F047DFF8908307467A
:104B000090B098F818009A4615460C46132803D31F
:104B1000FFF738FB002822D120460FF0FFFBA0BB97
:104B200028460FF0FBFB80BB20784FF00101C00747
:104B30004FF0000602D08DF83A1001E08DF83A608F
:104B40002078C0F3C1008DF800006278072042B1E0
:104B5000012A06D0022A02D0042A00D1062010B071
:104B60002AE58DF809106088ADF80A00A088ADF834
:104B7000100020788946C0F3C10001281FD0032807
:104B80001DD038460FF0CAFB08B11020E7E738788F
:104B9000400808D0012809D0022807D0032805D0F2
:104BA00043F20220DBE78DF8026001E08DF802900D
:104BB00057F8010FCDF80300B888ADF807000DF1E4
:104BC0000100FEF7E8FB08B10320C8E72888ADF82C
:104BD00016006888ADF81C00A888ADF82200E888A7
:104BE000ADF82800ADF82E60ADF8346068460AF0E4
:104BF000BDF8E8B998F818004546112801D00820FA
:104C0000ADE706200BF084FE38B12078C0F3C10078
:104C1000012804D0032802D004E012209FE795F871
:104C2000240028B1FEF730FA022803D2132096E7B9
:104C3000072094E7504600F00CF900288FD185F842
:104C400019A068460AF051FA04F010FA002886D13B
:104C5000687E00F00EF9E08864280AD248B101208D
:104C600000F047F9040091D11220FEF7F7F9204631
:104C700075E76421B0FBF1F0F2E770B50646154622
:104C80000C4608460FF070FB18B928460FF06CFB75
:104C900008B1102007E72A46214630460AF0A9FE4F
:104CA00004F0E4F90028F5D121787F29F2D105201C
:104CB000F9E67CB505460C4608460FF02FFB08B117
:104CC00010207CBD2846FEF7C6FB20B100782228C4
:104CD00004D208207CBD43F202007CBD6B4890F8F2
:104CE0003000400701D511207CBD2178C80802D1D1
:104CF0006078C20801D007207CBD890801D18008F6
:104D000001D006207CBDADF8005020788DF802005F
:104D100060788DF803000220ADF80400684609F0C1
:104D200042FF04F0A3F97CBD70B586B014460D4671
:104D30000646FEF790FB28B10078222805D208200D
:104D400006B0B0E643F20200FAE728460FF033FB64
:104D500020B944B120460FF025FB08B11020EFE741
:104D600000202060A080494890F83000800701D5DD
:104D70001120E5E703A9304609F0BDFD18B100BFD9
:104D800004F074F9DCE7ADF80060BDF81400ADF88C
:104D90000200BDF81600ADF80400BDF81000BDF823
:104DA0001210ADF80600ADF808107DB1298809B1E0
:104DB000ADF80610698809B1ADF80210A98809B1EB
:104DC000ADF80810E98809B1ADF80410DCB1BDF800
:104DD0000610814201D9081A2080BDF80210BDF8E2
:104DE0001400814201D9081A6080BDF80800BDF89E
:104DF0000410BDF816200144BDF812001044814291
:104E000001D9081AA080684609F0AAFEB8E71CB5C7
:104E10001F490968CDE90010684609F0AAFF04F0AF
:104E200025F91CBD1CB5002000900190684609F0D2
:104E3000A0FF04F01BF91CBD108008885080488832
:104E40009080C88810818888D0800020508190810F
:104E5000704710B5044604F075F830B1407830B1B1
:104E6000204604F07EFB002010BD052010BD12205E
:104E700010BD10B504F066F8040000D1FFDF6078C3
:104E800000B9FFDF6078401E607010BDD8010020BF
:104E90009C46020010B504F055F8040000D1FFDF75
:104EA0006078401C6070F0E71CB5ADF800008DF82C
:104EB00002308DF803108DF8042068460AF05EFD7C
:104EC00004F0D4F81CBD0CB52DA2D2E90012CDE936
:104ED00000120079694601EB501000780CBD027891
:104EE000520804D0012A02D043F202207047FEF794
:104EF00029BA10B548B183000022114605200FF0F1
:104F000017F9052801D00320BFE70020BDE71FB532
:104F10006A46FFF791FF68460AF04CF904F0A6F8DC
:104F200004B0B2E770B50C0006460DD0FEF793FA58
:104F3000050000D1FFDFA6802889208128896081B3
:104F40006889A081A889E081ADE510B500231A46E3
:104F500003E0845C2343521CD2B28A42F9D30BB1E2
:104F6000002092E7012090E700B530B1012803D07E
:104F7000022801D0FFDF002000BDFF2000BD00009F
:104F8000070605040302010010B504460FF0C6F938
:104F900008B1102010BD2078C0F30210042807D8F3
:104FA0006078072804D3A178102901D8814201D262
:104FB000072010BDE078410706D421794A0703D4C1
:104FC000000701D4080701D5062010BD002010BD40
:104FD00010B513785C08837F64F3C7138377137865
:104FE0009C08C37F64F30003C3771078C309487833
:104FF00063F34100487013781C090B7864F347137E
:105000000B701378DB0863F3000048705078487128
:1050100010BD10B5C4780B7864F300030B70C4782E
:10502000640864F341030B70C478A40864F382033A
:105030000B70C478E40864F3C3030B700379117830
:1050400063F30001117003795B0863F34101117090
:1050500003799B0863F3820111700079C00860F343
:10506000C301117010BD70B514460D46064604F01C
:10507000D1F980B10178182221F00F01891C21F0AB
:10508000F001A03100F8081B21461FF0D6F8BDE85A
:10509000704004F0C2B929463046BDE87040132282
:1050A000FEF7DCB92DE9F047064608A8894690E8E6
:1050B00030041F469046142128461FF01AF900219B
:1050C000CAF80010B8F1000F03D0B9F1000F03D1F6
:1050D00014E03878C00711D020680FF045F9C0BB44
:1050E000B8F1000F07D12068123028602068143012
:1050F00068602068A8602168CAF8001038788007C6
:1051000024D560680FF04EF918BBB9F1000F21D01B
:10511000FFF770F90168C6F868118188A6F86C116C
:10512000807986F86E0101F002FDF94FEF60626848
:1051300062B196F8680106F2691140081032FEF774
:1051400059F91022394660681FF032F80020BDE896
:10515000F08706E0606820B1E8606068C6F8640126
:10516000F4E71020F3E730B5054608780C4620F048
:105170000F00401C20F0F001103121700020607001
:1051800095F8230030B104280FD0052811D0062847
:1051900014D0FFDF20780121B1EB101F04D295F865
:1051A000200000F01F00607030BD21F0F0002030C2
:1051B00002E021F0F00030302070EBE721F0F00049
:1051C0004030F9E7F0B591B0022715460C46064687
:1051D0003A46ADF80870092103AB04F07AFF049059
:1051E000002810D004208DF804008DF80170E03400
:1051F000099605948DF818500AA968460DF0CAF86A
:1052000000B1FFDF012011B0F0BD10B588B00C4631
:105210000A99ADF80000C3B11868CDF802005868CB
:10522000CDF80600ADF80A20102203A81EF0C0FF3A
:1052300068460AF062F803F019FF002803D1A17F45
:1052400041F01001A17708B010BD0020CDF8020098
:10525000E6E72DE9F84F0646808A0D4680B2824681
:10526000FEF7F9F804463078DFF8A48200274FF003
:105270000509A8F120080F2870D2DFE800F06FF2CE
:105280003708387D8CC8F1F0EFF35FF3F300A07FAF
:1052900000F00300022809D05FF0000080F0010157
:1052A00050460BF085FB050003D101E00120F5E736
:1052B000FFDF98F85C10C90702D0D8F860000BE057
:1052C000032105F11D000EF004FDD5F81D009149E4
:1052D000B0FBF1F201FB1200C5F81D0070686867B1
:1052E000B068A8672078252800D0FFDFCAE0A07F3B
:1052F00000F00300022809D05FF0000080F00101F7
:1053000050460BF055FB060003D101E00120F5E704
:10531000FFDF3078810702D52178252904D040F0BD
:1053200001003070BDE8F88F02202870307F2871AE
:1053300006F11D002D36C5E90206F3E7A07F00F057
:105340000300022808D0002080F0010150460BF035
:105350002FFB040004D102E00120F5E7A7E1FFDF05
:105360002078C10604D5072028703D346C60D9E749
:1053700040F008002070D5E7E07F000700D5FFDF90
:10538000307CB28800F0010301B05046BDE8F04F18
:10539000092105F027BD04B9FFDF716821B1102292
:1053A00004F124001EF004FF28212046FDF7B2FE80
:1053B000A07F00F0030002280ED104F12400002396
:1053C00000901A4621465046FFF71FFF112807D0CC
:1053D00029212046FDF79EFE307A84F82000A1E7BF
:1053E000A07F000700D5FFDF14F81E0F40F0080073
:1053F0002070E782A761E761C109607861F341002D
:10540000014660F382016170307AE0708AE7A07F24
:1054100000F00300022809D05FF0000080F00101D5
:1054200050460BF0C5FA040003D101E00120F5E776
:10543000FFDF022104F185000EF04BFC04202870F0
:1054400004F5B4706860B4F88500288230481038DC
:105450007C346C61C5E9028064E703E024E15BE031
:105460002DE015E0A07F00F00300022807D0002007
:1054700080F0010150460BF09BFA18B901E00120C1
:10548000F6E7FFDF324621465046BDE8F84FEAE531
:1054900004B9FFDF20782128A1D93079012803D170
:1054A000E07F40F00800E077324621465046FFF7A3
:1054B000DAFD2046BDE8F84F2321FDF72BBE3279F7
:1054C000AA8005F108030921504604F002FEE860B5
:1054D00010B185F8009025E7A07F00F003000228B6
:1054E00008D0002080F0010150460BF061FA040062
:1054F00003D101E00120F5E7FFDF04F1620102239F
:105500001022081F0BF0DBF807703179417009E7B2
:105510003802002040420F00A07F00F00300022864
:1055200008D0002080F0010150460BF041FA050040
:1055300003D101E00120F5E7FFDF95F8840000F0DA
:10554000030001287AD1A07F00F00307E07F10F06C
:10555000010602D0022F04D133E095F8A000C00765
:105560002BD0D5F8601121B395F88320087C62F325
:1055700087000874A17FCA09D5F8601162F3410061
:105580000874D5F8601166F300000874AEB1D5F860
:105590006001102204F1240188351EF009FE287EE6
:1055A00040F001002876287820F0010005F88809ED
:1055B00000E016B1022F04D02DE095F88800C00756
:1055C00027D0D5F85C1121B395F88320087C62F3CD
:1055D00087000874A17FCA09D5F85C1162F3410005
:1055E0000874D5F85C1166F3000008748EB1D5F824
:1055F0005C01102204F1240188351EF0D9FD2878C1
:1056000040F0010005F8180B287820F0010005F89B
:10561000A009022F44D0002000EB400005EBC000A1
:1056200090F88800800709D595F87C00D5F86421AA
:10563000400805F17D011032FDF7DCFE8DF8009089
:1056400095F884006A4600F003008DF8010095F893
:1056500088108DF8021095F8A0008DF803002146FF
:10566000504601F04DFA2078252805D0212807D092
:10567000FFDF2078222803D922212046FDF74AFDAA
:10568000A07F00F0030002280CD0002080F0010170
:1056900050460BF09FF900283FF44FAEFFDF41E684
:1056A0000120B9E70120F1E7706847703AE6FFDFB3
:1056B00038E670B5FE4C002584F85C5025660CF089
:1056C00036FE04F11001204603F060FE84F83050ED
:1056D00070BD70B50D46FDF7BEFE040000D1FFDFC2
:1056E0004FF4B87128461EF004FE04F1240028612E
:1056F000A07F00F00300022808D0012105F1E0009E
:105700000CF016FE002800D0FFDF70BD0221F5E787
:105710000A46014602F1E0000CF02ABE70B50546CB
:10572000406886B001780A2906D00D2933D00E29A9
:105730002FD0FFDF06B070BD86883046FDF78BFEA8
:10574000040000D1FFDF20782128F3D028281BD1C6
:10575000686802210E3001F0C8F9A8B16868082114
:10576000801D01F0C2F978B104F1240130460AF03D
:10577000A2F803F07BFC00B1FFDF06B02046BDE8D5
:1057800070402921FDF7C6BC06B0BDE8704003F0AB
:1057900044BE012101726868C6883046FDF75BFE91
:1057A000040000D1FFDFA07F00F00301022902D135
:1057B00020F01000A077207821280AD06868017AAC
:1057C00009B1007980B1A07F00F00300022862D007
:1057D000FFDFA07F00F003000228ABD1FEF798F8AE
:1057E0000028A7D0FFDFA5E703F017FEA17F08067A
:1057F0002BD5E07FC00705D094F8200000F01F00F3
:10580000102820D05FF0050084F823002078292894
:105810001DD02428DDD1314604200EF033FD222195
:105820002046FDF777FCA07F00F00300022830D06F
:105830005FF0000080F0010130460BF0CBF800284B
:10584000C7D0FFDFC5E70620DEE70420DCE701F074
:105850000300022808D0002080F0010130460BF040
:10586000A7F8050003D101E00120F5E7FFDF2521BE
:105870002046FDF74FFC03208DF80000694605F136
:10588000E0000CF06CFD0228A3D00028A1D0FFDFBF
:105890009FE70120CEE703F0C0FD9AE72DE9F04332
:1058A00087B09946164688460746FDF7D4FD0400A2
:1058B0004BD02078222848D3232846D0E07F000709
:1058C00043D4A07F00F00300022809D05FF000005D
:1058D00080F0010138460BF06BF8050002D00CE0B7
:1058E0000120F5E7A07F00F00300022805D0012188
:1058F000002238460BF053F805466946284601F069
:1059000026F9009800B9FFDF45B10098E035056140
:105910002078222806D0242804D007E0009900200F
:10592000086103E025212046FDF7F4FB00980121E2
:1059300041704762868001A9C0E902890CF02AFD06
:10594000022802D0002800D0FFDF07B0BDE8F083B6
:1059500070B586B00546FDF77EFD017822291ED977
:10596000807F00F00300022808D0002080F00101B1
:1059700028460BF01DF804002FD101E00120F5E7C7
:10598000FFDF2AE0B4F85E0004F1620630440178DB
:10599000427829B121462846FFF714FCB0B9C9E680
:1059A000ADF804200921284602AB04F092FB0390D5
:1059B0000028F4D005208DF80000694604F1E000CD
:1059C0000CF0CDFC022801D000B1FFDF0223102231
:1059D000314604F15E000AF0A8FEB4F86000002829
:1059E000D0D1A7E610B586B00446FDF734FD0178A6
:1059F00022291BD9807F00F00300022808D0002054
:105A000080F0010120460AF0D3FF040003D101E039
:105A10000120F5E7FFDF06208DF80000694604F15C
:105A2000E0000CF09CFC002800D0FFDF06B010BDA9
:105A30002DE9F05F05460C460027007890460109E5
:105A40003E4604F1080BBA4602297DD0072902D050
:105A50000A2909D146E0686801780A2905D00D298C
:105A600030D00E292ED0FFDFBCE114271C26002CDD
:105A70006BD08088A080FDF7EEFC5FEA000900D1C2
:105A8000FFDF99F817005A46400809F11801FDF7A1
:105A9000B1FC6868C0892082696851F8060FC4F8B3
:105AA00012004868C4F81600A07E20F0060001E04D
:105AB0001802002040F00100A07699F81E0040F086
:105AC00020014DE01A270A26002CD1D0C088A080E2
:105AD000FDF7C1FC050000D1FFDF59462846FFF75E
:105AE00042FB7FE10CB1A88BA080287A0B287DD0E7
:105AF00006DC01287BD0022808D0032804D135E039
:105B00000D2875D00E2874D0FFDF6BE11E27092603
:105B1000002CADD0A088FDF79EFC5FEA000900D103
:105B2000FFDF287B00F003000128207A1BD020F043
:105B300001002072297B890861F341002072297BD2
:105B4000C90861F3820001E041E1F2E02072297BA3
:105B5000090961F3C300207299F81E0040F040016A
:105B600089F81E103EE140F00100E2E713270D2600
:105B7000002CAAD0A088FDF76EFC8146807F00F043
:105B80000300022808D0002080F00101A0880AF05C
:105B90000FFF050003D101E00120F5E7FFDF99F8D1
:105BA0001E0000F00302022A50D0686F817801F0D5
:105BB00003010129217A4BD021F001012172837860
:105BC0009B0863F3410121728378DB0863F3820150
:105BD000217283781B0963F3C3012172037863F395
:105BE00006112172437863F3C71103E061E0A9E075
:105BF00090E0A1E0217284F809A0C178A172022A84
:105C000029D00279E17A62F30001E1720279520847
:105C100062F34101E1720279920862F38201E1725A
:105C20000279D20862F3C301E1724279217B62F307
:105C3000000121734279520862F3410121734279D4
:105C4000920862F382012173407928E0A86FADE7E2
:105C500041F00101B2E74279E17A62F30001E172B9
:105C60004279520862F34101E1724279920862F38B
:105C70008201E1724279D20862F3C301E1720279D2
:105C8000217B62F3000121730279520862F3410122
:105C900021730279920862F3820121730079C008AE
:105CA00060F3C301217399F80000232831D926211C
:105CB00040E018271026E4B3A088FDF7CCFB83460C
:105CC000807F00F00300022809D0002080F001014D
:105CD000A0880AF06DFE5FEA000903D101E001200F
:105CE000F4E7FFDFE868A06099F8000040F00401E5
:105CF00089F8001099F80100800708D50120207369
:105D00009BF8000023286DD92721584651E084F8DC
:105D10000CA067E015270F265CB1A088FDF79BFB60
:105D2000814606225946E86808F059F90120A07317
:105D3000A2E041E048463CE016270926E4B3287B70
:105D400020724FE0287B19270E26ACB3C4F808A0B8
:105D5000A4F80CA0012807D0022805D0032805D0FC
:105D6000042803D0FFDF0DE0207207E0697B0428E0
:105D700001F00F0141F0800121721ED0607A20F005
:105D800003006072A088FDF766FB054600782128B5
:105D900028D0232800D0FFDFA87F00F003000228CE
:105DA00013D0002080F00101A0880AF013FE222108
:105DB0002846FDF7AFF915E004E0607A20F0030013
:105DC000401CDEE7A8F8006011E00120EAE70CB112
:105DD0006888A080287A03282ED004280AD00528B5
:105DE00050D0FFDFA8F800600CB12780668000204B
:105DF000BDE8F09F15270F26002CE3D0A088FDF703
:105E00002AFB807F00F00300022809D05FF0000029
:105E100080F00101A0880AF0CBFD050003D101E06C
:105E20000120F5E7FFDFD5F81D000622594608F0EE
:105E3000D6F884F80EA0D5E717270926002CC1D084
:105E4000A088FDF708FB8146807F00F00300022850
:105E500008D0002080F00101A0880AF0A9FD05000B
:105E600003D101E00120F5E7FFDF6878800701D565
:105E7000022000E00120207299F800002328B1D907
:105E8000272157E719270E26002C9BD0A088FDF765
:105E9000E2FA5FEA000900D1FFDFC4F808A0A4F825
:105EA0000CA084F808A0A07A40F00300A07299F832
:105EB0001E10C90961F38200A07299F81F2099F899
:105EC0001E1012EAD11F05D099F8201001F01F0111
:105ED00010292BD020F00800A07299F81F10607ACA
:105EE00061F3C3006072697A01F003010129A2D154
:105EF00040F00400607299F81E0000F003000228D0
:105F0000E87A16D0217B60F300012173AA7A607BC6
:105F100062F300006073EA7A520862F34101217370
:105F2000A97A490861F3410060735BE740F008001B
:105F3000D2E7617B60F300016173AA7A207B62F390
:105F400000002073EA7A520862F341016173A97A72
:105F5000490861F34100207344E710B5FE4C30B1AD
:105F60000146102204F120001EF022F9012084F8DD
:105F7000300010BD10B5044600F0D9FDF6492046AA
:105F80001022BDE8104020311EF012B970B5F24D5C
:105F900006004FF0000413D00EF0C0F908B1102431
:105FA0000CE00621304608F001F8411C05D02866B7
:105FB0005FF0010085F85C0000E00724204670BD1A
:105FC0000020F7E7007810F00F0204D0012A05D076
:105FD000022A0CD110E0000909D10AE000090128C9
:105FE00007D0022805D0032803D0042801D00720B9
:105FF00070470870002070470620704705282AD295
:10600000DFE800F003070F171F00087820F0FF00FB
:106010001EE0087820F00F00401C20F0F000103047
:1060200016E0087820F00F00401C20F0F00020302F
:106030000EE0087820F00F00401C20F0F000303017
:1060400006E0087820F00F00401C20F0F0004030FF
:10605000087000207047072070472DE9F041804606
:1060600088B00D46002708460EF0A5F9A8B94046AD
:10607000FDF7F1F9040003D02078222815D104E0BF
:1060800043F2020008B0BDE8F08145B9A07F4106A7
:1060900003D500F00300022801D01020F2E7A07F12
:1060A000C10601D4010702D50DB10820EAE7E17F5E
:1060B000090701D50D20E5E700F00300022805D10E
:1060C00025B12846FEF760FF0700DBD1A07F00F076
:1060D0000300022808D0002080F0010140460AF0A9
:1060E00067FC060002D00FE00120F5E7A07F00F07A
:1060F000030002280ED0002080F00101002240465B
:106100000AF04DFC060007D0A07F00F00300022833
:1061100004D009E00120EFE70420B3E725B12A46C7
:1061200031462046FEF754FF6946304600F00FFD29
:10613000009800B9FFDF0099022006F1E0024870E4
:10614000C1F824804A6100220A81A27F02F0030282
:10615000022A1CD001200871287800F00102087E74
:1061600062F3010008762A78520862F3820008760A
:106170002A78920862F3C30008762A78D20862F37C
:106180000410087624212046FCF7C4FF33E035B321
:106190000871301D88613078400908777078C0F345
:1061A00040004877287800F00102887F62F3010000
:1061B0008877A27FD20962F382008877E27F62F358
:1061C000C3008877727862F304108877A878C8775C
:1061D00001F1210228462031FEF71BFF03E00320D6
:1061E00008710520087625212046FCF793FFA07F43
:1061F00020F04000A07701A900980CF0CBF802280D
:1062000001D000B1FFDF38463CE72DE9FF4F534A8C
:106210000D4699B09A4607CA0BAB002783E80700E2
:106220001998FDF718F9060006D03078262806D010
:1062300008201DB0BDE8F08F43F20200F9E7B07FFF
:1062400000F00309B9F1020F03D00020284302D067
:1062500006E00120FAE71B98FEF796FE0028E8D139
:10626000B07F00F00300022801D11B9979BB0228FE
:1062700008D0002080F0010119980AF099FB040071
:1062800003D101E00120F5E7FFDF852D28D007DCF1
:10629000F5B1812D1ED0822D1ED0832D08D11DE099
:1062A000862D1FD0882D1FD0892D1FD08A2D1FD05D
:1062B0000F2020710F281DD003F0ACF8E0B10120B1
:1062C0008DF84000201D11902079B8B167E111E0F0
:1062D0000020EEE70120ECE70220EAE70320E8E7F0
:1062E0000520E6E70620E4E70820E2E70920E0E7EA
:1062F0000A20DEE707209CE711209AE7B9F1020F98
:1063000003D0A56F03D1A06F02E0656FFAE7606F5D
:10631000804632D04FF0010000904FF00200019013
:10632000214630461B9AFEF753FE1B98007800F07A
:106330000101A87861F30100A870B17FC90961F378
:106340008200A870F17F61F3C300A870617861F3E7
:106350000410A870207803E018020020A446020070
:10636000400928706078C0F3400068701B988078FE
:10637000E87000206871287103E00220009001207D
:106380000190A87898F80210C0F3C000C1F3C001D2
:1063900008405FEA000B2CD050460DF0BFFF90BBC9
:1063A000DAF80C000DF0BAFF68BBDAF81C000DF04B
:1063B000B5FF40BBDAF80C00A060DAF81C00E06022
:1063C00098F80100617800F0010041EA4000607037
:1063D00098F80210C0B2C1F30011891E0840607025
:1063E00000202077019906F1170002290CD0012125
:1063F0000BE098F80110607801F00101FD2242EAFB
:1064000041010840E3E732E0002104EB81014861EB
:106410000099701C022901D0012100E0002104EB49
:1064200081014861A87800F00300012858D198F84C
:10643000020000F00300012852D1B9F1020F04D08C
:106440002A1D691D1B98FEF7E4FD297998F80400C0
:1064500001408DF83810687998F8052010408DF8C3
:106460003C0001433CD050460DF058FF08B11020CD
:10647000DFE60AF110010491B9F1020F18D00846C5
:106480005FF0000104F18C03CDE9000304F5AE7266
:1064900002920EAB5A462046FEF704FE0028E7D1D2
:1064A000B9F1020F08D0504608D14FF0010107E0C2
:1064B00050464FF00101E5E70498F5E74FF0000181
:1064C00004F1A403CDE9000304F5B072029281F057
:1064D00001010FAB5A462046FEF7E4FD0028C7D164
:1064E0006078800734D4A87898F80210C0F3800050
:1064F000C1F3800108432BD0297898F800000BAA3B
:10650000B9F1020F06D032F811204300DA4002F050
:1065100003070AE032F810204B00DA4012F00307BC
:1065200005D0012F0BD0022F0BD0032F07D0BBF1CA
:10653000000F0DD0012906D0042904D008E002275D
:10654000F5E70127F3E7012801D0042800D104274B
:10655000B07F40F08000B077F17F6BF30001F177FE
:10656000607881074FF003000CD5A071BBF1000FDC
:1065700015D100BF8DF85C0017AA3146199800F0BC
:10658000BFFA0CE00221022F18D0012F18D0042FDF
:1065900022D00020A071B07F20F08000B0772521AC
:1065A0003046FCF7B7FD10A904F1E0000BF0D7FE70
:1065B00010B1022800D0FFDF00203AE6A171D9E730
:1065C000A1710D2104F120001DF093FE207840F010
:1065D000020020700420CDE70120A071DFE72DE943
:1065E000F04387B09046894604460025FCF733FF08
:1065F000060006D03078272806D0082007B0BDE86E
:10660000F08343F20200F9E7B07F00F003000228B4
:1066100008D0002080F0010120460AF0C9F90400EA
:1066200003D101E00120F5E7FFDFA7795FEA090068
:1066300005D0012821D0B9F1020F26D110E0B8F120
:10664000000F22D1012F05D0022F05D0032F05D036
:10665000FFDF2DE00C252BE0012529E0022527E0B6
:1066600040460DF05BFEB0B9032F0ED1102241461B
:1066700004F11D001DF09CFD1AE0012F02D0022F35
:1066800003D104E0B8F1000F12D00720B6E740466E
:106690000DF044FE08B11020B0E7102104F11D00F8
:1066A0001DF005FE0621404607F080FCC4F81D00E1
:1066B0002078252140F0020020703046FCF72AFDAA
:1066C0002078C10713D020F00100207002208DF83F
:1066D000000004F11D0002908DF804506946C3309B
:1066E0000BF03DFE022803D010B1FFDF00E025775C
:1066F000002083E730B587B00D460446FCF7ABFEBB
:10670000A0B1807F00F00300022812D05FF00000EB
:1067100080F0010120460AF04BF904000ED0284613
:106720000DF0FCFD38B1102007B030BD43F202007F
:10673000FAE70120ECE72078400701D40820F3E7CE
:10674000294604F13D00202205461DF031FD207848
:1067500040F01000207001070FD520F008002070D5
:1067600007208DF80000694604F1E00001950BF068
:10677000F6FD022801D000B1FFDF0020D4E770B59C
:106780000D460646FCF767FE18B10178272921D18E
:1067900002E043F2020070BD807F00F00300022897
:1067A00008D0002080F0010130460AF001F9040011
:1067B00003D101E00120F5E7FFDFA079022809D12C
:1067C0006078C00706D02A4621463046FEF7FAFC1C
:1067D00010B10FE0082070BDB4F860000E280BD295
:1067E00004F1620102231022081F09F068FF012151
:1067F00001704570002070BD112070BD70B5064657
:1068000014460D4608460DF089FD18B920460DF0D6
:10681000ABFD08B1102070BDA6F57F40FF380ED04B
:106820003046FCF718FE38B1417822464B08811CEF
:106830001846FCF7DFFD07E043F2020070BD20467A
:10684000FDF73EFE0028F9D11021E01D0DF041FAC0
:10685000E21D294604F1170000F089F9002070BDFF
:106860002DE9F04104468AB01546884600270846BF
:106870000DF0A1FD18B928460DF09DFD18B11020AE
:106880000AB0BDE8F0812046FCF7E5FD060003D024
:10689000307827281BD102E043F20200F0E7B07FF6
:1068A00000F00300022809D05FF0000080F0010131
:1068B00020460AF07DF8040003D101E00120F5E74D
:1068C000FFDF2078400702D56078800701D40820D8
:1068D000D6E7B07F00F00300022803D0A06F03D1F9
:1068E000A16F02E0606FFAE7616F407800B19DB17F
:1068F000487810B1B8F1000F0ED0ADB1EA1D06A86E
:10690000E16800F034F9102206A905F117001DF026
:1069100023FC18B1042707E00720B1E71022E91D86
:1069200004F12D001DF044FCB8F1000F06D0102238
:1069300008F1070104F11D001DF03AFC2078252123
:1069400040F0020020703046FCF7E4FB2078C107DD
:1069500015D020F00100207002208DF8000004F115
:106960001D000290103003908DF804706946B3301A
:106970000BF0F5FC022803D010B1FFDF00E0277711
:1069800000207DE7F8B515460E460746FCF763FD87
:10699000040004D02078222804D00820F8BD43F257
:1069A0000200F8BDA07F00F00300022802D043F2ED
:1069B0000500F8BD30460DF0B1FC18B928460DF0C1
:1069C000ADFC08B11020F8BD00953288B31C2146FB
:1069D0003846FEF71AFC112815D00028F3D1297C7F
:1069E0004A08A17F62F3C711A177297CE27F61F396
:1069F0000002E277297C890884F82010A17F21F029
:106A00004001A177F8BDA17F0907FBD4D6F80200A9
:106A1000C4F83600D6F80600C4F83A003088A086DC
:106A20001022294604F124001DF0C2FB287C4108F5
:106A3000E07F61F34100E077297C61F38200E07739
:106A4000287C800884F82100A07F40F00800A0770F
:106A50000020D3E770B50D4606460BB1072070BD88
:106A6000FCF7F9FC040007D02078222802D3A07F8D
:106A7000800604D4082070BD43F2020070BDADB1A1
:106A80002946304608F017FF02F0F0FA297C4A0840
:106A9000A17F62F3C711A177297CE27F61F3000235
:106AA000E277297C890884F8201004E0304608F059
:106AB0002AFF02F0DBFAA17F21F02001A17770BD4F
:106AC00070B50D46FCF7C7FC040005D028460DF054
:106AD0004BFC20B1102070BD43F2020070BD29466E
:106AE0002046FEF740FB002070BD04E010F8012BAB
:106AF0000AB100207047491E89B2F7D201207047C1
:106B000070B51546064602F085FC040000D1FFDF93
:106B1000207820F00F00801C20F0F0002030207042
:106B200066802868A060BDE8704002F076BC10B5B1
:106B3000134C94F83000002808D104F12001A1F191
:106B400010000BF04EFC012084F8300010BD10B195
:106B500090F8B9202AB10A4890F8350018B1002001
:106B600003E0B83001E0064834300860704708B5EB
:106B70000023009313460A460AF015F908BD0000E9
:106B80001802002018B18178012938D101E01020C5
:106B90007047018842F60112881A914231D018DC00
:106BA00042F60102A1EB020091422AD00CDC41B373
:106BB000B1F5C05F25D06FF4C050081821D0A0F502
:106BC0007060FF381BD11CE001281AD002280AD1BE
:106BD00017E0B0F5807F14D008DC012811D002281E
:106BE0000FD003280DD0FF2809D10AE0B0F5817F2E
:106BF00007D0A0F58070033803D0012801D0002011
:106C000070470F2070470A281ED007DC18D2DFE833
:106C100000F0191B1F1F171F231D1F21102815D03F
:106C200008DC0B2812D00C2810D00D2816D00F2805
:106C300006D10DE011280BD084280BD087280FD067
:106C400003207047002070470520704707207047D9
:106C50000F20704704207047062070470C207047B3
:106C600043F20200704738B50C46050041D0694632
:106C7000FFF7A8F9002819D19DF80010607861F39A
:106C8000020060706946681CFFF79CF900280DD16E
:106C90009DF80010607861F3C5006070A978C1F3B9
:106CA0004101012903D0022905D0072038BD2178F0
:106CB00021F0200102E0217841F0200121704107FC
:106CC00004D0A978C90861F386106070607810F06C
:106CD000380F07D0A978090961F3C710607010F068
:106CE000380F02D16078400603D5207840F040008C
:106CF0002070002038BD70B504460020088015467D
:106D00006068FFF7B0FF002816D12089A18988426A
:106D100011D860688078C0070AD0B1F5007F0AD822
:106D200040F20120B1FBF0F200FB1210288007E0D6
:106D3000B1F5FF7F01D90C2070BD01F2012129803E
:106D4000002070BD10B50478137864F3000313704D
:106D50000478640864F3410313700478A40864F3AE
:106D6000820313700478E40864F3C3031370047897
:106D7000240964F3041313700478640964F345135D
:106D800013700078800960F38613137031B10878AE
:106D9000C10701D1800701D5012000E0002060F388
:106DA000C713137010BD4278530702D002F00703D7
:106DB00006E012F0380F02D0C2F3C20300E0012354
:106DC0004A7863F302024A70407810F0380F02D01C
:106DD000C0F3C20005E0430702D000F0070000E066
:106DE000012060F3C5024A7070472DE9F04F95B05D
:106DF0000D00824612D0122128461DF058FA4FF697
:106E0000FF7B05AA0121584606F01BFF00242646F9
:106E100037464FF420586FF4205972E0102015B017
:106E2000BDE8F08F9DF81E0001280AD1BDF81C10A6
:106E300041450BD011EB09000AD001280CD00228E3
:106E40000CD0042C0ED0052C0FD10DE0012400E055
:106E50000224BDF81A6008E0032406E00424BDF80B
:106E60001A7002E0052400E00624BDF81A1051450E
:106E700047D12C74BEB34FF0000810AA4FF0070A98
:106E8000CDE90282CDE900A80DF13C091023CDF82F
:106E9000109042463146584606F086FF08BBBDF8C2
:106EA0003C002A46C0B210A90BF004FBC8B9AE8161
:106EB000CFB1CDE900A80DF1080C0AAE40468CE830
:106EC0004102132300223946584606F06DFF40B9AF
:106ED000BDF83C00F11CC01EC0B22A1D0BF0EAFA3E
:106EE00010B103209BE70AE0BDF82900E881062CD9
:106EF00005D19DF81E00A872BDF81C002881002055
:106F00008DE705A806F0A9FE00288BD0FFF77BFED1
:106F100085E72DE9F0471C46DDE90978DDF820908A
:106F200015460E00824600D1FFDF0CB1208818B153
:106F3000D5B11120BDE8F087022D01D0012100E07C
:106F4000002106F1140005F06BFDA8F800000246D0
:106F50003B462946504603F0BCF8C9F8000008B982
:106F6000A41C3C600020E5E71320E3E7F0B41446DE
:106F7000DDE904528DB1002314B1022C09D101E0E6
:106F8000012306E00D7CEE0703D025F00105012367
:106F90000D742146F0BC03F025BF1A80F0BC704789
:106FA0002DE9FE4F91461A881C468A468046FAB162
:106FB00002AB494603F08DF8050019D04046A61CE7
:106FC000278809F039FE3246072629463B460096B7
:106FD00009F047FA20882346CDE900504A46514639
:106FE0004046FFF7C3FF002020800120BDE8FE8F50
:106FF0000020FBE72DE9F04786B09146DDE90E461B
:107000000F46824603AA05A904A8109D8DE8070033
:107010009846324621465046FFF77BFF049909B156
:10702000012200E000222A70002818D1F94A03AB9F
:107030001060059A009104F11400CDE901204A4640
:107040003946504606F0A3F8A8B1092811D2DFE866
:1070500000F005080510100A0C0C0E00002006B008
:1070600068E71120FBE70720F9E70820F7E70D2084
:10707000F5E70320F3E7BDF80C100498CDE9000113
:107080004346324621465046FFF770FFE6E72DE9BA
:10709000F04389B00D46DDE9108781461C4616464F
:1070A000142103A81DF025F9012002218DF81010EC
:1070B0008DF80C008DF81170ADF8146064B1A278F1
:1070C000D20709D08DF81600E088ADF81A00A08824
:1070D000ADF81800A068079008A80095CDE9011048
:1070E000424603A948466B68FFF784FF09B0BDE834
:1070F000F083F0B58BB0002406460694079407276A
:10710000089405A80994019400970294CDE90340DE
:107110000D4610232246304606F046FE78B90AA8EE
:1071200006A9019400970294CDE90310BDF814302C
:1071300000222946304606F00DFC002801D0FFF75A
:1071400062FD0BB0F0BD06F0ADBA2DE9FC410C4676
:107150008046002602F05EF9054620780D287DD293
:10716000DFE800F0BC0713B325BD49496383AF9541
:107170009B00A848006820B1417841F0100141709F
:10718000ADE0404602F076F9A9E00421404609F05E
:107190000FFC070000D1FFDF07F11401404605F0A6
:1071A000D3FBA5BB13214046FDF748FC97E0042123
:1071B000404609F0FDFB070000D1FFDFE088ADF895
:1071C00000000020B8819DF80000010704D5C0062A
:1071D00002D5A088B88105E09DF8010040067ED563
:1071E000A088F88105B9FFDF22462946404601F014
:1071F00063FC022673E0E188ADF800109DF80110F1
:1072000009060FD5072803D006280AD00AE024E093
:107210000421404609F0CCFB060000D1FFDFA08826
:10722000F0810226CDB9FFDF17E00421404609F0C6
:10723000BFFB070000D1FFDF07F1140006F069FA79
:1072400090F0010F02D1E079000648D5387C022683
:1072500040F00200387405B9FFDF00E03EE022464E
:107260002946404601F028FC39E00421404609F057
:107270009FFB017C002D01F00206C1F3400161710A
:10728000017C21F002010174E7D1FFDFE5E702266E
:107290000121404602F020F921E00421404609F096
:1072A00087FB0546606800902089ADF80400012244
:1072B0006946404602F031F9287C20F0020028742B
:1072C0000DE0002DC9D1FFDFC7E7022600214046AF
:1072D000FBF788F8002DC0D1FFDFBEE7FFDF3046A7
:1072E000BDE8FC813EB50C0009D001466B4601AA01
:1072F000002006F0DBFD20B1FFF785FC3EBD10202D
:107300003EBD00202080A0709DF8050002A900F07D
:107310000700FEF773FE50B99DF8080020709DF835
:10732000050002A9C0F3C200FEF768FE08B1032001
:107330003EBD9DF8080060709DF80500C109A07869
:1073400061F30410A0709DF80510890961F3C30072
:10735000A0709DF80410890601D5022100E00121EA
:1073600061F342009DF8001061F30000A07000205E
:107370003EBD70B5144606460D4651EA040005D0E0
:1073800075B108460DF00EF878B901E0072070BD20
:107390002946304606F0EBFD10B1BDE8704032E4FE
:1073A00054B120460CF0FEFF08B1102070BD2146FC
:1073B0003046BDE8704095E7002070BD2DE9FC5FC8
:1073C0000C4690460546002701780822007A3E4682
:1073D000B2EB111F7ED104F10A0100910A31821E25
:1073E0004FF0020A04F1080B0191092A73D2DFE879
:1073F00002F0ECDF05F427277AA9CD006888042184
:1074000009F0D6FA060000D1FFDFB08920B152277B
:107410000726C2E07C02002051271026002C7DD0D8
:107420006888A0800120A071A88900220099FFF738
:10743000A0FF002873D1A8892081288AE081D1E0AB
:10744000B5F81290072824D1E87B000621D55127F2
:1074500009F1140086B2002CE1D0A889002200991D
:10746000FFF787FF00285AD16888A08084F806A01B
:10747000A88920810120A073288A2082A4F8129074
:10748000A88A009068884B46A969019A01F0F1FA30
:10749000A8E0502709F1120086B2002C3ED0A8893E
:1074A00000225946FFF765FF002838D16888A08080
:1074B000A889E080287A072813D002202073288A20
:1074C000E081E87BC0096073A4F81090A88A00905E
:1074D000688801E083E080E04B4604F11202A9696C
:1074E000D4E70120EAE7B5F81290512709F114001A
:1074F00086B2002C66D06888042109F059FA8346C8
:107500006888A080A88900220099FFF732FF002830
:107510006ED184F806A0A889208101E052E067E0DE
:107520000420A073288A2082A4F81290A88A0090D0
:1075300068884B46A969019A01F09BFAA989ABF8C2
:107540000E104FE06888FBF786FF07466888042125
:1075500009F02EFA064607B9FFDF06B9FFDF687BA0
:10756000C00702D05127142601E0502712264CB341
:107570006888A080502F06D084F806A0287B594642
:1075800001F087FA2EE0287BA11DF9E7FE49A889C2
:107590004989814205D1542706269CB16888A0807C
:1075A00020E053270BE06888A080A889E08019E0DC
:1075B0006888042109F0FCF900B9FFDF5527082687
:1075C000002CF0D1A8F8006011E056270726002C07
:1075D000F8D06888A080002013E0FFDF02E00128D7
:1075E00008D0FFDFA8F800600CB12780668000207B
:1075F000BDE8FC9F57270726002CE3D06888A080B1
:10760000687AA071EEE7401D20F0030009B1414304
:10761000091D01EB4000704713B5DB4A00201071D3
:10762000009848B10024684608F0DFFF002C02D122
:10763000D64A009911601CBD01240020F4E770B502
:107640000D46064686B014465C2128461CF051FEC5
:1076500004B9FFDFA0786874A2782188284601F079
:1076600042FA0020A881E881228805F11401304601
:1076700005F04FF96A460121304606F0E2FA19E0BA
:107680009DF80300000715D5BDF806103046FFF73A
:1076900030FD9DF80300BDF8061040F010008DF895
:1076A0000300BDF80300ADF81400FF233046059A2F
:1076B00006F028FC684606F0D0FA0028E0D006B0B4
:1076C00070BD10B50C4601F1140005F059F90146E2
:1076D000627C2046BDE8104001F03ABA70B505461C
:1076E000042109F065F9040000D1FFDF04F1140161
:1076F0000C46284605F028F921462846BDE870408A
:1077000005F029B970B58AB00C460646FBF7A3FE12
:10771000050014D02878222827D30CB1A08890B176
:1077200001208DF80C0003208DF8100000208DF84A
:10773000110054B1A088ADF81800206807E043F2AA
:1077400002000AB070BD0920FBE7ADF818000590F3
:107750000421304609F02CF9040000D1FFDF04F1C8
:10776000140005F024F9000701D40820E9E701F02E
:1077700051FE60B108A802210094CDE9011095F8EE
:10778000232003A930466368FFF734FCD9E71120B2
:10779000D7E72DE9F04FB2F802A0834689B015462D
:1077A00089465046FBF757FE07460421504609F02C
:1077B000FFF80026044605964FF002080696ADF83D
:1077C0001C6007B9FFDF04B9FFDF4146504603F0F4
:1077D00070FE50B907AA06A905A88DE80700424621
:1077E000214650466368FFF794FB674807AB066085
:1077F000DDE9051204F11400CDF80090CDE9032075
:10780000CDE9013197F82320594650466B6805F0C1
:1078100017F906000AD0022E04D0032E14D0042E2D
:1078200000D0FFDF09B03046BDE8F08FBDF81C0086
:107830000028F7D00599CDE9001042462146504670
:107840006368FFF793FBEDE7687840F00800687025
:10785000E8E72DE9F04F9BB004464FF000084A4896
:10786000ADF85480ADF83080ADF85080A0F80880B5
:10787000ADF81480ADF81880ADF82080ADF81C800C
:10788000007916460D464746012808D0022806D042
:10789000032804D0042802D008201BB0C4E72046E7
:1078A0000CF03CFDD0BB28460CF038FDB0BB606846
:1078B0000CF081FD90BB606848B1608921898842E5
:1078C00002D8B1F5007F01D90C20E6E780460BAA6B
:1078D00006A92846FFF70FFA0028DED168688078ED
:1078E000C0F34100022808D19DF8190010F0380FAC
:1078F00003D028690CF056FD80B905A92069FFF76F
:10790000B2F90028C9D1206950B1607880079DF88C
:10791000150000F0380002D5D0B301E011E0B8BB8B
:107920009DF8140080060ED59DF8150010F0380F54
:1079300003D060680CF036FD18B960680CF03BFDB0
:1079400008B11020A9E707A96069FFF78CF90028A2
:10795000A3D1606940B19DF81D0000F00701012925
:107960003FD110F0380F3CD008A9A069FFF77BF990
:10797000002892D19DF81C00800632D49DF820008A
:1079800080062ED4A06904E07C02002014000020B0
:1079900027E040B19DF8210000F00701012920D126
:1079A00010F0380F1DD0E06818B10078C8B11C285D
:1079B00017D20EAA611C2046FFF7C4F90120B94670
:1079C00060F30F27BA4607468DF84E0042F60300D3
:1079D000ADF84C000DF13B0217A928680AF089FDAB
:1079E00008B1072059E79DF85C0016A9CDF8009072
:1079F000C01CCDE9019100F0FF0B00230BF2012226
:107A0000514613A806F060F8F0BBBDF85800099085
:107A1000FE482A8929690092CDE901106B89BDF8D9
:107A20002C202868069906F04FF801007ED12078B6
:107A30004FF0020AC10601D480062BD5ADF80C9098
:107A4000606950B907A906A8FFF7ADF99DF81D00B8
:107A500020F00700401C8DF81D009DF81C008DF8DB
:107A60004E7040F0C8008DF81C0042F60210ADF8D0
:107A70004C000CA903AACDF800A0CDE901210023F8
:107A800040F2032213A800E01EE0079906F01CF85C
:107A900001004BD1DD484D4608385B460089ADF802
:107AA00039000EA8CDE90290CDF80490CDF81090E1
:107AB0004FF007090022CDF80090BDF858104FF69E
:107AC000FF7005F047FF10B1FFF79DF8E5E69DF860
:107AD0003800000625D52946012060F30F218DF8D6
:107AE0004E704FF42450ADF84C00ADF81050627851
:107AF0009DF81000002362F300008DF810006278FA
:107B0000CDF800A0520862F341008DF8100004AADD
:107B1000CDE9012540F2032213A805F0D5FF0100AD
:107B200004D1606888B32069A8B900E086E005A99F
:107B300006A8FFF738F96078800706D49DF815008D
:107B400020F038008DF8150005E09DF8140040F095
:107B500040008DF814008DF84E7042F60110ADF81B
:107B60004C00208940F20121B0FBF1F201FB12022E
:107B7000606814ABCDF80080CDE90103002313A8A1
:107B8000059905F0A1FF010058D12078C00729D040
:107B9000ADF80C50A06950B908A906A8FFF703F981
:107BA0009DF8210020F00700401C8DF821009DF871
:107BB00020008DF84E7040F040008DF8200042F615
:107BC0000310ADF84C0015A903AACDF800A0CDE92B
:107BD0000121002340F2032213A8089905F074FF45
:107BE00001002BD1E06868B32946012060F30F2122
:107BF0008DF84E7042F60410ADF84C00E06800239A
:107C000002788DF8602040788DF86100E06818AA4D
:107C10004088ADF86200E06800798DF86400E068A3
:107C2000C088ADF86500CDF80090CDE901254FF48E
:107C3000027213A805F048FF010003D0099800F074
:107C4000B3FF2AE6714803210838017156B1008953
:107C50003080BDF850007080BDF83000B080BDF8B5
:107C60005400F080002018E670B501258AB0164651
:107C70000B46012802D0022816D104E08DF80E50E0
:107C80004FF4205003E08DF80E5042F60100ADF89D
:107C90000C005BB10024601C60F30F2404AA08A947
:107CA00018460AF026FC18B107204AE5102048E5DE
:107CB00004A99DF820205548CDE90021801E02909E
:107CC0000023214603A802F2012205F0FDFE10B1B7
:107CD000FEF799FF35E54D4808380EB1C18831806F
:107CE000057100202DE5F0B593B0074601268DF80B
:107CF0003E6041F60100ADF83C0012AA0FA93046E3
:107D0000FFF7B2FF002848D1404C0025083CE7B3FC
:107D10001C2102A81CF0EDFA9DF808008DF83E60C9
:107D200040F020008DF8080042F60520ADF83C0038
:107D30000E959DF83A00119520F00600801C8DF8F4
:107D40003A009DF838006A4620F0FF008DF83800B0
:107D50009DF8390009A920F0FF008DF839000420B2
:107D6000ADF82C00ADF830000EA80A9011A80D90C7
:107D70000FA80990ADF82E5002A8FFF76AFD002861
:107D80000BD1BDF80000608100E008E0BDF8040000
:107D9000A081401CE0812571002013B0F0BD6581F9
:107DA000A581BDF84800F4E72DE9F74F1749A0B0C9
:107DB0000024083917940A79A146012A04D0022A1E
:107DC00002D0082023B02FE5CA88824201D00620C5
:107DD000F8E721988A46824201D10720F2E7012084
:107DE0002146ADF848004FF6FF7860F30F21ADF85B
:107DF0004A808DF86E0042F6020B06918DF87240B3
:107E0000ADF86CB0ADF870401CA901E08402002010
:107E10001391ADF8508012A805F043FF00252E46BF
:107E20002F460DAB072212A9404605F03DFF78B161
:107E30000A285DD195B38EB3ADF86450ADF8666095
:107E40009DF85E008DF8144019AC012864D06BE0F9
:107E50009DF83A001FB3012859D1BDF83810594593
:107E60001FD118A809A901940294CDE90310072095
:107E70000090BDF8361010230022404605F094FF14
:107E8000B0BBBDF86000042801D006284AD1BDF877
:107E90002410219881423AD10F2093E73AE001283B
:107EA00035D1BDF83800B0F5205F03D042F60101AE
:107EB00088422CD1BAF80600BDF83610884201D1AC
:107EC000012700E0002705B19EB1219881421ED113
:107ED00018A809AA01940294CDE903200720009074
:107EE0000D4610230022404605F05EFF00B902E077
:107EF0002DE04E460BE0BDF86000022801D01028AE
:107F000010D1C0B217AA09A90AF0D4FA50B9BDF825
:107F1000369086E7052055E705A917A8221D0AF027
:107F2000E8FA08B103204DE79DF814000023001D76
:107F3000C2B28DF8142022980092CDE901401BA80E
:107F4000069905F0C1FD10B902228AF80420FEF757
:107F50005AFE37E710B50B46401E88B084B205AA1A
:107F600000211846FEF7EEFE00200DF1080C06AACF
:107F700005A901908CE8070007200090012300224A
:107F800021464FF6FF7005F0E5FC0446BDF81800E9
:107F9000012800D0FFDF2046FEF735FE08B010BDF7
:107FA000F0B5FF4F044687B038790E46032804D059
:107FB000042802D0082007B0F0BD04AA03A9204677
:107FC000FEF799FE0500F6D160688078C0F34100A5
:107FD00002280AD19DF80D0010F0380F05D0206955
:107FE0000CF0E0F908B11020E5E7208905AA216925
:107FF0008DE807006389BDF810202068039905F01B
:1080000063FD10B1FEF7FFFDD5E716B1BDF8140012
:108010003080042038712846CDE7F8B50C000646BC
:108020000BD001464FF6FF7500236A46284605F03F
:108030003DFF20B1FEF7E7FDF8BD1020F8BD694611
:108040002046FEF710FE0028F8D1A078314600F057
:1080500001032846009A05F055FFEBE730B587B0DD
:10806000144600220DF1080C05AD01928CE82C009D
:10807000072200920A46014623884FF6FF7005F05A
:1080800069FCBDF814102180FEF7BDFD07B030BDBE
:1080900070B50D46042108F08BFC040000D1FFDF11
:1080A000294604F11400BDE8704004F079BC70B5B5
:1080B0000D46042108F07CFC040000D1FFDF2946B6
:1080C00004F11400BDE8704004F08DBC70B50D469D
:1080D000042108F06DFC040000D1FFDF294604F103
:1080E0001400BDE8704004F0A5BC70B5054604213D
:1080F00008F05EFC040000D1FFDF2146284623681B
:10810000BDE870400122FEF74BBF70B50646042162
:1081100008F04EFC040000D1FFDF04F1140004F06D
:108120002FFC401D20F0030511E0011D00880022F6
:10813000431821463046FEF733FF00280BD0607C01
:10814000ABB2684382B2A068011D08F0EEFAA068E5
:1081500041880029E9D170BD70B50546042108F0B9
:1081600027FC040000D1FFDF214628466368BDE8F4
:1081700070400222FEF714BF70B50E46054601F0AE
:1081800049F9040000D1FFDF01202072667265808A
:10819000207820F00F00001D20F0F000403020700B
:1081A000BDE8704001F039B910B50446012900D08E
:1081B000FFDF2046BDE810400121FAF713B92DE991
:1081C000F04F97B04FF0000A0C008346ADF814A0B2
:1081D000D04619D0E06830B1A068A8B10188ADF8E8
:1081E0001410A0F800A05846FBF735F9070043F239
:1081F000020961D0387822285CD30421584608F05F
:10820000D7FB050005D103E0102017B0BDE8F08FC3
:10821000FFDF05F1140004F0B3FB401D20F003065E
:10822000A078012803D0022801D00720EDE721889B
:1082300007AA584605F005FD30BB07A805F00DFD5F
:1082400010BB07A805F009FD48B99DF826000128D4
:1082500005D1BDF82400A0F52451023902D04FF415
:108260005050D2E7E068B0B1CDE902A007200090FD
:1082700005AACDF804A00492A2882188BDF8143084
:10828000584605F067FB10B1FEF7BDFCBDE7A168DD
:10829000BDF8140008809DF81F00C00602D543F207
:1082A0000140B2E70B9838B1A1780078012905D0D8
:1082B00080071AD40820A8E74846A6E7C007F9D0E7
:1082C00002208DF83C00A8684FF00009A0B1697C3D
:1082D0004288714391420FD98AB2B3B2011D08F0AE
:1082E000DAF98046A0F800A006E003208DF83C00F3
:1082F000D5F800804FF001099DF8200010F0380FEC
:1083000000D1FFDF9DF820002649C0F3C2000844D9
:1083100097F8231010F8010C884201D90F2074E758
:108320002088ADF8400014A90095CDE9019143469D
:1083300007220FA95846FEF75DFE002891D19DF84F
:10834000500050B9A078012807D1687CB3B27043BF
:1083500082B2A868011D08F0B2F9002055E770B597
:10836000064615460C460846FEF70CFC002805D1CB
:108370002A4621463046BDE8704075E470BD13E5DD
:1083800070B51E4614460D000ED06CB1616859B12F
:1083900060B10349C988814208D0072070BD000040
:1083A0007C020020FA2F00001020F7E72068FEF77B
:1083B000E9FB0028F2D1324621462846BDE870404C
:1083C000FFF747BA70B515460C0006D038B1FE4924
:1083D0000989814203D00720E0E71020DEE720680A
:1083E000FEF7D0FB0028D9D129462046BDE87040D1
:1083F000D6E570B5064686B00D46144610460BF01D
:10840000B3FFD0BB60680BF0D6FFB0BBA6F57F40D2
:10841000FF3803D03046FBF71EF880B12846694686
:10842000FEF7E3FC00280CD19DF810100F2008295E
:108430003CD2DFE801F008060606060A0A0843F205
:10844000020006B0AAE70320FBE79DF8021001290D
:1084500008D1BDF80010B1F5C05FF2D06FF4C05282
:10846000D142EED09DF8061001290DD1BDF80410BF
:10847000A1F52851062907D200E028E0DFE801F045
:10848000030304030303DCE79DF80A1001290ED15E
:10849000BDF80810B1F5245FD3D0A1F524510239FD
:1084A000CFD00129CDD0022901D1CAE7FFDF606812
:1084B00078B9002305AA2946304605F0F7FC10B12B
:1084C000FEF7A1FBBDE79DF81400800601D4102043
:1084D000B7E76188224628466368FFF7BFFDB0E72B
:1084E0002DE9F043814687B08846144610460BF0CC
:1084F0003BFF18B1102007B0BDE8F083002306AAA7
:108500004146484605F0D2FC18B100BFFEF77BFBA0
:10851000F1E79DF81800C00602D543F20140EAE7F2
:108520000025072705A8019500970295CDE903507E
:1085300062884FF6FF734146484605F035FC060059
:1085400013D160680BF010FF60B960680195CDE948
:10855000025000970495238862884146484605F0FA
:1085600023FC0646BDF8140020803046CEE739B122
:10857000954B0A889B899A4202D843F203007047C0
:108580001DE610B586B0904C0423ADF81430638915
:1085900043B1A4898C4201D2914205D943F2030030
:1085A00006B010BD0620FBE7ADF8101000210091C9
:1085B0000191ADF8003002218DF8021005A9029159
:1085C00004A90391ADF812206946FFF7F8FDE7E72B
:1085D0002DE9FC4781460E4608460BF09FFE88BBFE
:1085E0004846FAF738FF5FEA00080AD098F800001A
:1085F000222829D30421484608F0DAF9070005D1DA
:1086000003E043F20200BDE8FC87FFDF07F114003E
:1086100004F0CDF905463078012803D0022804D0B3
:108620000720F0E7A8070FD502E015F01C0F0BD0CC
:10863000B079341DC00709D0E08838B1A0680BF0CC
:108640006DFE18B11020DEE70820DCE732782088C4
:10865000002628B3A0F201130721112B18D20CD247
:10866000DFE803F00B090D0B1D0B121D100B0B1D8A
:108670001D1D1D0B1D00022A11D10846C3E7012A4A
:10868000FBD00CE02A0700E0EA06002AF5DA06E053
:10869000A0F5C0721F2A02D97D3A022AEDD8C6B2CF
:1086A00000F0B8FE50B198F82300CDE90006FA8931
:1086B000234639464846FEF7EAFCA4E71120A2E724
:1086C0002DE9F04F8BB01F4615460C468346002619
:1086D000FAF7C1FE28B10078222805D208200BB095
:1086E00094E543F20200FAE7B80801D00720F6E764
:1086F000032F00D100274FF6FF79CCB1022D73D3A1
:1087000020460BF058FE30B904EB0508A8F1010033
:108710000BF051FE08B11020E1E7AD1EAAB22146D0
:10872000484605F06DFC38F8021C88425CD1ADB2B9
:108730002549B80702D58889401C00E001201FFAAE
:1087400080F8F80701D08F8900E04F4605AA41461E
:10875000584605F076FA4FF0070A4FF00009ACB31F
:10876000204608E0408810283ED8361D304486B2A6
:10877000AE4239D2A01902884245F3D354E000BF7B
:108780009DF8170002074FD584B304EB0608361D89
:10879000B8F80230B6B2102B26D89A19AA4223D8BC
:1087A000B8F8002091421FD1C00620D5CDE900A91C
:1087B0000DF1080C0AAAA11948468CE80700B8F880
:1087C00000100022584603E07C0200202CE00BE061
:1087D00005F0C0F810B1FEF716FA80E7B8F802000D
:1087E000BDF82810884202D00B2078E704E0B8F8E2
:1087F0000200304486B206E0C00604D55846FEF7B3
:1088000078FC002888D19DF81700BDF81A1020F0D8
:1088100010008DF81700BDF81700ADF80000FF2319
:108820005846009A05F06EFB05A805F016FA18B92F
:10883000BDF81A10B942A3D90421584608F0B8F877
:10884000040000D1FFDFA2895AB1CDE900A94D464D
:10885000002321465846FEF71AFC0028BDD1A58109
:108860003DE700203BE72DE9FF4F8BB01E46170088
:108870000D464FF0000412D0B00802D007200FB010
:10888000C4E4032E00D100265DB108460BF08AFD3A
:1088900028B93888691E08440BF084FD08B11020FF
:1088A000EDE7C74AB00701D5D18900E00121F00703
:1088B0004FF6FF7802D0D089401E00E0404686B2D5
:1088C00006AA0B9805F0BDF94FF000094FF0070B11
:1088D0000DF1140A39E000BF9DF81B00000734D5E4
:1088E000CDF80490CDF800B0CDF80890CDE9039A0A
:1088F000434600220B9805F057FA60BB05B3BDF85C
:1089000014103A8821442819091D8A4230D3BDF831
:108910001E2020F8022BBDF8142020F8022BCDE9F0
:1089200000B9CDE90290CDF810A0BDF81E10BDF839
:10893000143000220B9805F037FA08B103209EE7A7
:10894000BDF814002044001D84B206A805F085F986
:1089500020B10A2806D0FEF756F990E7BDF81E10A0
:10896000B142B9D934B17DB13888A11C884203D253
:108970000C2084E7052082E722462946404605F080
:108980003FFB014628190180A41C3C80002076E7AB
:1089900010B504460BF0E8FC08B1102010BD884863
:1089A000C0892080002010BDF0B58BB00D46064672
:1089B000142103A81BF09DFC01208DF80C008DF8FC
:1089C000100000208DF81100ADF814503046FAF771
:1089D00042FD48B10078222812D30421304607F026
:1089E000E7FF040005D103E043F202000BB0F0BD45
:1089F000FFDF04F11400074603F0D9FF800601D41D
:108A00000820F3E7207C022140F00100207409A82F
:108A10000094CDE90110072203A930466368FEF7F0
:108A2000E9FA20B1217C21F001012174DEE7294619
:108A30003046F9F7C8FC08A9384603F0A7FF00B193
:108A4000FFDFBDF82040172C01D2172000E02046A0
:108A5000A84201D92C4602E0172C00D21724214647
:108A60003046FFF724FB21463046F9F7D2F90020C3
:108A7000BCE7F8B51C4615460E46069F08F0CAF836
:108A80002346FF1DBCB231462A46009407F0B5FCD0
:108A9000F8BD70B50C4605460E2120461BF007FCBC
:108AA000002020802DB1012D01D0FFDF76E40620CB
:108AB00000E00520A07171E410B5488008781346E5
:108AC00020F00F00001D20F0F00080300C460870F0
:108AD0001422194604F108001BF0AFFB00F09DFCC6
:108AE0003748046010BD2DE9F047DFF8D890491DE4
:108AF000064621F0030117460C46D9F8000007F09E
:108B000092FD050000D1FFDF4FF000083560A5F8A9
:108B100000802146D9F8000007F085FD050000D14E
:108B2000FFDF7560A5F800807FB104FB07F1091D28
:108B30000BD0D9F8000007F076FD040000D1FFDF6C
:108B4000B460C4F80080BDE8F087C6F80880FAE792
:108B50002DE9F0411746491D21F00302194D064643
:108B600001681446286807F089FD22467168286864
:108B700007F084FD3FB104FB07F2121D03D0B1687A
:108B8000286807F07BFD042007F0BAFE04460420A5
:108B900007F0BEFE201A012804D12868BDE8F04184
:108BA00007F036BDBDE8F08110B50C4605F015F8AC
:108BB00000B1FFDF2046BDE81040FEF724B80000FA
:108BC0007C0200201400002038B50C468288817B8E
:108BD00019B14189914200D90A462280C188121DEB
:108BE00090B26A4606F092FFBDF80000032800D359
:108BF0000320C1B2208800F0A3FF38BD38B50C4671
:108C00008288817B19B10189914200D90A4622806C
:108C1000C188121D90B26A4606F078FFBDF80000C8
:108C2000022800D30220C1B2208800F089FF401C36
:108C3000C0B238BD2DE9FE4F0C46FD4981464022A9
:108C4000D1E90201CDE9010109F1030020F003019E
:108C5000C91C21F0030100916846114607F0C5FCCC
:108C6000F44E002C02D1F44A00999160009901441D
:108C70000091357F05F1010504D1E8B209F0C0FB90
:108C800000B1FFDF009800EB0510C01C20F00301CD
:108C900000915CB9707AB27A1044C2B200200870B8
:108CA000308C80B204F021FE00B1FFDF0098316A01
:108CB000084400902146684600F00DFF0098C01C53
:108CC00020F003000090B37AF27A717A04B10020A8
:108CD00007F081FD0099084400902146684600F0A5
:108CE0003AFF00273D46B24696F801800CE0284640
:108CF00000F0D4FE064681788088F9F721F9717872
:108D00006D1C00FB0177EDB24545F0D10098C01C09
:108D100020F00300009004B100203946F9F71BF958
:108D200000990027084400903D469AF801800CE025
:108D3000284600F0B3FE0646C1788088FEF763FC43
:108D400071786D1C00FB0177EDB24545F0D10098BC
:108D5000C01C20F00300009004B100203946FEF74B
:108D60005BFC00994FF000080844009045469AF8D3
:108D700001700EE0284600F091FE0646807B30B17F
:108D800006F1080001F0DDFE727800FB02886D1C20
:108D9000EDB2BD42EED10098C01C20F0030000905F
:108DA00004B10020414601F0D0FE00990844009033
:108DB0002146684600F049FE0098C01D20F00702D9
:108DC00000922CBB9D490020FAF747F8FBF715FBF2
:108DD000984801AA00211030F8F7CEFA00B1FFDF61
:108DE0009AF81D00FEF77FFF00B1FFDF91484FF4B6
:108DF000F67144301BF07DFA8E480421443080F82F
:108E0000E91180F8EA11062180F8EB1103210171C4
:108E10000099A1EB0900BDE8FE8F70B5854C0646B0
:108E20004434207804EB4015E078083590B9A01957
:108E300090F8E80100280ED0A0780F2800D3FFDFBB
:108E4000202128461BF055FA687866F30200687006
:108E50000120E070284670BD2DE9F04105460C4622
:108E600000270078052190463E46B1EB101F00D048
:108E7000FFDF287A50B101280ED0FFDFA8F800608C
:108E80000CB1278066800020BDE8F081012709260B
:108E900074B16888A08008E00227142644B168886D
:108EA000A0802869E060A88A2082287B2072E5E7FC
:108EB000A8F80060E7E710B55F4C6068C11D21F0BD
:108EC0000701814200D0FFDF5A48012100220170D2
:108ED00042700172417203238372C1720273027481
:108EE000052202831F224283417455A242610A2255
:108EF000027741774FF4B06101626168416010BD53
:108F000030B54D4C1568636810339D4202D2042081
:108F1000136030BD474B5D785A6802EB0512107044
:108F200051700320D080172090800120D070907065
:108F3000002090735878401C587060681030606052
:108F4000002030BD70B506463A480024457807E059
:108F5000204600F0A3FD0178B14204D0641CE4B2C5
:108F6000AC42F5D1002070BDF7B5074608780C4635
:108F700010B3FFF7E7FF0546A7F12006202F06D024
:108F8000052E19D2DFE806F00F2B2B151A0000F082
:108F900090FD0DB1697800E00021401AA17880B2FF
:108FA0000844FF2808D8A07830B1A088022824D22D
:108FB00002E06088172820D20720FEBD207AE0B1A9
:108FC00061881729F8D3A1881729F5D3A179002939
:108FD000F2D0E1790029EFD0402804D9ECE7242F22
:108FE0000BD1207A48B161884FF6FB70814202D8DC
:108FF000A188814201D90420FEBD65B9207802AA6A
:109000000121FFF77DFF0028F6D12078FFF79AFFB6
:10901000050000D1FFDF052E25D2DFE806F003189A
:109020001B151E00A0786870A088E8801CE0000076
:10903000B0460200980300201C0000200000002021
:109040006E524635780000006088A8800CE0A07859
:10905000A87009E0A078E87006E054F8020FA86054
:109060006068E86000E0FFDF0020FEBD1A2835D010
:109070000DDC132832D2DFE800F01B31203131271C
:109080002723252D313129313131312F0F0030285F
:1090900002D003DC1E2821D1072070473A38092866
:1090A0001CD2DFE800F0151B0F1B1B1B1B1B07004E
:1090B0000020704743F20400704743F202007047FB
:1090C000042070470D2070470F207047082070471C
:1090D0001120704713207047062070470320704707
:1090E00010B5007800F0010006F001FDBDE8104069
:1090F000BCE70EB5017801F001018DF80010417850
:1091000001F001018DF801100178C1F340018DF8E3
:1091100002104178C1F340018DF8031001788908ED
:109120008DF80410417889088DF8051081788DF844
:109130000610C1788DF8071000798DF80800684690
:1091400005F0ACFAFFF792FF0EBD2DE9F84FDFF8FE
:10915000F883FE4C00261FE0012000F03FFD0120B7
:10916000FFF75BFE054640214746D8F8080007F0A8
:109170005AFA686000B9FFDF686805F03EF8A8B1E8
:109180002846FAF75AFC284600F02EFD20B9402266
:109190006968B86807F072FA94F9E9010428DBDA23
:1091A000022007F0ADFB07460025A6E040226968D3
:1091B000D8F8080007F062FAF2E7B8F80210404663
:1091C000491C89B2A8F80210B94201D3002141809C
:1091D0000221B8F8020007F0EBFB002865D0B8F8D0
:1091E0000200694606F0F1FBFFF740FF00B1FFDF28
:1091F0009DF8000078B1B8F8020007F01DFD5FEAA5
:10920000000900D1FFDF484606F08BFF18B1B8F81F
:10921000020002F03DF9B8F8020007F0FBFC5FEA3B
:10922000000900D1FFDF484606F073FFE8BB0321C9
:10923000B8F8020007F0BCFB5FEA000B48D1FFDF83
:1092400046E000BFDBF8100010B10078FF2849D0DD
:10925000022000F0C3FC0220FFF7DFFD82464846F3
:1092600007F063F8CAF8040000B9FFDFDAF8040079
:1092700007F02BF9002100900170B8F80210504659
:10928000AAF8021001F00AFE484607F020F900B9DA
:10929000FFDF504600F0A8FC18B99AF8010000075B
:1092A00004D50099CBF8101012E024E0DBF8100090
:1092B00038B10178491C11F0FF01017008D1FFDFBE
:1092C00006E000221146484600F0BDFB00B9FFDF72
:1092D00094F9EA01022805DBB8F8020001F0A3FDC9
:1092E0000028AFD194F9E901042804DB484607F0CF
:1092F00052F900B101266D1CEDB2BD4204D294F9C1
:10930000EA010228BFF659AF002E7FF423AFBDE873
:10931000F84F032000F062BC10B58B4CE060086889
:109320002061AFF2D91002F012FD607010BD8748C5
:1093300000214438017084480170854941607047BC
:1093400070B505464FF080500C46D0F8A410491C6B
:1093500005D1D0F8A810C9430904090C0BD050F866
:10936000A01F01F001012970416821608068A08080
:10937000287830B970BD062120460AF0AAFC0120E9
:109380002870607940F0C000607170BD70B54FF01A
:1093900080540D46D4F88010491C0BD1D4F88410A9
:1093A000491C07D1D4F88810491C03D1D4F88C107B
:1093B000491C0CD0D4F880100160D4F884104160AE
:1093C000D4F888108160D4F88C10C16002E01021BC
:1093D0000AF07FFCD4F89000401C0BD1D4F8940024
:1093E000401C07D1D4F89800401C03D1D4F89C004D
:1093F000401C09D054F8900F286060686860A0682D
:10940000A860E068E86070BD2846BDE870401021A3
:109410000AF05FBC4D480079FFE470B54B4CE07832
:1094200030B3207804EB4010407A00F0070020446D
:1094300090F9E801002800DCFFDF2078002504EB2C
:109440004010407A00F00700011991F8E801401E31
:1094500081F8E8012078401CC0B220700F2800D1AC
:109460002570A078401CA0700AF096FBE57070BDD6
:10947000FFDF70BD3EB50546032107F099FA0446AB
:10948000284607F0C7FB054604B9FFDF206918B17D
:109490000078FF2800D1FFDF01AA6946284600F0C6
:1094A000D2FA60B9FFDF0AE0002202A9284600F0E4
:1094B000CAFA00B9FFDF9DF8080000B1FFDF9DF890
:1094C0000000411E8DF80010EED2206901998842FB
:1094D00001D1002020613EBD70B50546A0F57F405A
:1094E0000C46FF3800D1FFDF012C01D0FFDF70BD3B
:1094F000FFF790FF040000D1FFDF207820F00F007D
:10950000401D20F0F0005030207065800020207257
:1095100001202073BDE870407FE72DE9F041164639
:109520000D460746FFF776FF040000D1FFDF2078E5
:1095300020F00F00401D20F0F000503020706780B8
:1095400001202072286805E01C000020DC030020B8
:10955000C81400202061A888A0822673BDE8F041CD
:109560005BE77FB5FFF7EEFC040000D1FFDF02A947
:109570002046FFF729FB054603A92046FFF73EFBDF
:109580008DF800508DF80100BDF80800001DADF801
:109590000200BDF80C00001DADF80400E088ADF835
:1095A0000600684606F08CFA002800D0FFDF7FBD79
:1095B0002DE9F047DFF8FC930546002799F80000F5
:1095C00010B10820BDE8F08728460AF0CDFE08B1AA
:1095D0001020F7E7F84C207808B9FFF76CFCA07A68
:1095E000617A0844C6B200F064FAB04207D2301A79
:1095F000C1B22A460020FFF783FC0700E2D1D9F868
:1096000004004E46C01C20F00300C9F8040000F01E
:1096100040FB716800EB010801214046FFF70AFB9F
:10962000064629684044884202D8B6F5803F15D3E3
:1096300028600020FFF786FC05000DD005F113001F
:10964000D9F8041020F003004E46884200D0FFDF16
:109650006078401E607075600420B3E700214046CA
:10966000FFF7E8FA0446A64200D0FFDF04EB08014A
:10967000C9F8041029604FF6FF71A9F80210012102
:1096800089F8001038469DE72DE9F0410446C948A5
:1096900017460E46007810B10820BDE8F081084654
:1096A0000AF03CFE08B11020F7E7C34D287808B94E
:1096B000FFF701FC601E1E2807D8012C22D130784C
:1096C000FE281FD828770020E7E7A4F120001F28F4
:1096D00005D8E0B23A463146BDE8F04144E4A4F191
:1096E00040001F2805D831462046BDE8F04100F073
:1096F000A3BAA4F1A0001F2804D80020A02C03D0F6
:10970000A12C06D00720C8E7317801F00101697764
:10971000C3E731680922F82901D38B0701D010462D
:10972000BBE76B7C03F00303012B04D16B8BD733B6
:109730009CB28C42F3D82962AFE72DE9F04781460D
:109740000E4608460AF010FE48B948460AF02AFEBE
:1097500028B909F1030020F00301494501D0102088
:1097600030E795484FF0000A4430817869B141787C
:10977000804600EB411408343788324600212046E9
:1097800000F040FA050004D027E0A6F800A005206C
:1097900018E7B9F1000F24D03088B84201D90C2560
:1097A0001FE0607800F00705284600F017FA08EB84
:1097B0000507324697F8E8014946401C87F8E8015A
:1097C000204607F5F47700F01DFA05463878401E6C
:1097D0003870032000F002FA2DB10C2D01D0A6F84C
:1097E00000A02846EEE66078724E00F007010129DD
:1097F00023D002290CD0032933D0FFDF98F80110C1
:109800004046491CC9B288F801100F2934D035E010
:10981000616821B1000702D46088FFF72BFE98F839
:10982000EA014746012802D1707802F0AFFA97F9B1
:10983000EA010428E2DBFFDFE0E7616819B14022BA
:10984000B06806F01BFF98F8E9014746032802D1EB
:10985000707802F09BFA97F9E9010428CEDBFFDF6C
:10986000CCE7C00602D56088FFF704FE98F9EB014B
:109870000628C3DBFFDFC1E780F801A08178491E1D
:109880008170617801F0070101EB080090F8E811A0
:10989000491C80F8E811A4E770B50D4604460AF0AB
:1098A0003DFD18B928460AF05FFD08B1102070BDD3
:1098B00029462046BDE8704008F0D9BD70B5044681
:1098C00015460E4608460AF029FD18B928460AF042
:1098D0004BFD08B1102070BD022C03D0102C01D01C
:1098E000092070BD2A463146204608F0E3FD0028D5
:1098F000F7D0052070BD70B514460D4606460AF037
:109900000DFD38B928460AF02FFD18B920460AF097
:1099100049FD08B1102070BD22462946304608F0A6
:10992000E8FD0028F7D0072070BD3EB504460AF0D8
:109930001BFD08B110203EBD684604F00FFEFFF786
:1099400095FB0028F7D19DF806002070BDF80800AF
:109950006080BDF80A00A08000203EBD70B50546BD
:109960000C4608460AF01EFD20B93CB120680AF0FA
:10997000FBFC08B1102070BDA08828B12146284604
:10998000BDE87040FDF7BEBE092070BD70B504464D
:109990000D4608460AF0C2FC30B9601E1E2818D8D1
:1099A00028460AF0BBFC08B1102070BD022C05D976
:1099B000072070BD1C0000209803002004B9FFDFC1
:1099C000F94800EB840050F8041C2846BDE87040BC
:1099D0000847A4F120001F2805D829462046BDE8E5
:1099E0007040FAF792BCF02CE2D1A8680AF096FC1D
:1099F0000028D9D1284606F0CBF8BDE87040FFF723
:109A000035BB70B504460D4608460AF0ADFC30B9CA
:109A1000601E1E280DD828460AF080FC08B11020D0
:109A2000C7E7012C01D0022C01D10620C1E7072095
:109A3000BFE7A4F120001F28F9D829462046BDE839
:109A40007040FAF7BABC06F033BB38B50446D748C5
:109A5000007B00F00105D9B9F9F78BFA0DB1226846
:109A600000E00022D2484178C06804F06EFBD04884
:109A70001030C0788DF8000010B1012802D004E049
:109A8000012000E000208DF80000684604F0DFFDB2
:109A9000002D02D020682830206038BD30B5C34D7D
:109AA00004466878A04200D8FFDF686800EB041025
:109AB00030BD70B5BD4800252C46467807E02046ED
:109AC000FFF7ECFF4078641C2844C5B2E4B2B4420E
:109AD000F5D128466DE72DE9F0410C46064600F029
:109AE00006F907463068C01C20F00302326014BB40
:109AF000AE483B46082124300AF0EAFA002409E087
:109B0000082C10D2DFE804F0060408080A04040652
:109B1000A84804E0A84802E0A84800E0A8480AF0E5
:109B2000F7FA054600E0FFDFA54200D0FFDF641C26
:109B3000E4B2082CE4D3306800EB07103060ACE5E9
:109B4000021D5143452900D245210844C01CB0FBE9
:109B5000F2F0C0B270472DE9FC5F064693484FF023
:109B600000088B464746444690F8019022E0204684
:109B7000FFF794FF050000D1FFDF6878694638449D
:109B8000C7B22846FFF720F8824601A92846FFF70A
:109B900035F80346BDF804005246001D81B2BDF8F9
:109BA0000000001D80B206F081FF6A78641C00FB93
:109BB0000288E4B24C45DAD13068C01C20F00300C2
:109BC0003060BBF1000F00D000204246394606F05D
:109BD0007BFF316808443060BDE8FC9F7349443125
:109BE00008710020C870704770494431CA782AB1A2
:109BF0000A7801EB42110831814201D001207047FF
:109C0000002070472DE9F04106460078154600F027
:109C10000F0400201080601E0F46052800D3FFDFD0
:109C200061482A46103000EB8400394650F8043C65
:109C30003046BDE8F041184770B50C46402802D0C8
:109C4000412806D120E0A07861780D18E1788142A2
:109C500001D90720ADE62078012801D91320A8E614
:109C6000FF2D08D808F0B0FD064609F04CFF301A69
:109C7000801EA84201DA12209BE64C4821688160D0
:109C800021790173002094E6BDE87040084600F099
:109C90005EB82DE9F0470027DFF810A13E463D46AB
:109CA000B9463C469AF801800AE02046FFF7F6FEE6
:109CB0004178807B0E4410FB0155641CE4B27F1C8C
:109CC0004445F2D109EB8700C6EBC60100EB8100E9
:109CD0009AF8092000EB850101EBC2019AF80A20ED
:109CE0009AF80B0001EBC20101EB80006AE42DE958
:109CF000F047DFF8B8900026344699F8090099F843
:109D00000A2099F801700244D5B299F80B2010444A
:109D100000F0FF0808E02046FFF7C0FE817B407896
:109D200011FB0066641CE4B2BC42F4D199F809004E
:109D300099F80A10284428444044401C01B10121EC
:109D400008448419FF2C00D9FFDFE0B23AE438B5AB
:109D50000446407800F00300012803D002280BD00D
:109D6000072038BD606858B10AF025FBD0B960689B
:109D70000AF018FB20B915E060680AF0CFFA88B93C
:109D800069462046FCF71EF90028EAD1607800F009
:109D90000300022816D19DF8000098B160680AF00F
:109DA00001FB78B1102038BDB046020098030020B6
:109DB0001C000020B941000017AC00005D2F00001E
:109DC000F32101006189F8290DD8208988420AD839
:109DD000607800F003020A48012A06D1D731026AEE
:109DE00089B28A4201D20920DDE794E80E0000F131
:109DF000100585E80E000AB9002101830020D2E792
:109E0000980300202DE9F04107461446884608468D
:109E100001F01CFD064608EB88001C22796802EB65
:109E2000C0000D18688C58B14146384601F016FD47
:109E3000014678680078C200082305F120000CE094
:109E4000E88CA8B14146384601F00FFD014678681C
:109E500008234078C20005F1240006F066FC38B102
:109E6000062121726681D0E90010C4E9031009E0DF
:109E7000287809280BD00520207266816868E06088
:109E8000002028702046BDE8F04101F0D5BC072035
:109E900020726681F4E72DE9F04116460D4607462B
:109EA000406801EB85011C2202EBC10144182046E9
:109EB00001F0FDFC40B10021708865F30F2160F3D3
:109EC0001F4107200AF0DEF909202070324629469A
:109ED0003846BDE8F04195E72DE9F0410E460746CA
:109EE00000241C21F07816E004EB8403726801EB77
:109EF000C303D25C6AB1FFF78DFA050000D1FFDF22
:109F00006F802A4621463046FFF7C5FF0120BDE895
:109F1000F081641CE4B2A042E6D80020F7E770B5F7
:109F2000064600241C21C0780AE000BF04EB84032D
:109F3000726801EBC303D5182A782AB1641CE4B215
:109F4000A042F3D8402070BD282128461AF0AFF96E
:109F5000706880892881204670BD70B50346002056
:109F60001C25DC780DE000BF00EB80065A6805EB8D
:109F7000C6063244167816B1128A8A4204D0401CB2
:109F8000C0B28442F0D8402070BDF0B50446002035
:109F90001C26E5780EE000BF00EB8007636806EB47
:109FA000C7073B441F788F4202D15B78934204D0AD
:109FB000401CC0B28542EFD84020F0BD0078032895
:109FC00001D000207047012070470078022801D09E
:109FD00000207047012070470078072801D000203A
:109FE0007047012070472DE9F041064688461078F9
:109FF000F1781546884200D3FFDF2C781C27641CBB
:10A00000F078E4B2A04201D8201AC4B204EB840173
:10A01000706807EBC1010844017821B141468847C7
:10A0200008B12C7073E72878A042E8D1402028704E
:10A030006DE770B514460B880122A240134207D188
:10A0400013430B8001230A22011D06F038FB047024
:10A0500070BD2DE9FF4F81B00878DDE90E7B9A468F
:10A0600091460E4640072CD4019806F0E5FD040009
:10A0700000D1FFDF07F1040820461FFA88F105F040
:10A0800024FF050000D1FFDF204629466A4606F07E
:10A090006EF90098A0F80370A0F805A0284606F015
:10A0A00014FA017869F306016BF3C71101702046B9
:10A0B0001FFA88F105F04CFF00B9FFDF019803F0AB
:10A0C000B9FF06EB0900017F491C017705B0BDE827
:10A0D000F08F2DE9F84F0E469A4691460746032128
:10A0E00006F066FC0446008DDFF8B485002518B143
:10A0F00098F80000B0421ED1384606F09DFD0700DA
:10A1000000D1FFDF09F10401384689B205F0DDFE18
:10A11000050010D0384629466A4606F028F900980E
:10A1200000210A460180817004F054F80098C01D97
:10A13000CAF8000021E098F80000B04216D104F1FE
:10A14000260734F8341F012000FA06F911EA090F36
:10A1500000D0FFDF2088012340EA090020800A2286
:10A16000391D384606F0C6FA067006E0324604F19C
:10A17000340104F12600FFF75CFF0A2188F8001083
:10A180002846BDE8F88FFEB514460D46064602ABDC
:10A190000C220621FFF79DFF002826D0029968783F
:10A1A00012220A70801C487008224A80A8702088F9
:10A1B00088806088C880A0880881E0884881002461
:10A1C0000C20CDE900040523062229463046FFF77E
:10A1D00040FF2146002266F31F41F023104609F09C
:10A1E000A7FF6878801C68700120FEBDFEB514468C
:10A1F0000D460622064602AB1146FFF76AFF00280D
:10A2000012D0029B132000211870A87858700220E9
:10A2100058809C800620CDE900010246052329468E
:10A220003046FFF716FF0120FEBD2DE9FE430C4628
:10A23000804644E002AB0E2207214046FFF749FF6B
:10A24000002841D060681C2267788678BF1C06EB26
:10A25000860102EBC1014518029814210170477074
:10A260000A214180698A0181E98A4181A988818026
:10A27000A9898181304601F0E9FA02990523072274
:10A28000C8806F700420287000250E20CDE90005DD
:10A2900021464046FFF7DDFE294666F30F2168F3AD
:10A2A0001F41F0230022072009F042FF6078FD499A
:10A2B000801C607062682046921CFFF794FE606804
:10A2C00080784028B6D10120BDE8FE83FEB50D465A
:10A2D000064638E002AB0E2207213046FFF7F9FEB2
:10A2E000002835D068681C23C17801EB810203EB9C
:10A2F000C2028418029815220270627842700A2203
:10A300004280A2894281A2888281084601F09EFA99
:10A31000014602988180618AC180E18A0181A0881A
:10A32000B8B10020207000210E20CDE900010523E6
:10A33000072229463046FFF78CFE6A68DA4928462C
:10A34000D21CFFF750FE6868C0784028C2D10120B7
:10A35000FEBD0620E6E72DE9FE430C46814644E0BB
:10A36000204601F08EFAD0B302AB082207214846FE
:10A37000FFF7AFFE0028A7D060681C226578067939
:10A38000AD1C06EB860102EBC10147180298B7F835
:10A39000108006210170457004214180304601F093
:10A3A00055FA0146029805230722C180A0F80480CF
:10A3B0007D70082038700025CDE90005214648460B
:10A3C000FFF747FE294666F30F2169F31F41F0238B
:10A3D0000022072009F0ACFE6078801C6070626883
:10A3E000B2492046121DFFF7FEFD60680179402941
:10A3F000B6D1012068E72DE9F34F83B00E4680E027
:10A40000304601F03EFA002875D071681C2091F8A2
:10A41000068008EB880200EBC2000C18414630466B
:10A4200001F023FA0146A078C30070684078C200AA
:10A4300004F1240006F095F907468088E18B401A64
:10A4400080B2002581B3AA46218B814200D80846FC
:10A450008146024602AB07210398FFF73AFE01004E
:10A4600028D0BAF1000F03D0029AB88802251080D4
:10A470008B46E28B3968A9EB05001FFA80FA0A4483
:10A480000398009206F0D8FBED1D009A59465346FA
:10A49000009505F0E6FFE08B504480B2E083B98878
:10A4A000884209D1012508E0FFE7801C4FF0010A2E
:10A4B00080B2C9E7002009E60025CDE90095238A8E
:10A4C000072231460398FFF7C4FDE089401EE08172
:10A4D0008DB1A078401CA0707068F178427811FBB3
:10A4E00002F1CAB2816901230E3006F0E8F880F863
:10A4F00000800020E08372686D493046921DFFF7AE
:10A5000072FD7068817940297FF47AAF0120DDE522
:10A5100070B5064648680D4614468179402910D129
:10A5200004EB84011C2202EBC101084401F0E0F9B4
:10A53000002806D06868294684713046BDE870401E
:10A5400059E770BDFEB50C460746002645E020469B
:10A5500001F097F9D8B360681C22417901EB8101C1
:10A5600002EBC1014518688900B9FFDF02AB082280
:10A5700007213846FFF7ADFD002833D002996078F7
:10A5800016220A70801C4870042048806068407958
:10A5900001F05CF901460298052307228180698950
:10A5A000C1800820CDE9000621463846FFF751FD5D
:10A5B0006078801C6070A88969890844B0F5803F84
:10A5C00000D3FFDFA88969890844A8816E81626889
:10A5D00038492046521DFFF706FD60684179402941
:10A5E000B5D10120FEBD30B5438C458BC3F3C70404
:10A5F000002345B1838B641EED1AC38A6D1E1D4472
:10A6000095FBF3F3E4B22CB1008918B1A04200D855
:10A61000204603444FF6FF70834200D30346138065
:10A620000C7030BD2DE9FC41074616460D464868C2
:10A6300002EB86011C2202EBC10144186A4601A903
:10A640002046FFF7D0FFA089618901448AB2BDF896
:10A650000010914212D0081A00D50020608168686D
:10A66000407940280AD1204601F038F9002805D069
:10A670006868294646713846FFF764FFBDE8FC81EB
:10A680002DE9FE4F8946804615465088032106F085
:10A690008FF98346B8F8020040280DD240200CE024
:10A6A00030000020BD9F0000CB9F0000D99F00001C
:10A6B000F1B80000DDB80000403880B282460146A3
:10A6C000584601F0DEF800287ED00AEB8A001C22F2
:10A6D000DBF8041002EBC0000C18204601F0E7F88C
:10A6E000002877D1B8F80000E18A88423CD8A189D7
:10A6F000D1B348456ED100265146584601F0AEF818
:10A70000218C0F18608B48B9B9F1020F62D3B8F8E9
:10A7100004006083618A884226D80226A9EB0600DD
:10A720001FFA80F9B888A28B801A002814DD4946E8
:10A73000814500DA084683B2688869680291396801
:10A740000A44CDE9003206F065FADDE90121F61D83
:10A75000009B009605F051FEA18B01EB090080B231
:10A76000A083618B884207D9688803B05246594656
:10A77000BDE8F04F01F0D9B81FD14FF009002872A1
:10A78000B8F802006881D7E90001C5E90401608BCF
:10A79000A881284601F050F85146584601F05EF86D
:10A7A0000146DBF8040008230078C20004F1200011
:10A7B00005F0BBFF0020A0836083A0890AF0FF02A0
:10A7C000401EA081688800E004E003B05946BDE85F
:10A7D000F04F27E7BDE8FE8F2DE9F041064615460C
:10A7E0000F461C46184609F099FD18B9206809F073
:10A7F000BBFD08B1102015E47168688C0978B0EBD6
:10A80000C10F01D313200DE43946304601F026F87C
:10A810000146706808230078C20005F1200005F0A9
:10A820004EFFD4E90012C0E900120020E3E710B5A2
:10A830000446032106F0BCF80146007800F003004E
:10A84000022805D02046BDE8104001F114029AE428
:10A850008A8A2046BDE81040C8E470B5044603214A
:10A8600006F0A6F8054601462046FFF774FD0028CD
:10A8700016D029462046FFF765FE002810D029464D
:10A880002046FFF723FD00280AD029462046FFF77F
:10A89000CCFC002804D029462046BDE87040AAE53B
:10A8A00070BD2DE9F0410C4680461EE0E17842780B
:10A8B00011FB02F1CAB2816901230E3005F035FFA8
:10A8C000077860681C22C179491EC17107EB8701B6
:10A8D000606802EBC10146183946204600F0D1FFFE
:10A8E00018B1304600F0DCFF20B16068C179002962
:10A8F000DCD180E7FEF78EFD050000D1FFDF0A20E6
:10A900002872384600F0A2FF68813946204600F0E0
:10A91000ACFF0146606808234078C20006F12400BD
:10A9200005F003FFD0E90010C5E90310A5F8028087
:10A93000284600F081FFB07800B9FFDFB078401EF4
:10A94000B07058E770B50C460546032106F030F8A4
:10A9500001464068C2792244C2712846BDE8704071
:10A960009FE72DE9FE4F8246507814460F464FF080
:10A97000000800284FD0012807D0022822D0FFDF8E
:10A980002068B8606068F86024E702AB0E220821F6
:10A990005046FFF79EFB0028F2D0029815210523B0
:10A9A0000170217841700A214180C0F80480C0F80C
:10A9B0000880A0F80C80628882810E20CDE9000812
:10A9C000082221E0A678304600F040FF054606EB5D
:10A9D00086012C22786802EBC1010822465A02AB9C
:10A9E00011465046FFF775FB0028C9D00298072191
:10A9F0000170217841700421418008218580C68042
:10AA0000CDE9001805230A4639465046FFF721FBD9
:10AA100087F80880DEE6A678022516B1022E13D04C
:10AA2000FFDF2A1D914602AB08215046FFF751FB7C
:10AA30000028A5D002980121022E017021784170D2
:10AA40004580868002D005E00625EAE7A188C1801E
:10AA5000E1880181CDE90098052308223946504656
:10AA6000D4E710B50446032105F0A2FF014600F12A
:10AA700008022046BDE8104073E72DE9F05F0C4660
:10AA800001281DD0957992F80480567905EB85014F
:10AA90001F2202EBC10121F0030B08EB060111FBA1
:10AAA00005F14FF6FF7202EAC10909F1030115FB36
:10AAB0000611F94F21F0031A40B101283DD124E0DD
:10AAC0006168E57891F800804E78DFE7594678684C
:10AAD00005F0A9FD606000B9FFDF5946606819F014
:10AAE00008FCE5705146786805F09DFD6168486195
:10AAF00000B9FFDF6068426902EB090181616068AB
:10AB000080F800806068467017E0606852464169CE
:10AB1000786805F0B3FD5A466168786805F0AEFDC7
:10AB2000032005F0EDFE0446032005F0F1FE201A97
:10AB3000012802D1786805F06BFD0BEB0A00BDE837
:10AB4000F09F02460021022097E773B5D24D0A20FC
:10AB50002870009848B100244FEA0D0005F045FD2B
:10AB6000002C01D1009969607CBD01240020F5E72B
:10AB700070B50C4615463821204619F0BAFB01265F
:10AB800066700A2104F11C0019F0B3FB05B9FFDF60
:10AB9000297A207861F301002070A879002817D065
:10ABA0002A4621460020FFF768FF61684020887030
:10ABB0006168C8706168087161684871616888710E
:10ABC0006168288808816168688848816068868132
:10ABD00070BDC878002802D0002201204DE77047E0
:10ABE00070B50546002165F31F41002009F04AFBBE
:10ABF0000321284605F0DCFE040000D1FFDF2146DA
:10AC00002846FFF769F9002804D0207840F01000AA
:10AC10002070012070BD2DE9FF4180460E460F0CCB
:10AC2000FEF7F8FB050007D06F800321384605F0DA
:10AC3000BFFE040008D106E004B03846BDE8F0418C
:10AC40001321F9F7FBBEFFDF5FEA080005D0B8F17A
:10AC5000070F18D0FFDFBDE8FF8120782A4620F0DB
:10AC6000080020700020ADF8020002208DF80000DE
:10AC70004FF6FF70ADF80400ADF80600694638469F
:10AC8000F9F7EFFAE7E7C6F3072101EB81021C238E
:10AC9000606803EBC202805C042803D008280AD055
:10ACA000FFDFD8E7012000904FF440432A462046BA
:10ACB00000F004FECFE704B02A462046BDE8F0418C
:10ACC000FFF7E9B82DE9F05F0027B0F80A90904649
:10ACD0000C4605463E46B9F1400F01D2402001E046
:10ACE000A9F140001FFA80FA287AC01E08286BD20A
:10ACF000DFE800F00D04192058363C477227102673
:10AD0000002C6CD0D5E90301C4E902015CE0702796
:10AD10001226002C63D00A2205F10C0104F1080070
:10AD200019F08BFA50E071270C26002C57D0E868F8
:10AD3000A06049E0742710269CB3D5E90301C4E95B
:10AD400002016888032105F033FE8346FEF762FBAB
:10AD500002466888508051465846FFF753F833E062
:10AD600075270A26ECB1A88920812DE076271426C4
:10AD7000BCB105F10C0004F1080307C883E8070023
:10AD800022E07727102664B1D5E90301C4E9020166
:10AD90006888032105F00CFE01466888FFF781FDF5
:10ADA00012E01CE073270826CCB16888032105F067
:10ADB000FFFD01460078C00606D56888FFF78CF8CD
:10ADC00010B96888F8F71DFEA8F800602CB127803C
:10ADD000A4F8069066806888A0800020AFE6A8F8F6
:10ADE0000060FAE72DE9FC410C461E4617468046F6
:10ADF000032105F0DDFD05460A2C0AD2DFE804F048
:10AE000005050505050509090907042303E00623CF
:10AE100001E0FFDF0023CDE90076224629464046C7
:10AE2000FFF717F92AE438B50546A0F57F40FF384B
:10AE300030D0284605F0EEFE040000D1FFDF2046AA
:10AE400005F073FA002815D001466A46204605F041
:10AE50008EFA00980321B0F80540284605F0A8FDB9
:10AE60000546052C03D0402C05D2402404E0007A8E
:10AE700080B1002038BD403CA4B2214600F001FD65
:10AE800040B1686804EB84013E2202EBC101405AE4
:10AE90000028EFD0012038BD300000202DE9F04F10
:10AEA000044689B0408805F0B5FE050000D1FFDFFB
:10AEB00006AA2846616800F0BDFC069D001F81B20D
:10AEC00035F8032F6B888A4205D1042B0AD0052B55
:10AED0001DD0062B15D022462846FFF7D1FB09B01E
:10AEE000BDE8F08F16462D1D224629463046F7F75D
:10AEF00054FA0828F3D1224629463046FCF749FC8B
:10AF0000EDE76088291D6368FAF7C8FCE7E7174694
:10AF10006088032105F04CFD4FF000088DF8048097
:10AF20000646ADF80680042FD9D36A79002AD6D018
:10AF300028794FF6FF794FF01C0A13282CD008DC33
:10AF4000012878D0062847D0072875D0122874D158
:10AF500006E0142872D0152871D016286DD1ACE106
:10AF60000C2F6AD1307800F00301022965D140F03E
:10AF7000080030706879B07001208DF804002889CD
:10AF8000ADF808006889ADF80A00A889ADF80C0092
:10AF9000E889ADF80E0019E0B07890429FD1307882
:10AFA00001079CD5062F9AD120F0080030706088E8
:10AFB000414660F31F41002009F064F902208DF83A
:10AFC0000400ADF808902889ADF80A006088224690
:10AFD00001A9F9F746F982E7082F80D12F89B5F842
:10AFE0000A90402F01D2402001E0A7F1400080B23A
:10AFF00080460146304600F044FC08B3716808EB17
:10B0000088002C2202EBC000095A4945E3D1FE48D2
:10B0100007AAD0E90210CDE9071068798DF81C0065
:10B0200008F0FF058DF81E5060883146FFF799FC47
:10B030002246294639E0B6E014E03CE039E0E6E09B
:10B04000F148D0E90010CDE907106879ADF820701B
:10B050008DF81C00ADF82290608807AA3146FFF7F2
:10B0600080FC3CE7082FB6D16889B5F808804028F5
:10B0700001D2402000E0403887B23946304600F027
:10B0800000FC0028A7D007EB870271680AEBC2001A
:10B090000844028A42459ED1017808299BD1407814
:10B0A0006979884297D1F9B222463046FEF7F3FE1D
:10B0B00015E70E2F07D0CDF81C80CDF820806879D9
:10B0C0008DF81C00C8E76989EF898B46B5F80C90AC
:10B0D0003046FEF742FFABF14001402901D3092081
:10B0E0004AE0B9F1170F01D3172F01D20B2043E02B
:10B0F00040280ED000EB800271680AEBC2000844C1
:10B100000178012903D1407869798842A9D00A20C1
:10B1100032E03046FEF703FF014640282BD001EB1A
:10B12000810372680AEBC30002EB0008012288F871
:10B1300000206A7988F8012070682A894089B8421D
:10B1400000D938462D8A03232372A282E781208208
:10B15000A4F80C906582084600F078FB6081A8F89E
:10B160001490A8F81870A8F80E50A8F810B020464F
:10B1700000F062FBB3E6042005212172A4F80A80E6
:10B18000E08101212173A049D1E90421CDE9072102
:10B1900069798DF81C10ADF81E00608807AA314649
:10B1A000FFF7DFFBE3E7062FE4D3B078904215D139
:10B1B0003078010712D520F00800307060884146D1
:10B1C00060F31F41002009F05DF802208DF80400B3
:10B1D0002889ADF80800ADF80A90F7E6042130465A
:10B1E000FEF7D3FE05464028C4D00220830300901A
:10B1F00022462946304600F061FB4146608865F3EF
:10B200000F2160F31F41072009F03CF867E60E2F7D
:10B21000B0D104213046FEF7B8FE81464028A9D0BF
:10B220004146608869F30F2160F31F41072009F050
:10B2300029F8288A0790E88900907068AF894089CA
:10B24000B84200D938468346B5F80A802889059067
:10B25000484600F0FBFA6081079840B10220079B46
:10B26000009022464946304600F028FB37E6B8F108
:10B27000170F1ED3172F1CD3042020720098608252
:10B28000E781A4F810B0A4F80C8009EB890271687A
:10B290000AEBC2000D1800990598A5F81480A5F8CE
:10B2A00018B0E9812882204600F0C6FA06202870EE
:10B2B00015E601200B230090D3E7082FA6D129899A
:10B2C0003046FEF74AFE074640289FD007EB87022C
:10B2D00071680AEBC2000844804600F0E8FA0028D2
:10B2E00094D16D89B8F80E002844B0F5803F05D39D
:10B2F00060883A46314600F018FBF0E5002D85D015
:10B30000A8F80E0060883A463146FFF701F9082098
:10B310002072384600F09AFA6081A58127E770B55F
:10B320000D460646032105F043FB040004D02078B7
:10B33000000704D5112070BD43F2020070BD2A46FB
:10B3400021463046FEF71FFF18B92868606168681B
:10B35000A061207840F008002070002070BD70B51A
:10B360000D460646032105F023FB040004D0207897
:10B37000000704D4082070BD43F2020070BD2A46C5
:10B3800021463046FEF732FF00B9A582207820F032
:10B3900008002070002070BD2DE9F04F0E4691B0DE
:10B3A0008046032105F004FB0446404605F044FCBA
:10B3B00007460020079008900990ADF830000A90E9
:10B3C00002900390049004B9FFDF0DF1080917BB48
:10B3D000FFDF20E038460BA9002204F069FE9DF84B
:10B3E0002C0000F07F050A2D00D3FFDF6019017FDC
:10B3F000491E01779DF82C0000060CD52A460CA9A1
:10B4000007A8FEF716FE01E0D846020019F805105D
:10B41000491C09F80510761EF6B2DBD204F134009F
:10B42000FA4D04F1260BDFF8E8A304F12A07069091
:10B4300010E05846069900F06AFA064628700A2875
:10B4400000D3FFDF5AF8261040468847E08CC05DE5
:10B45000B04202D0208D0028EBD10A202870EC4D9C
:10B460004E4628350EE00CA907A800F050FA044615
:10B47000375D55F8240000B9FFDF55F82420394620
:10B4800040469047BDF81E000028ECD111B027E5DA
:10B4900010B5032105F08CFA040000D1FFDF0A216A
:10B4A00004F11C0018F025FF207840F00400207003
:10B4B00010BD10B50C46032105F07AFA2044007F38
:10B4C000002800D0012010BD2DE9F84F894615460F
:10B4D0008246032105F06CFA070004D0284608F0E4
:10B4E0001DFF40B903E043F20200BDE8F88F484673
:10B4F00008F03AFF08B11020F7E7786828B16988AA
:10B500000089814201D90920EFE7B9F800001C2425
:10B5100018B1402809D2402008E03846FEF7FFFC69
:10B520008046402819D11320DFE7403880B280469A
:10B530000146384600F0A5F948B108EB8800796863
:10B5400004EBC000085C012803D00820CDE70520EB
:10B55000CBE7FDF75FFF06000BD008EB88007968AA
:10B5600004EBC0000C18B9F8000020B1E88910B154
:10B5700013E01120B9E72888172802D36888172814
:10B5800001D20720B1E7686838B12B1D2246414639
:10B590003846FFF721F90028A7D104F10C026946CB
:10B5A0002046FFF720F8288860826888E082B9F892
:10B5B000000030B102202070E889A080E889A0B1A5
:10B5C0002BE003202070A889A0807868817840292A
:10B5D00005D180F8028039465046FEF726FE4046E7
:10B5E00000F034F9A9F8000021E07868218B408947
:10B5F000884200D908462083A6F802A004203072B1
:10B60000B9F800007081E0897082F181208B30826E
:10B61000A08AB081304600F00FF97868C1784029DF
:10B6200005D180F8038039465046FEF74FFE0020D2
:10B630005BE770B50D460646032105F0B9F9040035
:10B6400003D0402D04D2402503E043F2020070BD38
:10B65000403DADB2294600F014F958B105EB850123
:10B660001C22606802EBC101084400F020F918B107
:10B67000082070BD052070BD2A462146304600F0E6
:10B6800054F9002070BD2DE9F0410D461646804664
:10B69000032105F08DF90446402D01D2402500E03C
:10B6A000403DADB28CB1294600F0EBF880B105EB1E
:10B6B00085011C22606802EBC1014718384600F082
:10B6C000F6F838B10820BDE8F08143F20200FAE74D
:10B6D0000520F8E733463A4629462046FFF77CF82E
:10B6E0000028F0D1EAB221464046FEF79BFF002039
:10B6F000E9E72DE9F0410D4616468046032105F0A5
:10B7000057F90446402D01D2402500E0403DAFB23C
:10B7100024B1304608F002FE38B902E043F20200DC
:10B72000D1E7306808F0FAFD08B11020CBE73946C0
:10B73000204600F0A6F860B107EB87011C22606884
:10B7400002EBC1014518284600F0B1F818B10820F5
:10B75000B9E70520B7E7B088A98A884201D90C204B
:10B76000B1E76168E88C4978B0EBC10F01D31320D1
:10B77000A9E73946204600F078F8014660680823BA
:10B780004078C20005F1240004F099FFD6E90012C8
:10B79000C0E90012FAB221464046FEF7B9FE002089
:10B7A00091E72DE9F0470D461F469046814603215B
:10B7B00005F0FEF80446402D01D2402001E0A5F13D
:10B7C000400086B23CB14DB1384608F0EBFD50B1B7
:10B7D0001020BDE8F08743F20200FAE76068C8B1C4
:10B7E000A0F80C8024E03146204600F04AF888B1E9
:10B7F00006EB86011C22606802EBC1014518284651
:10B8000000F055F840B10820E3E7000030000020C8
:10B81000F04602000520DCE7A5F80880F2B22146D8
:10B820004846FEF7FFFE1FB1A889698908443880A1
:10B830000020CEE704F09BBD017821F00F01491CE8
:10B8400021F0F00110310170FDF7E7BD10B504469D
:10B85000402800D9FFDF4034A0B210BD40684269E3
:10B860000078484302EBC0007047C2784068037814
:10B8700012FB03F24378406901FB032100EBC10096
:10B880007047C2788A4209D9406801EB81011C22C5
:10B8900002EBC101405C08B10120704700207047F5
:10B8A0000078062801D901207047002070470078F1
:10B8B000062801D00120704700207047F0B401EB4A
:10B8C00081061C27446807EBC6063444049D052600
:10B8D0002670E3802571F0BCFEF794BA10B541895B
:10B8E00011B1FFF7DDFF08B1002010BD012010BD30
:10B8F00010B5C18C8278B1EBC20F04D9C18911B1E6
:10B90000FFF7CEFF08B1002010BD012010BD10B51B
:10B910000C4601230A22011D04F007FF007821884C
:10B92000012282409143218010BDF0B402EB8205D8
:10B930001C264C6806EBC505072363554B681C792C
:10B94000402C03D11A71F0BCFEF705BDF0BC704766
:10B9500010B5EFF3108000F0010472B6EE484178A4
:10B96000491C41704078012801D1F7F70DFB002CEC
:10B9700000D162B610BD70B5E74CE07848B901253A
:10B98000E570FFF7E5FFF7F707FB20B1002008F0AF
:10B990000AF9002070BD4FF080406571C0F8045373
:10B9A000F7E770B5EFF3108000F0010572B6DA4CDE
:10B9B000607800B9FFDF6078401E6070607808B979
:10B9C000F7F7E6FA002D00D162B670BDD24810B587
:10B9D000C17821B100214171C170FFF7E2FF002061
:10B9E00010BD10B50446F7F7D7FACB49C97808401F
:10B9F00000D001202060002010BD2DE9F05FDFF8AD
:10BA000018934278817889F80620002589F8071074
:10BA1000064689F8085000782F4620B101280FD03B
:10BA200002280FD0FFDFF7F7C4FA98B1F7F7C8FA8A
:10BA3000A8420FD12846F7F7C7FA0028FAD047E006
:10BA40000125F0E7FFF784FFF7F7A6FA0028FBD0FF
:10BA50000225E8E701208407E060C4F80471AF49DB
:10BA60000D600107D1F84412AC4AC1F342312432CF
:10BA70001160AA49343108604FF0020BC4F804B3D6
:10BA8000A060DFF89CA2DAF80010C94341F300116E
:10BA900001F10108DAF8001041F01001CAF80010B5
:10BAA00000E020BFD4F804010028FAD02846F7F7B8
:10BAB0008BFA0028FAD0B8F1000F05D1DAF800109F
:10BAC00021F01001CAF80010C4F808B3C4F80471DA
:10BAD00099F807004C4670B1307860B9F7F75CFA16
:10BAE000064608F0BDF96FF0004116B1C4E9031035
:10BAF00001E0C4E9030115B12771BDE8F09F012001
:10BB00002071BDE8F05F00F0ABB870B5050000D162
:10BB1000FFDF4FF080424FF0FF30C2F808030021F2
:10BB2000C2F80011C2F80411C2F80C11C2F81011C9
:10BB3000794C6170F7F736FA10B10120E07060704F
:10BB40002846BDE8704058E72DE9F05F7548D0F809
:10BB500000B0744A7449083211608406D4F80801B0
:10BB600008B1012600E00026D4F8000110B14FF022
:10BB7000010801E04FF00008D4F8040108B10127E2
:10BB800000E00027D4F80C0100B101208246D4F86F
:10BB9000100108B1012100E00021894646EA0801B0
:10BBA00027EA010020EA0A0030EA090000D0FFDF9E
:10BBB000002526B1C4F80851012007F0F4FF564EC5
:10BBC000B8F1000F10D0C4F80051707918B1757138
:10BBD000002007F0E8FF307830B10120534935707C
:10BBE000B07002220A6020610FB1C4F80451BAF1AA
:10BBF000000F0BD0C4F80C51B07800B9FFDF4B48F0
:10BC00000560B57001206061FFF7CBFEB9F1000F50
:10BC100005D0C4F81051307908B100F045F8414919
:10BC2000091DC1F800B068E770B53B4DE87808B968
:10BC3000F7F7AEF901208407A061A87858B100BFDA
:10BC4000D4F80C0120B90020F7F7BEF90028F7D18D
:10BC50000020C4F80C014FF0FF30C4F8080370BD99
:10BC60002DE9F0411926B407C4F808630125A56140
:10BC70000020C4F80001C4F80C01C4F81001F7F763
:10BC80008BF9254F28B12949BD7002200860256134
:10BC900000E03D70FFF75CFE2049B8792031086074
:10BCA000C4F80463BDE8F0812DE9F0411A4C4FF06F
:10BCB00080470125E079F0B1012803D0217A401EA8
:10BCC000814218DAF7F768F9064608F0C9F8E17911
:10BCD000012902D9217A491C21720EB1216900E0A3
:10BCE000E168411A022902DA11F1020F0EDC0EB1ED
:10BCF000206100E0E060FFF72BFEF7F74DF938B167
:10BD00000A49022008603D61A57002E07D61C9E733
:10BD1000257000202072C5E73C0000201805004077
:10BD200010ED00E01005024001000001340C00405D
:10BD30004FF0E0214FF00070C1F88001C1F880029F
:10BD4000384B802283F80024C1F80001704700B509
:10BD500002460420344903E001EBC0031B792BB1F8
:10BD6000401EC0B2F8D2FFDFFF2000BD41F83020F6
:10BD700001EBC00100224A718A7101220A7100BDE3
:10BD8000294A002102EBC0000171704710B504463A
:10BD9000042800D3FFDF244800EBC40420790128E5
:10BDA00000D0FFDF6079A179401CC0B2814200D091
:10BDB00060714FF0E0214FF00070C1F8000210BD3B
:10BDC0002DE9F041194805681849194808310860FB
:10BDD0001448042690F80004134F4009154C042819
:10BDE00018D0FFDF16E0217807EBC1000279012AA5
:10BDF00008D1427983799A4204D04279827157F806
:10BE0000310080472078401CC0B22070042801D344
:10BE100000202070761EF6B2E5D20448001D0560B1
:10BE2000BDE8F08119E000E0C805002010050240DF
:10BE30000100000150000020F8B51D46DDE906476D
:10BE40000E000AD004F0F8FE2346FF1DBCB23146B6
:10BE50002A46009404F005FBF8BDD0192246194685
:10BE600018F0A6F92046F8BD70B50D46044610211D
:10BE700018F01DFA258117206081A07B40F00A0090
:10BE8000A07370BD4FF6FF720A800146022008F0D1
:10BE9000F9B9704700897047827BD30701D19207B7
:10BEA00003D4808908800020704705207047827B7A
:10BEB000920700D58181704701460020098841F62C
:10BEC000FE52114200D00120704700B50346807B2E
:10BED000C00701D0052000BD59811846FFF7ECFFCF
:10BEE000C00703D0987B40F004009873987B40F023
:10BEF00001009873002000BD827B520700D509B174
:10BF00004089704717207047827B61F3C3028273B8
:10BF100070472DE9FC5F0E460446017896460120E5
:10BF200000FA01F14DF6FF5201EA020962684FF68C
:10BF3000FF7B1188594502D10920BDE8FC9FB9F16A
:10BF4000000F05D041F6FE55294201D00120F4E74B
:10BF500041EA090111801D0014D04FF0000C85F852
:10BF600000C023780521032267464FF0020A0E2BFA
:10BF700074D2DFE803F0F809252F4762697447900F
:10BF800092B3D0D70420D8E7616820898B7B9B07C8
:10BF90007DD5172848D30B89834245D38989172932
:10BFA00001D3814240D185F800A0A5F8010032807C
:10BFB000616888816068817B21F002018173C5E03E
:10BFC000042028702089A5F801006089A5F80300E5
:10BFD0003180BBE0208A3188C01D1FFA80F84145BE
:10BFE00022D3062028702089A5F801006089A5F8D1
:10BFF0000300A089A5F805000721208ACDE90001EA
:10C0000063693EE0082B10D0082028702089A5F82D
:10C0100001006089A5F8030031806A1D694604F1BA
:10C020000C0006F066FA10B15FE01020EDE73088F2
:10C030009DF800100844308088E00A20287020898C
:10C04000A5F80100328045E00C2028702089A5F871
:10C0500001006089A5F8030031803BE083E021897D
:10C06000338800EB41021FFA82F843453DD3B8F113
:10C07000050F3AD30E222A700BEA4101CDE90010D8
:10C08000E36860882A467146FFF7D6FE00E04DE07F
:10C09000A6F800805AE04020287060893188C01CD2
:10C0A0001FFA80F8414520D32878714620F03F00E0
:10C0B000123028702089A5F801006089CDE90002BE
:10C0C00060882A46E368FFF7B7FEA6F80080287864
:10C0D00040063BD461682089888037E0A089328897
:10C0E000401D1FFA80F8424501D204273EE0162089
:10C0F00028702089A5F801006089A5F80300A089AF
:10C10000CDE9000160882A4671462369FFF794FE55
:10C11000A6F80080DEE718202870207A6870A6F85C
:10C1200000A013E061680A88920401D405271DE08D
:10C13000C9882289914201D0062717E01E21297063
:10C1400030806068018821F400510180B9F1000F4E
:10C150000CD0618878230022022007F0E9FF616893
:10C160002078887007E0A6F800C00327606801887F
:10C1700021EA090101803846DFE62DE9FF4F85B04D
:10C180001746129C0D001E461CD03078C10703D004
:10C1900000F03F00192801D9012100E000212046CC
:10C1A000FFF7AAFEA8420DD32088A0F57F41FF39F2
:10C1B00008D03078410601D4000605D5082009B022
:10C1C000BDE8F08F0720FAE700208DF800008DF819
:10C1D000010030786B1E00F03F0C0121A81E4FF0CB
:10C1E000050A4FF002094FF0030B9AB2BCF1200F81
:10C1F00075D2DFE80CF08B10745E7468748C749CDC
:10C2000074B674BB74C974D574E2747474F274F047
:10C2100074EF74EE748B052D78D18DF80090A078B2
:10C220008DF804007088ADF8060030798DF80100B3
:10C23000707800F03F000C2829D00ADCA0F1020041
:10C24000092863D2DFE800F0126215621A621D62EB
:10C250002000122824D004DC0E281BD01028DBD1AB
:10C260001BE016281FD01828D6D11FE020788007A1
:10C2700001E020784007002848DAEFE02078000746
:10C28000F9E72078C006F6E720788006F3E7207803
:10C290004006F0E720780006EDE72088C005EAE7D1
:10C2A00020884005E7E720880005E4E72088C004EF
:10C2B000E1E72078800729D5032D27D18DF800B03C
:10C2C000B6F8010082E0217849071FD5062D1DD35D
:10C2D00081B27078012803D0022817D102E0CAE0A9
:10C2E000022000E0102004228DF8002072788DF8E2
:10C2F0000420801CB1FBF0F2ADF8062092B242435C
:10C300008A4203D10397ADF80890A7E07AE020783D
:10C31000000777D598B282088DF800A0ADF8042008
:10C32000B0EB820F6ED10297ADF8061096E021783F
:10C33000C90667D5022D65D381B206208DF80000AD
:10C34000707802285ED300BFB1FBF0F28DF80400D4
:10C35000ADF8062092B242438A4253D1ADF808901C
:10C360007BE0207880064DD5072003E0207840064A
:10C370007FD508208DF80000A088ADF80400ADF846
:10C380000620ADF8081068E02078000671D5092075
:10C39000ADF804208DF80000ADF8061002975DE0BE
:10C3A0002188C90565D5022D63D381B20A208DF895
:10C3B0000000707804285CD3C6E72088400558D573
:10C3C000012D56D10B208DF80000A088ADF8040097
:10C3D00044E021E026E016E0FFE72088000548D58C
:10C3E000052D46D30C208DF80000A088ADF8040080
:10C3F000B6F803006D1FADF80850ADF80600ADF8B3
:10C400000AA02AE035E02088C00432D5012D30D1C1
:10C410000D208DF8000021E02088800429D4B6F892
:10C420000100E080A07B000723D5032D21D33078C5
:10C4300000F03F001B2818D00F208DF80000208846
:10C4400040F40050A4F80000B6F80100ADF8040074
:10C45000ED1EADF80650ADF808B003976946059893
:10C46000F5F7E6FC050008D016E00E208DF8000078
:10C47000EAE7072510E008250EE0307800F03F00DD
:10C480001B2809D01D2807D00220059907F0FAFEC5
:10C49000208800F400502080A07B400708D520466B
:10C4A000FFF70AFDC00703D1A07B20F00400A073B2
:10C4B000284684E61FB5022806D101208DF8000029
:10C4C00088B26946F5F7B4FC1FBD0000F8B51D46FB
:10C4D000DDE906470E000AD004F0AEFB2346FF1D3F
:10C4E000BCB231462A46009403F0BBFFF8BDD01918
:10C4F0002246194617F05CFE2046F8BD2DE9FF4F95
:10C500008DB09B46DDE91B57DDF87CA00C46082B5F
:10C5100005D0E06901F002F950B11020D2E028887E
:10C52000092140F0100028808AF80010022617E048
:10C53000E16901208871E2694FF420519180E1693D
:10C540008872E06942F601010181E069002181738E
:10C550002888112140F0200028808AF80010042645
:10C5600038780A900A2038704FF0020904F1180058
:10C570004D460C9001F095FBB04681E0BBF1100FE9
:10C580000ED1022D0CD0A9EB0800801C80B2022134
:10C59000CDE9001005AB52461E990D98FFF796FFA6
:10C5A000BDF816101A98814203D9F74800790F9008
:10C5B00004E003D10A9808B138702FE04FF002016F
:10C5C000CDE900190DF1160352461E990D98FFF79B
:10C5D0007DFF1D980088401B801B83B2C6F1FF00C1
:10C5E000984200D203461E990BA8D9B15FF0000211
:10C5F000DDF878C0CDE9032009EB060189B2CDE969
:10C6000001C10F980090BDF8161000220D9801F09E
:10C61000CBFB387070B1C0B2832807D0BDF81600CC
:10C6200020833AE00AEB09018A19E1E7022011B000
:10C63000BDE8F08FBDF82C00811901F0FF08022D34
:10C640000DD09AF80120424506D1BDF82010814254
:10C6500007D0B8F1FF0F04D09AF801801FE08AF8E4
:10C660000180C94800680178052902D1BDF816107B
:10C67000818009EB08001FFA80F905EB080085B2FC
:10C68000DDE90C1005AB0F9A01F00EFB28B91D98DF
:10C690000088411B4145BFF671AF022D13D0BBF19D
:10C6A000100F0CD1A9EB0800801C81B20220CDE94B
:10C6B000000105AB52461E990D98FFF707FF1D9824
:10C6C0000580002038700020B1E72DE9F8439C4632
:10C6D000089E13460027B26B9AB3491F8CB2F18FA4
:10C6E000A1F57F45FF3D05D05518AD882944891D2A
:10C6F0008DB200E000252919B6F83C80083141458B
:10C7000020D82A44BCF8011022F8021BBCF8031000
:10C7100022F8021B984622F8024B914604F07AFA5E
:10C720004FF00C0C41464A462346CDF800C003F0BA
:10C7300064FEF587B16B00202944A41D21440880C4
:10C7400003E001E0092700E083273846BDE8F883CD
:10C7500010B50B88848F9C420CD9846BE018048838
:10C7600044B1848824F40044A41D23440B80106049
:10C77000002010BD0A2010BD2DE9F0478AB0002529
:10C78000904689468246ADF8185007274BE0059839
:10C7900006888088000446D4A8F8006007A80195A0
:10C7A00000970295CDE903504FF400730022314603
:10C7B000504601F0F9FA04003CD1BDF81800ADF87C
:10C7C0002000059804888188B44216D10A0414D444
:10C7D00001950295039521F400410097049541F4D9
:10C7E000804342882146504601F0B4F804000BD142
:10C7F0000598818841F40041818005AA08A948462E
:10C80000FFF7A6FF0400DCD000970598029501957C
:10C81000039504950188BDF81C300022504601F0B4
:10C8200099F80A2C06D105AA06A94846FFF790FFF9
:10C830000400ACD0ADF8185004E00598818821F4CC
:10C840000041818005AA06A94846FFF781FF00281C
:10C85000F3D00A2C03D020460AB0BDE8F0870020B0
:10C86000FAE710B50C46896B86B051B10C218DF8F2
:10C870000010A18FADF80810A16B01916946FAF77D
:10C8800064FC00204FF6FF71A063E187A08706B02B
:10C8900010BD2DE9F0410D460746896B0020069E2C
:10C8A0001446002911D0012B0FD1324629463846B3
:10C8B000FFF762FF002808D1002C06D03246294637
:10C8C0003846BDE8F04100F038BFBDE8F0812DE901
:10C8D000FC411446DDE9087C0E46DDE90A15521DCF
:10C8E000BCF800E092B2964502D20720BDE8FC8178
:10C8F000ACF8002017222A70A5F80160A5F80330D3
:10C900000522CDE900423B462A46FFF7DFFD002025
:10C91000ECE770B50C4615464821204617F0E9FCB7
:10C9200004F1080044F81C0F00204FF6FF71E0618D
:10C9300061842084A5841720E08494F82A0040F0C4
:10C940000A0084F82A0070BD4FF6FF720A80014683
:10C95000032007F097BC30B585B00C460546FFF7BD
:10C9600080FFA18E284629B101218DF8001069466B
:10C97000FAF7EBFB0020E0622063606305B030BD96
:10C98000B0F84000704700005400002090F84620A6
:10C99000920703D4408808800020F3E70620F1E7DF
:10C9A00090F846209207EDD5A0F84410EAE701463A
:10C9B000002009880A0700D5012011F0F00F01D0EE
:10C9C00040F00200CA0501D540F004008A0501D5F7
:10C9D00040F008004A0501D540F010000905D1D506
:10C9E00040F02000CEE700B5034690F84600C007AF
:10C9F00001D0062000BDA3F842101846FFF7D7FF6C
:10CA000010F03E0F05D093F8460040F0040083F884
:10CA1000460013F8460F40F001001870002000BDDA
:10CA200090F84620520700D511B1B0F84200A9E7AE
:10CA30001720A7E710F8462F61F3C3020270A1E7A1
:10CA40002DE9FF4F9BB00E00DDE92B34DDE929789D
:10CA5000289D24D02878C10703D000F03F00192872
:10CA600001D9012100E000212046FFF7D9FFB042A3
:10CA700015D32878410600F03F010CD41E290CD0B4
:10CA8000218811F47F6F0AD13A8842B1A1F57F4223
:10CA9000FF3A04D001E0122901D1000602D504209A
:10CAA0001FB0C5E5F9491D984FF0000A08718DF8CF
:10CAB00018A08DF83CA00FAA0A60ADF81CA0ADF834
:10CAC00050A02978994601F03F02701F5B1C04F1C9
:10CAD000180C4FF0060E4FF0040BCDF858C01F2A6B
:10CAE0007ED2DFE802F07D7D107D267DAC7DF47D79
:10CAF000F37DF27DF17DF47DF07D7D7DEF7DEE7D3A
:10CB00007D7D7D7DED0094F84610B5F80100890724
:10CB100001D5032E02D08DF818B022E34FF4006146
:10CB2000ADF85010608003218DF83C10ADF8400046
:10CB3000D8E2052EEFD1B5F801002083ADF81C0036
:10CB4000B5F80310618308B1884201D901207FE163
:10CB50000020A07220814FF6FF702084169801F00B
:10CB6000A0F8052089F800000220029083460AAB55
:10CB70001D9A16991B9801F097F890BB9DF82E000E
:10CB8000012804D0022089F80100102003E00120D0
:10CB900089F8010002200590002203A90BA805F0E6
:10CBA000A8FCE8BB9DF80C00059981423DD13A886C
:10CBB000801CA2EB0B01814237DB02990220CDE9F8
:10CBC00000010DF12A034A4641461B98FFF77EFCFF
:10CBD00002980BF1020B801C80B217AA03A901E096
:10CBE000A0E228E002900BA805F083FC02999DF8D2
:10CBF0000C00CDE9000117AB4A4641461B98FFF7F0
:10CC000065FC9DF80C100AAB0BEB01001FFA80FBD2
:10CC100002981D9A084480B2029016991B9800E071
:10CC200003E001F041F80028B6D0BBF1020F02D0BA
:10CC3000A7F800B053E20A208DF818004FE2002157
:10CC40000391072EFFF467AFB5F801002083ADF81C
:10CC50001C00B5F80320628300283FF477AF9042B0
:10CC60003FF674AF0120A072B5F8050020810020C6
:10CC7000A073E06900F052FD78B9E1690120887184
:10CC8000E2694FF420519180E1698872E06942F6CF
:10CC900001010181E06900218173F01F20841E9849
:10CCA000606207206084169800F0FBFF072089F877
:10CCB00000000120049002900020ADF82A0028E036
:10CCC0001DE2A3E13AE1EAE016E2AEE086E049E0E7
:10CCD0000298012814D0E0698079012803D1BDF8B9
:10CCE0002800ADF80E00049803ABCDE900B04A4629
:10CCF00041461B98FFF7EAFB0498001D80B20490A0
:10CD0000BDF82A00ADF80C00ADF80E00059880B211
:10CD100002900AAB1D9A16991B9800F0C5FF28B91E
:10CD200002983988001D05908142D1D202980128CD
:10CD300081D0E0698079012805D0BDF82810A1F5DF
:10CD40007F40FF3803D1BDF82800ADF80E000498ED
:10CD500003ABCDE900B04A4641461B98FFF7B6FB4E
:10CD60000298BBE1072E02D0152E7FF4D4AEB5F8A1
:10CD700001102183ADF81C10B5F80320628300294F
:10CD80003FF4E4AE91423FF6E1AE0121A1724FF0D3
:10CD9000000BA4F808B084F80EB0052E07D0C0B27E
:10CDA000691DE26905F086FB00287FF444AF4FF669
:10CDB000FF70208401A906AA14A8CDF800B081E86C
:10CDC00085032878214600F03F031D9A1B98FFF742
:10CDD00095FB8246208BADF81C0080E10120032EDC
:10CDE000C3D14021ADF85010B5F801102183ADF842
:10CDF0001C100AAAB8F1000F00D00023CDE90203ED
:10CE000004921D98CDF80480009038880022401EBE
:10CE100083B21B9800F0C8FF8DF8180090BB0B2060
:10CE200089F80000BDF8280037E04FF0010C052E0E
:10CE30009BD18020ADF85000B5F801102183B5F8E2
:10CE400003002084ADF81C10B0F5007F03D9072043
:10CE50008DF8180085E140F47C4222840CA8B8F1DA
:10CE6000000F00D00023CDE90330CDE9018C1D98DF
:10CE700000903888401E83B21B9800F095FF8DF813
:10CE8000180028B18328A8D10220BDE0540000205A
:10CE90000D2189F80010BDF83000401C1EE1032E62
:10CEA00004D248067FF537AE002017E1B5F801102F
:10CEB000ADF81C102878400602D58DF83CE002E061
:10CEC00007208DF83C004FF000080320CDE9020850
:10CED0001E9BCDF810801D980193A6F1030B0090C6
:10CEE0001FFA8BF342461B9800F034FD8DF81800B2
:10CEF0008DF83C80297849060DD52088C00506D5D7
:10CF0000208BBDF81C10884201D1C4F82480404613
:10CF10008DF81880E2E0832801D14FF0020A4FF427
:10CF20008070ADF85000BDF81C002083A4F820B03C
:10CF30001E986062032060841321CCE0052EFFF46C
:10CF4000EAADB5F80110ADF81C10A28F62B3A2F5DE
:10CF50007F43FE3B28D008228DF83C204FF0000B89
:10CF60000523CDE9023BDDF878C0CDF810B01D9A5D
:10CF700080B2CDF804C040F400430092B5F803201D
:10CF80001B9800F0E7FC8DF83CB04FF400718DF871
:10CF90001800ADF85010832810D0F8B1A18FA1F57A
:10CFA0007F40FE3807D0DCE00B228DF83C204FF6A6
:10CFB000FE72A287D2E7A4F83CB0D2E000942B46E0
:10CFC00031461E9A1B98FFF780FB8DF8180008B1B8
:10CFD00083284BD1BDF81C00208355E700942B46D5
:10CFE00031461E9A1B98FFF770FB8DF81800E8BBBE
:10CFF000E18FA06B0844811D8DE8820343888288FD
:10D0000001881B98FFF763FC824668E095F8018071
:10D01000022E70D15FEA080002D0B8F1010F6AD188
:10D0200009208DF83C0007A800908DF84080434609
:10D03000002221461B98FFF72CFC8DF842004FF090
:10D04000000B8DF843B050B9B8F1010F12D0B8F110
:10D05000000F04D1A18FA1F57F40FF380AD0A08F27
:10D0600040B18DF83CB04FF4806000E037E0ADF89F
:10D0700050000DE00FA91B98FAF767F882468DF86B
:10D080003CB04FF48060ADF85000BAF1020F06D00A
:10D09000FC480068C07928B18DF8180027E0A4F892
:10D0A000188044E0BAF1000F03D081208DF81800F9
:10D0B0003DE007A800904346012221461B98FFF758
:10D0C000E8FB8DF8180021461B98FFF7CAFB9DF876
:10D0D000180020B9192189F80010012038809DF826
:10D0E0003C0020B10FA91B98FAF72FF88246BAF13D
:10D0F000000F33D01BE018E08DF818E031E0207805
:10D10000000712D5012E10D10A208DF83C00E088CE
:10D11000ADF8400003201B9907F0B4F80820ADF8E3
:10D120005000C1E648067FF5F6AC4FF0040A2088AF
:10D13000BDF8501008432080BDF8500080050BD585
:10D14000A18FA1F57F40FE3806D11E98E062289895
:10D150002063A6864FF0030A5046A1E49DF818000C
:10D1600078B1012089F80000297889F80110BDF80C
:10D170001C10A9F802109DF8181089F80410052059
:10D1800038802088BDF8501088432080E4E72DE9DE
:10D19000FF4F8846087895B0012181404FF2090081
:10D1A000249C0140ADF820102088DDF88890A0F57F
:10D1B0007F424FF0000AFF3A06D039B1000705D58B
:10D1C000012019B0BDE8F08F0820FAE7239E4FF048
:10D1D000000B0EA886F800B018995D460988ADF8D6
:10D1E0003410A8498DF81CB0179A0A718DF838B020
:10D1F000086098F8000001283BD0022809D00328D5
:10D200006FD1307820F03F001D303070B8F8040046
:10D21000E08098F800100320022904D1317821F031
:10D220003F011B31317094F84610090759D505AB01
:10D23000B9F1000F13D0002102AA82E80B000720E9
:10D24000CDE90009BDF83400B8F80410C01E83B25F
:10D250000022159800F0A8FD0028D1D101E0F11CB2
:10D26000EAE7B8F80400A6F80100BDF81400C01CF5
:10D2700004E198F805108DF81C1098F804000128B6
:10D2800006D04FF4007A02282CD00328B8D16CE1E4
:10D290002188B8F8080011F40061ADF8201020D002
:10D2A00017281CD3B4F84010814218D3B4F84410A6
:10D2B000172901D3814212D1317821F03F01C91CD5
:10D2C0003170A6F801000321ADF83410A4F8440031
:10D2D00094F8460020F0020084F8460065E1052538
:10D2E0007EE177E1208808F1080700F4FE60ADF8E0
:10D2F000200010F0F00F1BD010F0C00F03D03888C2
:10D30000228B9042EBD199B9B878C00710D0B96898
:10D310000720CDE902B1CDF804B00090CDF810B0EF
:10D32000FB88BA883988159800F014FB0028D6D1FC
:10D330002398BDF82010401C80294ED006DC10290F
:10D340000DD020290BD0402987D124E0B1F5807F72
:10D350006ED051457ED0B1F5806F97D1DEE0C80622
:10D3600001D5082000E0102082460DA907AA05205B
:10D37000CDE902218DF83800ADF83CB0CDE9049636
:10D3800008A93888CDE9000153460722214615989F
:10D39000FFF7B4F8A8E09DF81C2001214FF00A0A1D
:10D3A000002A9BD105ABB9F1000F00D00020CDE9D8
:10D3B00002100720CDE90009BDF834000493401E97
:10D3C00083B2218B0022159800F0EEFC8DF81C0032
:10D3D0000B203070BDF8140020E09DF81C200121C6
:10D3E0004FF00C0A002A22D113ABB9F1000F00D084
:10D3F0000020CDE902100720CDE900090493BDF813
:10D400003400228C401E83B2218B159800F0CCFC96
:10D410008DF81C000D203070BDF84C00401CADF89C
:10D42000340005208DF83800208BADF83C00BCE0BE
:10D430003888218B88427FF452AF9DF81C004FF052
:10D44000120A00281CD1606AA8B1B878C0073FF45E
:10D4500046AF00E018E0BA680720CDE902B2CDF887
:10D4600004B00090CDF810B0FB88BA88159800F091
:10D4700071FA8DF81C00132030700120ADF83400D3
:10D4800093E00000540000203988208B8142D2D1E3
:10D490009DF81C004FF0160A0028A06B08D0E0B3DE
:10D4A0004FF6FF7000215F46ADF808B0019027E00D
:10D4B00068B1B978C907BED1E18F0DAB0844821DB0
:10D4C00003968DE80C0243888288018809E0B878C9
:10D4D000C007BCD0BA680DAB03968DE80C02BB88C0
:10D4E000FA881598FFF7F3F905005ED0072D72D082
:10D4F00076E0019005AA02A92046FFF729F9014626
:10D50000E28FBDF80800824201D00029F1D0E08FFF
:10D51000A16B084407800198E08746E09DF81C0055
:10D520004FF0180A40B1208BC8B1388820832146BB
:10D530001598FFF796F938E004F118000090237E63
:10D54000012221461598FFF7A4F98DF81C00002848
:10D55000EDD1192030700120ADF83400E7E7052542
:10D5600021461598FFF77DF93AE0208800F4007015
:10D57000ADF8200050452DD1A08FA0F57F41FE3998
:10D5800001D006252CE0D8F808004FF0160A48B163
:10D59000A063B8F80C10A1874FF6FF71E187A0F8DF
:10D5A00000B002E04FF6FF70A087BDF8200030F415
:10D5B0007F611AD0782300220320159906F0B8FD68
:10D5C00098F8000020712088BDF8201008432080C2
:10D5D0000EE000E007252088BDF820108843208059
:10D5E000208810F47F6F1CD03AE02188814321808D
:10D5F0009DF8380020B10EA91598F9F7A6FD05464B
:10D600009DF81C000028EBD086F801A001203070A6
:10D61000208B70809DF81C0030710520ADF834001F
:10D62000DEE7A18EE1B118980DAB0088ADF83400AB
:10D630002398CDE90304CDE90139206B0090E36A1A
:10D64000179A1598FFF7FCF9054601208DF8380068
:10D650000EA91598F9F779FD00B10546A4F834B084
:10D6600094F8460040070AD52046FFF7A0F910F0CD
:10D670003E0F04D114F8460F20F0040020701898D3
:10D68000BDF83410018028469BE500B585B003281D
:10D6900006D102208DF8000088B26946F9F755FDE1
:10D6A00005B000BD10B5384C0B782268012B02D0B4
:10D6B000022B2AD111E013780BB1052B01D10423E1
:10D6C000137023688A889A802268CB88D380226866
:10D6D0000B891381498951810DE08B8893802268E1
:10D6E000CB88D38022680B8913814B8953818B8926
:10D6F0009381096911612168F9F727FD22680021EA
:10D700000228117003D0002800D0812010BD832092
:10D7100010BD806B002800D001207047817801295E
:10D7200009D10088B0F5205F03D042F6010188429C
:10D7300001D10020704707207047F0B587B0002462
:10D7400015460E460746ADF8144010E006980188CD
:10D750002980811DCDE902410721019404940091A3
:10D76000838842880188384600F0F4F830B906AA68
:10D7700005A93046FEF7ECFF0028E7D00A2800D1C3
:10D78000002007B0F0BD00005400002010B58B78D9
:10D7900083B102789A4205D10B885BB102E08B79A4
:10D7A000091D4BB18B789A42F9D1B0F801300C8841
:10D7B000A342F4D1002010BD812010BD072826D03F
:10D7C00012B1012A27D103E0497801F0070102E0F4
:10D7D0004978C1F3C20105291DD2DFE801F0031821
:10D7E000080C12000AB10320704702207047042879
:10D7F0000DD250B10DE0052809D2801E022808D3B1
:10D8000003E0062803D0032803D00520704700203A
:10D8100070470F20704781207047C0B282060BD43A
:10D82000000607D5FE48807A4143C01D01EBD000B9
:10D8300080B27047084670470020704770B5138863
:10D840000B800B781C0625D5F54CA47A844204D8AD
:10D8500043F010000870002070BD956800F00706C6
:10D8600005EBD0052D78F54065F304130B701378A4
:10D87000D17803F0030341EA032140F20123B1FB15
:10D88000F3F503FB15119268E41D00FB012000EB8A
:10D89000D40070BD906870BD37B51446BDF8041053
:10D8A00011809DF804100A061ED5C1F30013DC494F
:10D8B000A568897A814208D8FE2811D1C91DC908F6
:10D8C0005A42284616F0EBFC0AE005EBD00100F0C6
:10D8D0000702012508789540A84393401843087033
:10D8E000207820F0100020703EBD2DE9F041074661
:10D8F000C81C0E4620F00300B04202D08620BDE8CE
:10D90000F081C74D002034462E60AF802881AA7276
:10D91000E8801AE0E988491CE980810614D4E1789E
:10D9200000F0030041EA002040F20121B0FBF1F2D7
:10D9300001FB12012068FFF770FF2989084480B2BB
:10D940002881381A3044A0600C3420784107E1D493
:10D950000020D4E72DE9FF4F89B01646DDE9168A8D
:10D960000F46994623F44045084600F00DFB04009D
:10D970000FD0099802F0E2FF0290207800060AD545
:10D98000A748817A0298814205D887200DB0BDE86A
:10D99000F08F0120FAE7224601A90298FFF74EFF17
:10D9A000834600208DF80C004046B8F1070F1AD0CE
:10D9B00001222146FFF702FF0028E7D12078400628
:10D9C00011D502208DF80C00ADF81070BDF80400E0
:10D9D000ADF81200ADF814601898ADF81650CDF8F7
:10D9E0001CA0ADF818005FEA094004D500252E46BA
:10D9F000A84601270CE02178E07801F0030140EA15
:10DA0000012040F20121B0FBF1F2804601FB1287B8
:10DA10005FEA494009D5B84507D1A178207901F0DE
:10DA2000030140EA0120B04201D3BE4201D90720E0
:10DA3000ACE7A8191FFA80F9B94501D90D20A5E76F
:10DA40009DF80C0028B103A90998F9F77CFB002880
:10DA50009CD1B84507D1A0784FEA192161F30100A4
:10DA6000A07084F804901A9800B10580199850EAC3
:10DA70000A0027D0199830B10BEB06002A461999F5
:10DA800016F096FB0EE00BEB06085746189E099819
:10DA900003F0C0F82B46F61DB5B239464246009554
:10DAA00002F0ABFC224601A90298FFF7C7FE9DF8E1
:10DAB0000400224620F010008DF80400DDE901107A
:10DAC000FFF7EAFE002061E72DE9FF4FDFF85091F4
:10DAD00082461746B9F80610D9F8000001EB41015B
:10DAE00000EB810440F20120B2FBF0F185B000FBB5
:10DAF00011764D46DDF84C8031460698FFF78DFED5
:10DB000029682A898B46611A0C3101441144AB887B
:10DB100089B28B4202D8842009B038E70699CDB289
:10DB2000290603D5A90601D50620F5E7B9F806C0F0
:10DB30000CF1010C1FFA8CFCA9F806C0149909B16C
:10DB4000A1F800C0A90602D5C4F8088007E0104477
:10DB500080B2A9F80800191A01EB0B00A060224658
:10DB6000FE200699FFF798FEE77026712078390AA3
:10DB700061F30100320AA17840F0040062F3010170
:10DB8000A17020709AF802006071BAF80000E0807D
:10DB900000262673280602D599F80A7000E00127AE
:10DBA000A80601D54FF000084D4600244FF00709A4
:10DBB0000FE0CDE902680196CDF800900496E9885F
:10DBC0002046129B089AFFF7C5FE0028A4D1641CCA
:10DBD000E4B2BC42EDD300209EE72DE9F047804639
:10DBE00000F0D2F9070005D0002644460C4D40F263
:10DBF000012919E00120BDE8F087204600F0C4F9B2
:10DC00000278C17802F0030241EA0222B2FBF9F382
:10DC100009FB13210068FFF700FE304486B201E0E3
:10DC2000E8050020641CA4B2E988601E8142E4DC9F
:10DC3000A8F10100E8802889801B28810020387025
:10DC4000D9E710B5144631B1491E218002F076FEA5
:10DC5000A070002010BD012010BD10B5D2490446AF
:10DC60000088CA88904201D30A2010BD096800EBE1
:10DC7000400001EB80025079A072D0882081917819
:10DC8000107901F0030140EA0120A081A078E11C95
:10DC9000FFF7D4FD20612088401C2080E080002018
:10DCA00010BD0121018270472DE9FF4F85B04FF66D
:10DCB000FF788246A3F8008048681F460D468078AA
:10DCC0008DF8060048680088ADF8040000208DF843
:10DCD0000A00088A0C88A04200D304462C8241E046
:10DCE000288A401C2882701D6968FFF74FFDB8BB69
:10DCF0003988414501D1601E38806888A04236D3FA
:10DD0000B178307901F0030140EA012901A9701DC1
:10DD1000FFF73CFD20BB298941452CD0002231462C
:10DD20000798FFF74BFDD8B92989494518D1E9680B
:10DD30000391B5F80AC0D6F808B05046CDF800C037
:10DD400002F068FFDDF800C05A460CF1070C1FFA1C
:10DD50008CFC4B460399CDF800C002F018FB50B183
:10DD6000641CA4B2204600F00FF90600B8D1641E6E
:10DD70002C820A20D0E67C807079B871F088B88057
:10DD80003178F07801F0030140EA01207881A7F8AA
:10DD90000C90504602F0D2FD324607F10801FFF721
:10DDA0004DFD38610020B7E62DE9FF4F87B0814671
:10DDB0001C469246DDF860B0DDF85480089800F00B
:10DDC000E3F805000CD0484602F0B8FD29780906B2
:10DDD00008D57549897A814204D887200BB0D6E5E9
:10DDE0000120FBE7CAF309062A4601A9FFF726FD31
:10DDF0000746149807281CD000222946FFF7DEFCAE
:10DE00000028EBD12878400613D501208DF80800B2
:10DE10000898ADF80C00BDF80400ADF80E00ADF8A0
:10DE20001060ADF8124002A94846F9F78CF90028B5
:10DE3000D4D12978E87801F0030140EA0121AA78D9
:10DE4000287902F0030240EA0220564507D0B1F5D6
:10DE5000007F04D9611E814201DD0B20BEE78642AE
:10DE600001D90720BAE7801B85B2A54200D9254613
:10DE7000BBF1000F01D0ABF80050179818B1B919D9
:10DE80002A4616F095F9B8F1000F0DD03E444846E9
:10DE90004446169F02F0D0FE2146FF1DBCB232461A
:10DEA0002B46009402F0DDFA002097E72DE9F041BF
:10DEB00007461D461646084600F066F804000BD0DB
:10DEC000384602F03BFD2178090607D53649897AA4
:10DED000814203D8872012E5012010E52246314611
:10DEE000FFF7ACFC65B12178E07801F0030140EA6E
:10DEF0000120B0F5007F01D8012000E0002028704B
:10DF00000020FCE42DE9F04107461D461646084670
:10DF100000F03AF804000BD0384602F00FFD2178EB
:10DF2000090607D52049897A814203D88720E6E48B
:10DF30000120E4E422463146FFF7AEFCFF2D14D069
:10DF40002178E07801F0030240EA022040F2012249
:10DF5000B0FBF2F302FB130015B900F2012080B20E
:10DF6000E070000A60F3010121700020C7E410B5E1
:10DF70000C4600F009F828B1C18821804079A070D2
:10DF8000002010BD012010BD0749CA88824209D374
:10DF900040B1096800EB40006FF00B0202EB80001B
:10DFA0000844704700207047E805002070B503461C
:10DFB000002002466FF02F050EE09C5CA4F13006B5
:10DFC0000A2E02D34FF0FF3070BD00EB800005EB4E
:10DFD0004000521C2044D2B28A42EED370BD30B50C
:10DFE0000A240AE0B0FBF4F304FB13008D18303070
:10DFF00005F8010C521E1846D2B2002AF2D130BDEB
:10E0000030B500234FF6FF7510E0040A44EA002003
:10E0100084B2C85C6040C0F30314604005EA003479
:10E020004440E0B25B1C84EA40109BB29342ECD3C4
:10E0300030BD000010B582B0694601F0D1FD002866
:10E0400018BFFFDF9DF80000002448B1019890F848
:10E05000DD0028B1019880F8DD4001980AF0AFF9A1
:10E06000F8488068A0F8D24002B010BD2DE9F04712
:10E0700004460D46062002F043FC0646072002F047
:10E080003FFC304400F0FF08002718EB050618BFDE
:10E090004FF000091DD02088401C80B22080B04283
:10E0A00028BFA4F800902588454501D3B54209D37F
:10E0B0000621284602F07CFC20B90721284602F000
:10E0C00077FC10B10020BDE8F087781CC7B2BE42D3
:10E0D000E1D84FF6FF7020801220BDE8F08770B5C0
:10E0E00082B007F073FB0DF0AFF9D74C4FF6FF7617
:10E0F00000256683A683D5A12570D1E90001CDE96D
:10E10000000165706946A01C16F008FAA11C601C8D
:10E1100014F04CF825721B2060814FF4A471A1818A
:10E12000E08121820321A1740422E274A082E082B2
:10E13000A4F13E00218305704680C6480570A4F115
:10E1400010000570468002B070BDF8B5BD4D174691
:10E150000E466860297007F0B3FA4FF6FF70ADF80D
:10E16000000000216846FFF781FFA0B90621BDF835
:10E17000000002F02FFC04460721BDF8000002F069
:10E1800029FC002C1CBF0028FFDF00216846FFF798
:10E190006DFF0028EAD0FFF7A2FF287812F07CF884
:10E1A0000FF0A0FC2978686813F013FF28780CF0B2
:10E1B000ABFB30460AF00FF807F020FC29786868BE
:10E1C0000BF048FA3946287814F0ADFDBDE8F84068
:10E1D0000DF03AB910B50124002A1CBF002010BD73
:10E1E000002908BF022105D0012918BF002401D051
:10E1F000204610BD0EF088FEFAE72DE9F04F8BB0F7
:10E20000040008BFFFDF02218F4E06F11C00FFF75C
:10E210002DFF002818BFFFDFB6F81CA0062002F073
:10E220006FFB0546072002F06BFB284400F0FF0857
:10E2300008F1010000F0FF094FF0000BB78B4745D4
:10E2400025D120460FF022F8002840F0CE8030780B
:10E25000002800F0CE8084F801B014202070C4F8AB
:10E2600004B0C4F808B0C4F80CB0C4F810B0C4F8D6
:10E2700014B0C4F818B0C4F81CB00220C4F820B020
:10E28000207186F800B00BB00120BDE8F08F4F453B
:10E2900020D1204607F04CFB00287DD007F02AFF54
:10E2A000002859D02078172856D12079002853D03B
:10E2B000E088072102F07CFB050008BFFFDF28880B
:10E2C00007F017FAE088072102F084FB002818BF46
:10E2D000FFDF8AE004A9384601F082FC00285BD108
:10E2E0009DF8100048B107F07EFBB84254D021469B
:10E2F00038460BF0B8F880B377E00FF05AF8B84220
:10E3000077D02146384613F085FD00286DD1059859
:10E3100000F1580590F8D00018B9E87E08B1012046
:10E3200000E00020079095F8370000281CBF95F802
:10E33000380010F0020F1CD084F801B001202070CA
:10E3400084F804B0E78095F839002072688F608106
:10E35000A88FA08185F837B047E0FFE7059800F166
:10E36000580590F80C010028DBD1E87E0028D8D0B1
:10E37000D5E7384602F060FC0290002808BFFFDFB6
:10E38000029801F06FFE50B184F801B00F212170A6
:10E39000E7802081012000E02BE0207125E0384655
:10E3A00002F038FC0290002808BFFFDF079800B396
:10E3B000029801F0AEFEE0B19DF8100038B9059862
:10E3C000D0F8F8004188B94208BF80F800B038465C
:10E3D00007F08FF984F801B00C20207084F804B0A5
:10E3E000E780287F207285F81BB00BB00120BDE8C4
:10E3F000F08F022106F11C00FFF738FE18B9B08B30
:10E4000050457FF41BAF0BB02046BDE8F04F14F031
:10E41000D0BC10B512F08AFC042803D012F086FCA0
:10E42000052802D10FF078FD28B90AF0A9F920B12A
:10E4300007F08AFC08B10C2010BD0DF051F8002047
:10E4400010BD00005C00002032060020FFFFFFFF2F
:10E450001F0000006800002010B504460078002866
:10E460001EBF0128122010BD12F060FC042806D047
:10E4700012F05CFC052802D00AF082F928B10DF0F8
:10E480007EF900281CBF0C2010BD2078002816BF84
:10E4900002280020012004F11703E21D611CBDE8E1
:10E4A00010400DF075B810B50446007800281EBF66
:10E4B0000128122010BD12F039FC042803D012F0FC
:10E4C00035FC052802D10FF027FD28B90AF058F9CC
:10E4D00020B107F039FC08B10C2010BD20780028CD
:10E4E00016BF022800200120611C0CF0BFFF00288D
:10E4F00014BF0020072010BD10B50DF043F900280F
:10E5000014BF0020302010BD10B5044612F00EFCE0
:10E51000042806D012F00AFC052802D00AF030F9CF
:10E5200008B10C2010BD20460DF026F9002010BDCA
:10E5300010B512F0FBFB042806D012F0F7FB0528FB
:10E5400002D00AF01DF928B10DF019F900281CBFFE
:10E550000C2010BD0DF075F8002010BDFF2181705A
:10E560004FF6FF718180FE4949680A7882718A8876
:10E57000028149884181012141700020704710B516
:10E58000002482B012F1080F16D00CDC12F1280F13
:10E5900018BF12F1140F0FD012F1100F18BF12F1A3
:10E5A0000C0F09D00EE012F1040F18BF002A03D09F
:10E5B000032A18BF042A05D1012807D0022809D050
:10E5C00003280BD0122402B0204610BD104607F0DD
:10E5D0008CFDF8E710460FF03AFAF4E708461446C7
:10E5E000694601F0FDFA002818BF0224EBD19DF81E
:10E5F0000000019880F857400024E4E710B5134666
:10E6000001220DF0A6FF002010BD10B5044612F047
:10E610008DFB052804BF0C2010BD204611F02AFEFA
:10E62000002010BD10B5044612F080FB042806D06F
:10E6300012F07CFB052802D00AF0A2F808B10C20E9
:10E6400010BD2146002007F0C2F8002010BD10B513
:10E65000044611F0B9FE50B10AF085F838B12078BF
:10E6600009F0DDFD20780FF090FC002010BD0C209B
:10E6700010BD10B5044612F059FB042806D012F064
:10E6800055FB052802D00AF07BF808B10C2010BD1C
:10E690002146012007F09BF8002010BD38B5044644
:10E6A0004FF6FF70ADF80000A079E179884213D0F1
:10E6B00021791F299CBF61791F290DD8002211469D
:10E6C00014F030FF40B90022E079114614F02AFF1F
:10E6D00010B9207A072801D9122038BD0AF050F865
:10E6E00060B912F023FB48B900216846FFF7BEFC71
:10E6F00020B1204606F031F8002038BD0C2038BD8E
:10E7000070B504468078002582B01A2825D00EDC2A
:10E71000162844D2DFE800F04343434343214343F8
:10E7200043434343434343434343432121212A2853
:10E7300035D00BDCA0F11E000C2830D2DFE800F051
:10E740002F2F2F2F2F2F2F2F2F2F2F0D3A38042819
:10E7500025D2DFE800F0240224022088B0F5706F93
:10E760001DD20126694601F03BFA00281EBF022097
:10E7700002B070BD9DF80000002801980BBF00F1A9
:10E78000F40100F5B87100F1F50300F271130246CF
:10E7900012D192F8D00092F8732052B903E002B07F
:10E7A0004FF0120070BD002818BF042801D008786F
:10E7B00068B102B00C2070BD92F80C0192F8732081
:10E7C000002AF6D1002818BF0428F0D1F1E70E7016
:10E7D000A07818709DF8000048B1019890F8DD000D
:10E7E00028B1019880F8DD50019809F0E8FD02B0E9
:10E7F000002070BDF0B583B00C46694601F0F0F919
:10E8000028B1204615F074FE03B00220F0BD019837
:10E81000002700F1580500F1080600BF85F8407098
:10E820003146204615F07AFE95F840000028F5D1D3
:10E8300003B0F0BD2DE9F0410D4604460189808802
:10E8400000230DF0BCFF696A814228BFBDE8F0815A
:10E85000401A401C4108A0884FF0000C401A80B2BA
:10E86000A08022896FF00E07511A8AB2228195F892
:10E870005460618816F00C0F6FF00D0328D0B0F5CE
:10E88000747F38BF604606D35038C61700EB9660D9
:10E8900003EBA01080B2814238BF0846608095F833
:10E8A0005510E08811F00C0F1BD0B2F5747F09D31E
:10E8B000A2F15001CA1701EB926103EBA11100BF55
:10E8C0001FFA81FC604528BF6046E080BDE8F0810A
:10E8D000022E1ABF03EBD00080B207EB9000DAD112
:10E8E000D8E702291ABF03EBD2011FFA81FC07EB1C
:10E8F0009201E7D1E4E7F0B587B00C46054604A9DC
:10E9000001F06EF900281CBF07B0F0BD9DF81000A3
:10E91000002814BF002201220599B1F84A30FB2BD0
:10E9200028BFFB23B1F84CC0BCF1FB0F28BF4FF050
:10E93000FB0C0C4FD7E90006BF68009001960297C8
:10E94000ADF80230ADF806C06846FFF773FF65808A
:10E95000BDF80400E080BDF80800608104E000001C
:10E960005C00002040470200BDF80200A080BDF816
:10E970000600208107B00020F0BD2DE9F04F89B0DE
:10E9800004460088694601F02BF95FEA00081CBFC5
:10E9900009B0BDE8F08FB4F806C02289ACF11B01C4
:10E9A0001220E12924BF09B0BDE8F08FB2F5A47FA1
:10E9B0003CBF09B0BDE8F08F44F29025AA4284BF65
:10E9C00009B0BDE8F08F00276388A188A3F11B067A
:10E9D000E12E24BF09B0BDE8F08FB1F5A47F2EBFB2
:10E9E0008D4209B0BDE8F08F1120BCF1FB0F99BF3B
:10E9F00040F64806B24209B0BDE8F08FFB2B92BF4B
:10EA0000B14209B0BDE8F08F208806A901F0E8F80E
:10EA1000002818BFFFDF35D19DF8180000280CBF73
:10EA2000012200220799B1F84A00FB2828BFFB20E9
:10EA3000B1F84C30FB2B28BFFB23DFF858B7DBF8CD
:10EA400000C0DBF804A0DBF808B0CDF808C0CDF8B2
:10EA50000CA0CDF810B0ADF80A00ADF80E3002A849
:10EA6000FFF7E8FEBDF80C0060F31F45BDF810008D
:10EA700060F31F49BDF80A0060F30F05BDF80E00F2
:10EA800060F30F0962881FFA89F1092091423CBFA7
:10EA900009B0BDE8F08FA9B2E28891423CBF09B04D
:10EAA000BDE8F08F4FEA1941A288238901EB154197
:10EAB0001A4491423CBF09B0BDE8F08F9DF80000B8
:10EAC0004FF001090028019808D000F5CD7580F8B5
:10EAD0009B91019890F8DE0148B307E000F582753C
:10EAE00080F80591019890F8280110B14FF03A088C
:10EAF00018E0E08868806088E8802089A880A08885
:10EB00002881012228460199FFF794FEA888B04287
:10EB100028BF40F64800A8802889B0421DD228812D
:10EB200085F800906F7009B04046BDE8F08FE0882E
:10EB300068806088E8802089A880A08828810022D9
:10EB400028460199FFF776FEA888B04228BF40F614
:10EB50004800A8802889B042E1D340F64800DEE7AB
:10EB60000BE710B5044612F0E1F8042806D012F0C5
:10EB7000DDF8052802D009F003FE28B10CF0FFFDF6
:10EB800000281CBF0C2010BD2078002816BF0228CA
:10EB900000200120E279611C0CF075FF002814BFF1
:10EBA0000020022010BD817831F0070207BFC27833
:10EBB00032F007031220704711F0040F0EBF12F05D
:10EBC000040F1120704701F023B810B504460178F6
:10EBD000122084B0012918BF002904D002291EBFC9
:10EBE000032904B010BD6178002918BF012904D0A1
:10EBF00002291EBF032904B010BDE17B21B9A17811
:10EC000001291CBF04B010BDA17831F005021CBF62
:10EC100004B010BD11F0050F04BF04B010BD11F019
:10EC2000040F1EBF112004B010BDE178E388628993
:10EC300000291EBF012904B010BD042B2EBF042AD9
:10EC400004B010BDA17B002904BF04B010BD07298A
:10EC500084BF04B010BD12F069F8042837D012F058
:10EC600065F8052833D0A0788DF80800A0788DF8D5
:10EC7000000060788DF8040020788DF80300A07BF8
:10EC80008DF80500E07B002818BF01208DF80600F4
:10EC9000A07810F0010F10D0E078012808BF022002
:10ECA00003D000280CBF012000208DF80100E0886F
:10ECB000ADF80A006089ADF80C0002A811F091FBD4
:10ECC000002804BF68460FF065F904B010BD04B019
:10ECD0000C2010BD10B5044602781220012A0FD076
:10ECE000002A18BF10BD012A26D012F01FF80528EF
:10ECF00004D011F0F6F9002808BF10BD0C2010BD9B
:10ED00006178002918BF012906D0022918BF10BD5B
:10ED1000A188002908BF10BD6388002B1CBFA188F3
:10ED20000029E0D003EB83035B0001EB8101B3EB2F
:10ED3000012F28BF10BDD6E70FF01DF8002804BF33
:10ED4000122010BD0FF02CF800200FF0D3F800288F
:10ED500018BF10BD60780FF0B1F8002818BF10BDC3
:10ED6000A1886088BDE8104011F064BB002100F06C
:10ED7000B1BF017811F0010F02D0406813F0ECBF71
:10ED800013F0B9BF2DE9F04F8FB00D460246AFF634
:10ED90004411D1E90001CDE90B011146284600F0EC
:10EDA00099FF00281CBF0FB0BDE8F08F11F0BEFF27
:10EDB00004280CD011F0BAFF052808D0F64F387897
:10EDC00028B90EF0F6FAA0F57F41FF3903D00FB055
:10EDD0000C20BDE8F08FF1480890F1480990F14807
:10EDE0000A9008AA06210DA801F0B0FD040002BF98
:10EDF00009200FB0BDE8F08F03210DF052F9B98A58
:10EE0000A4F84A10FA8AA4F84C20F87C0090BB7C45
:10EE1000208801F088FE002818BFFFDF208806F058
:10EE200067FC268804F10E094FF0000B4FF00A0A28
:10EE30000421484604F04DFF48460DF001FB062032
:10EE400001F05EFD80461CE005A9062001F039FDB9
:10EE500005A801F014FD5FEA000B10D1BDF8180001
:10EE6000B04206D00798042249460E3015F074F9D6
:10EE700070B105A801F003FD5FEA000BEED0A8F128
:10EE80000108B8F1000F07DDBBF1000FDCD007E08F
:10EE900048460DF0DEFAF2E7BBF1000F08BFFFDFD6
:10EEA000D9F800000CF07AFFBAF1010A01D000286D
:10EEB000BED0BDA004F1120600680190032101A894
:10EEC00004F0DEFE002001A90A5C3254401CC0B2EE
:10EED0000328F9D3A88B6080688CA080288DE080FF
:10EEE000687A10F0010F18BF01217CD0388B0A46D8
:10EEF00011F009FB0146A062204611F030FB4FF0F3
:10EF0000000884F85E8084F85F80A878002816BF27
:10EF10000228002001206076D5F80300C4F81A000A
:10EF2000B5F80700E0830BA904F1080015F0F6FA24
:10EF30004FF0010984F80091B4F84C0004F5827692
:10EF40004A46FB2828BFFB207989814238BF084602
:10EF500094F855104FF4747A11F00C0F1CBF0AEBA3
:10EF600080111FFA81FC72D0B989614538BF8C4687
:10EF7000B4F84A10FB2928BFFB21FB898B4238BF1C
:10EF8000194694F854B01BF00C0F1CBF0AEB811308
:10EF90009BB265D03F8A9F4238BF3B461B2918BFB2
:10EFA000B3F5A47F65D0F080A6F808C07180B38067
:10EFB00021463046FFF73EFCB08840F648018842C3
:10EFC00028BF40F64800B0803089884228BF40F60C
:10EFD0004800308186F800908DF800800121684655
:10EFE00004F04EFE00E02BE09DF8000000F0070169
:10EFF000C0F3C1021144C0F3401008448DF8000072
:10F00000401D207609283CBF08302076002120468C
:10F010000DF047F868780EF0B9FEA9782878EA1C58
:10F020000EF087FE002808BF122650D00EF0B8FE62
:10F03000A9782878EA1C0EF01BFF06001FD046E0D6
:10F0400010F0020F14BF022100214FE7FFE7022951
:10F0500007BF81003C31C10070311FFA81FC83E79A
:10F06000BBF1020F07BF8B003C33CB0070339BB268
:10F0700090E71B2818BFBCF5A47F94D1ACE7012012
:10F080000EF04CFE060022D1214603200EF028FF90
:10F0900006001CD1687A8DF8000010F0010F05D031
:10F0A0006889ADF80200288AADF80400684611F0BE
:10F0B00098F9064695F83A00002818BF01200EF08E
:10F0C00033FE26B9204611F026F9060009D0208823
:10F0D00006F00FFB2088062101F07CFC002818BFF9
:10F0E000FFDF30460FB0BDE8F08F0146002049E653
:10F0F00038B5294C207870B911F018FE052805D0D4
:10F100000EF057F9A0F57F41FF3904D0684611F0A1
:10F11000CCF910B113E00C2038BD0098008806F03F
:10F12000E8FA00980621008801F054FC002818BF76
:10F13000FFDF012020701D480078FCF727FE00202B
:10F1400038BD70B4B0F802C08188C3880289448990
:10F150008089ACF1060640F67B45AE423CBF8E1F6F
:10F16000AE4214D28C4598BFB3F5FA7F3EBFA2F1F0
:10F170000A0C0F4D15EB0C0509D25B1C5943B1EB82
:10F18000820F04DA84429EBF002070BC704730209A
:10F1900070BC70474047020032060020F405002092
:10F1A0006800002022060020112233005C000020AD
:10F1B00089F3FFFF2DE9F047B0F802C004468188CB
:10F1C000C388028947898689ACF1060940F67B48E5
:10F1D00030200025C1453ABFA1F10609C145BDE86F
:10F1E000F0878C4598BFB3F5FA7F3DBFA2F10A0CBA
:10F1F000DFF8B48418EB0C08BDE8F0875B1C5943BA
:10F20000B1EB820FA8BFBDE8F087B74288BFBDE869
:10F21000F0872088062101F0CBFB68B190F8D01070
:10F2200090F8732042B9002918BF042904D0D0F8FF
:10F23000F8100A781AB106E00220BDE8F087D0F88D
:10F240004421127812B13A20BDE8F08705228A7174
:10F25000D0F8F8100D81D0F8F820A1885181D0F8AD
:10F26000F820E1889181D0F8F8202189D181D0F867
:10F27000F8100A894B899A429EBF8A79082A9A42D5
:10F2800024BF1220BDE8F08722884A80D0F8F80019
:10F29000022101700020BDE8F087F0B583B005467B
:10F2A0000DF0F2F8002802BF122003B0F0BD0026D6
:10F2B000FE4F012429467C70B81C15F02FF97E7092
:10F2C0006946062001F0FDFA002818BFFFDF6846F6
:10F2D00001F0D5FA002808BFBDF804500AD1029801
:10F2E00080F80041684601F0CAFA18B9BDF8040078
:10F2F000A842F4D103B00020F0BD10B50446008848
:10F30000062101F055FB68B190F8D01090F87320F9
:10F3100042B9002918BF042904D0D0F8F8100A789F
:10F3200012B105E0022010BDD0F8442112780AB1D4
:10F330003A2010BD90F8962012F0010F04BF0C2067
:10F3400010BDD4F80220D4F806304A608B60D0F8A3
:10F35000F81062898A81D0F8F810E268C1F80E20AE
:10F360002269C1F812206269C1F81620A269C1F8A9
:10F370001A20D0F8F82003211170D0F8F800218865
:10F380004180002010BDF8B515460E46044609F030
:10F39000F7F900281CBF0C20F8BD20781223EF28B5
:10F3A00073D86088ADF8000010F0100F4FF0000126
:10F3B0000CD010F0010F00F002021BD0B2B110F01F
:10F3C000080F08BF10F0040F1ED01AE010F0080F4D
:10F3D0007ED110F0200F18BF10F0030F78D110F07D
:10F3E000010F18BF10F0020F72D10DE010F0040FE2
:10F3F0000AD106E02AB110F0080F08BF10F0040F80
:10F4000002D010F00F0F63D1608810F0080F09D1FF
:10F41000D4E901C2624528BFBCF1200F58D3B2F134
:10F42000807F55D2227B002A52D0072A50D894F8E8
:10F430000DC0BCF1000F18BFBCF1010F05D0BCF12D
:10F44000020F18BFBCF1030F42D110F0040F05D119
:10F45000BCF1020F18BFBCF1030F07D1A27B002A39
:10F4600018BF012A34D110F0040F08D1627D002AA0
:10F4700018BF012A03D0022A18BF032A28D1E27D2F
:10F4800010F0100F02D0012A10D021E0012A18BF7D
:10F49000032A1DD110F0100F08D1627E012A1CBF73
:10F4A000022A032A14D1A27E0F2A11D8E27E002A52
:10F4B00018BF012A0CD1E27D1123032A08D010F0D5
:10F4C000100F04BF627E032A02D010F0400F01D05B
:10F4D0001846F8BD3170A17555B9FF208DF80000B0
:10F4E0006946002006F0EDFD6946002006F0D4FDD7
:10F4F0002046BDE8F84006F004BD002243E72DE9B0
:10F50000F0470446C0780F46122510B106F063FD9F
:10F5100050B1607804280AD094F8038094F80090E1
:10F520006678B8F1FB0F12D92846BDE8F08709F0DC
:10F5300027F90028F8D006F0A6FD0028F4D106F03F
:10F540009AFA002804BFE0780028EDD1E4E71FB163
:10F55000B8F11F0F23D9E7E706F08DFA28B1B8F10B
:10F560001F0F98BF032E07D0DEE7032E18BF042E0F
:10F5700002D0B8F1000FD7D009F002F9002818BF67
:10F58000032E04D0042E1CBF0C20BDE8F087484693
:10F5900006F069FA002804BF4220BDE8F087E07851
:10F5A00061781F2898BF03291CBF1120BDE8F08790
:10F5B000211D06F086FD0020BDE8F08700219EE7B2
:10F5C0002DE9F0470446C0788846122710B106F0AE
:10F5D00098FD38B16578042D04D0E67894F8009051
:10F5E000FB2E02D93846BDE8F087B8F1000F02D0F3
:10F5F0001F2E21D9F6E706F03EFA20B11F2E98BF44
:10F60000032D06D0EEE7032D18BF042D01D0002EE8
:10F61000E8D009F0B5F8002818BF032D04D0042D58
:10F620001CBF0C20BDE8F087484606F01CFA0028F5
:10F6300004BF4220BDE8F087E07861781F2898BFBA
:10F6400003291CBF1120BDE8F087211D06F024FD11
:10F650000020BDE8F0870021B2E72DE9F041044623
:10F660004078422582B0012808D8A07806F0FBF93E
:10F6700020B120781225012804D0A0B102B028467C
:10F68000BDE8F08106F04BFD20B1A0880028F5D040
:10F690008028F3D806F050FD90B160780028EDD0B6
:10F6A0002078012810D003E089F3FFFF3206002004
:10F6B00007F0EAFE044608F0DBFC002800F0EA80D0
:10F6C00002B00C20BDE8F08106F046FB38B906F028
:10F6D0001FFD002802BF122002B0BDE8F08109F032
:10F6E0004FF80028ECD106F07EF9A0F57F41FF39F4
:10F6F000E6D106F050FBA08842F2107100FB01F643
:10F70000A079314606F078FC06F0F4FC18B300222C
:10F71000072101A801F01AF9040002BF092002B074
:10F72000BDE8F081F6480321846020460CF072FBAE
:10F73000204607F0EBF8F34DA88AA4F84A00E88ABF
:10F74000A4F84C0006F097F968B1288B012108F065
:10F7500013FEA0620FE03146002008F063FD002890
:10F7600018BFFFDFA1E006F0E9FC2A8B0146104636
:10F7700008F002FEA06201460022204607F087FE44
:10F7800006F079F9002808BF06F0D8FCE87C009064
:10F79000AB7CEA8AA98A208801F0C5F9002818BF45
:10F7A000FFDF208805F0A4FF3146204608F03AFD2F
:10F7B000002818BFFFDF2146B4F84C00002204F5F2
:10F7C000CD76FB2828BFFB206B89834238BF1846C3
:10F7D00091F855304FF4747413F00C0F1CBF04EB08
:10F7E00080131FFA83FC38D0AF89674528BF67466E
:10F7F000B1F84A30FB2B28BFFB23B5F80EC09C455F
:10F8000038BF634691F854C01CF00C0F1CBF04EBCA
:10F81000831C1FFA8CF829D02C8A444528BF444603
:10F820001B2B18BFB4F5A47F2ED0F08037817380D6
:10F83000B4803046FEF7FEFFB08840F648018842AB
:10F8400028BF40F64800B0803089884228BF40F683
:10F85000480030810120307027E0022B07BF830071
:10F860003C33C30070331FFA83FCBDE7BCF1020FC9
:10F8700007BF4FEA830C0CF13C0C4FEAC30C0CF1B0
:10F88000700C1FFA8CF8C7E71B2818BFB7F5A47FC8
:10F89000CBD10AE04CB1208805F02BFF208807214E
:10F8A00001F098F8002818BFFFDF002002B0BDE883
:10F8B000F0810021D1E610B50C46072101F078F85F
:10F8C000002804BF022010BD90F8731109B10C206C
:10F8D00010BD90F86510142912BF152990F8C011B9
:10F8E0000029F4D12168C0F874116168C0F878115A
:10F8F000A168C0F87C11E168C0F88011012180F88E
:10F900007311002010BD10B5072101F051F8002837
:10F9100004BF022010BD90F8731109B10C2010BD76
:10F9200090F86510142918BF1529F7D1022180F825
:10F930007311002010BDF0B50E464BF68032122137
:10F9400083B0964217D8B6B1694600F049F900284D
:10F950001CBF03B0F0BD019800F15807841C258836
:10F960003246294638460CF00FFA2088A842F6D1D4
:10F9700003B00020F0BD03B00846F0BD10B582B062
:10F9800004460088694600F02BF900281CBF02B02D
:10F9900010BD0198A37800F1580190F82C209A42EC
:10F9A00002BF0C2002B010BD7F220A728A720022B0
:10F9B000CA72E17880F82D10217980F82E10A17894
:10F9C00080F82C1002B0104610BD10B582B00C4665
:10F9D000694600F005F900281CBF02B010BD01986F
:10F9E00090F87300002818BF0120207002B000209A
:10F9F00010BD30B583B00D461446694600F0F0F8EE
:10FA000000281CBF03B030BD019890F82C000128DD
:10FA10001EBF0C2003B030BD019890F86010297013
:10FA200090F86100207003B0002030BD70B50D4625
:10FA30001646072100F0BCFF002804BF022070BD5D
:10FA400083884FF0010CC28841880CEB430C65455C
:10FA50001AD342F2107C02FB0CF240F6C41C01FBEC
:10FA60000CF1B2FBF1F1491E8CB2B4F5FA7F88BFFC
:10FA70004FF4FA74A54238BF2C46621C591CB2FBE5
:10FA8000F1F25143491E8BB290F8AC11002908BF26
:10FA900003843380002070BD10B50C46072100F0B0
:10FAA00087FF002804BF022010BD80F8DF40002C33
:10FAB0001EBF90F8DD10002908F081FC002010BD69
:10FAC000017800291CBF417800290ED041881B29EC
:10FAD00021BF81881B29C188022906D30A490268EF
:10FAE00040680A654865002070471220704710B5CD
:10FAF000044610F005FD204608F009FC002010BD6A
:10FB00005C00002032060020F40500202DE9F041C1
:10FB100016460F46044601221146384610F0F3FC03
:10FB200005460121384608F027FC854228BF2846B3
:10FB30000123E100503189B2E631884206D901F152
:10FB40009602401AB0FBF2F0401C83B233800020D2
:10FB5000BDE8F08110B5044611F0E8F8042806D09D
:10FB600011F0E4F8052802D008F00AFE08B10C20D4
:10FB700010BD601C0BF05DFF207800F0010006F066
:10FB800005F9207800F001000EF005F9002010BD05
:10FB900010B50446072000F0A5FE00281CBF0C206D
:10FBA00010BD207810F0010F11D0002260781146AE
:10FBB00013F0B8FC00281CBF122010BDA0680AF08A
:10FBC00048FA607861680AF04DFA002010BD002004
:10FBD0000AF03FFA002108460AF044FA002010BD5E
:10FBE00070B50C460546062100F0E2FE606010B1DB
:10FBF0000020207070BD0721284600F0D9FE60600B
:10FC0000002804BF022070BD01202070002070BDBC
:10FC100010B582B0044600886946FFF7E1FF020094
:10FC20001CBF02B010BDA088002818BF012804D056
:10FC300002281EBF122002B010BDA178002908BF03
:10FC40000321E078002808BF03204FF0000C9DF846
:10FC500000400123002C019C06D084F8A531019CB2
:10FC600094F8F241ECB124E084F80F31019C94F84F
:10FC700034413CB9019C94F80E411CB9019C94F8A4
:10FC80007D400CB13A2208E0019C84F80E31019BC2
:10FC900083F81011019981F81101019880F80FC1C2
:10FCA00015E0019C94F8A4411CB9019C94F87D4096
:10FCB0000CB13A2208E0019C84F8A431019B83F83E
:10FCC000A611019981F8A701019880F8A5C102B099
:10FCD000104610BD427A12F0070F10D032F0070321
:10FCE0000DD112F0040F01D011207047012A18BF66
:10FCF000022AF9D190F83A301BB9012A01D012201A
:10FD000070472DE9F0074FF0000C12F0010F40F69C
:10FD1000774740F67B4337D069B14489B0F810C0CB
:10FD2000261F43F6FD75AE423CBFACF10406AE4261
:10FD300026D2644524D3C68AB0F81CC0448C058DF5
:10FD4000B0F82E90B0F83480A6F1060A9A453CBF70
:10FD5000ACF1060A9A4513D2664598BFB4F5FA7F0E
:10FD60003CBFA5F10A06BE420AD2641C04FB0CFC8F
:10FD7000BCEB850F04DAC14598BF4FF0010C03D9E5
:10FD8000BDE8F0073020704712F0020F22D000EBE0
:10FD90004C02D68AB2F81CC0558C148DB2F82E8055
:10FDA000928EA6F106094B4584BFACF106094B457E
:10FDB000E6D9664598BFB5F5FA7F3CBFA4F10A03C2
:10FDC000BB42DDD26B1C03FB0CF3B3EB840FD7DA21
:10FDD0009045D5D802782AB1012A13D0BDE8F007A2
:10FDE000122070470029817808D0002918BF012906
:10FDF00008D0022918BF032904D0EFE7002918BF53
:10FE00000129EBD14078002818BF012803D002282F
:10FE100018BF0328E2D1BDE8F007002070470000BA
:10FE200030B5058825F4004421448CB24FF40041DC
:10FE300094420AD2121B92B21B339A4201D2A943B6
:10FE400007E005F40041214303E0A21A92B2A9435E
:10FE50001143018030BD0844083050434A31084402
:10FE600080B2704770B51D4616460B4604462946BB
:10FE70003046049AFFF7EFFF0646B34200D2FFDF99
:10FE80002821204614F035FA4FF6FF70A082283E54
:10FE9000B0B265776080B0F5004F00D9FFDF6188B0
:10FEA00005F13C00814200D2FFDF60880835401B2D
:10FEB000343880B220801B2800D21B2020800020F4
:10FEC000A07770BD8161886170472DE9F05F0D46B4
:10FED000C188044600F12809008921F4004620F475
:10FEE000004800F062FB10B10020BDE8F09F4FF029
:10FEF000000A4FF0010BB0450CD9617FA8EB06005A
:10FF0000401A0838854219DC09EB060000210580FB
:10FF100041801AE06088617F801B471A083F0DD43A
:10FF20001B2F00DAFFDFBD4201DC294600E0B9B239
:10FF3000681A0204120C04D0424502DD84F817A0AE
:10FF4000D2E709EB06000180428084F817B0CCE7C5
:10FF500070B5044600F12802C088E37D20F400401B
:10FF60002BB110440288438813448B4201D20020F5
:10FF700070BD00258A4202D30180458008E0891ABD
:10FF80000904090C418003D0A01D00F01EFB08E00D
:10FF9000637F00880833184481B26288A01DFFF790
:10FFA0003FFFE575012070BD70B5034600F12804E0
:10FFB000C588808820F400462644A84202D100204B
:10FFC000188270BD98893588A84206D3401B758871
:10FFD0002D1A2044ADB2C01E05E02C1AA5B25C7FDC
:10FFE00020443044401D0C88AC4200D90D809C89CF
:10FFF00024B1002414700988198270BD0124F9E726
:020000040001F9
:1000000070B5044600F12801808820F400404518AE
:10001000208A002825D0A189084480B2A08129889F
:100020006A881144814200D2FFDF2888698800264F
:100030000844A189884212D1A069807F287169880B
:1000400019B1201D00F0C1FA08E0637F2888083349
:10005000184481B26288201DFFF7E2FEA681268245
:10006000012070BD2DE9F0414189878800260446B2
:1000700000F12805B94218D004F10A0821F4004023
:100080002844418819B1404600F09FFA08E0637F98
:1000900000880833184481B262884046FFF7C0FEEA
:1000A000761C6189B6B2B942E8D13046BDE8F0812C
:1000B0002DE9F04104460B4627892830A68827F40D
:1000C0000041B4F80A8001440D46B74201D1002036
:1000D000ECE70AB1481D106023B1627F691D184624
:1000E00014F066F82E88698804F1080021B18A1995
:1000F00096B200F06AFA06E0637F628808339919C5
:1001000089B2FFF78DFE474501D1208960813046D5
:10011000CCE78188C088814201D10120704700204E
:10012000704701898088814201D1012070470020F9
:10013000704770B58588C38800F1280425F4004213
:1001400023F4004114449D421AD08389058A5E1924
:1001500025886388EC18A64214D313B18B4211D3BF
:100160000EE0437F08325C192244408892B2801A24
:1001700080B22333984201D211B103E08A4201D107
:10018000002070BD012070BD2DE9F0478846C18870
:100190000446008921F4004604F1280720F40045B4
:1001A00007EB060900F001FA002178BBB54204D93B
:1001B000627FA81B801A002503E06088627F801B95
:1001C000801A083823D4E28962B1B9F80020B9F85E
:1001D00002303BB1E81A2177404518DBE08938440A
:1001E000801A09E0801A217740450ADB607FE189A7
:1001F0000830304439440844C01EA4F81280BDE8D9
:10020000F087454503DB01202077E7E7FFE76182C0
:100210000020F4E72DE9F74F044600F12805C088D7
:10022000884620F4004A608A05EB0A0608B140457A
:1002300002D20020BDE8FE8FE08978B13788B6F899
:10024000029007EB0901884200D0FFDF207F4FF0CA
:10025000000B50EA090106D088B33BE00027A07FDD
:10026000B9463071F2E7E18959B1607F294408301D
:1002700050440844B4F81F1020F8031D94F82110CE
:100280008170E28907EB080002EB0801E181308010
:10029000A6F802B002985F4650B1637F30880833F9
:1002A000184481B26288A01DFFF7BAFDE78121E002
:1002B000607FE18908305044294408442DE0FFE77D
:1002C000E089B4F81F102844C01B20F8031D94F8DF
:1002D0002110817009EB0800E28981B202EB08006D
:1002E000E081378071800298A0B1A01D00F06DF907
:1002F000A4F80EB0A07F401CA077A07D08B1E088D4
:10030000A08284F816B000BFA4F812B084F817B029
:1003100001208FE7E0892844C01B30F8031DA4F8B2
:100320001F10807884F82100EEE710B5818800F175
:10033000280321F400442344848AC288A14212D0B5
:10034000914210D0818971B9826972B11046FFF76C
:10035000E8FE50B91089283220F400401044197981
:100360000079884201D1002010BD184610BD00F16F
:100370002803407F08300844C01E1060088808B970
:10038000DB1E136008884988084480B270472DE955
:10039000F04100F12806407F1C4608309046431883
:1003A00008884D88069ADB1EA0B1C01C80B290421E
:1003B00014D9801AA04200DB204687B298183A462A
:1003C000414613F0C9FE002816D1E01B84B2B844A0
:1003D000002005E0ED1CADB2F61EE8E7101A80B271
:1003E0000119A94206D8304422464146BDE8F041F1
:1003F00013F0B2BE4FF0FF3058E62DE9F04100F1A6
:100400002804407F1E46083090464318002508887F
:100410004F88069ADB1E90B1C01C80B2904212D960
:10042000801AB04200DB304685B299182A46404611
:1004300013F0BEFE701B86B2A844002005E0FF1C2E
:10044000BFB2E41EEAE7101A80B28119B94206D899
:1004500021183246404613F0ABFEA81985B2284653
:1004600024E62DE9F04100F12804407F1E460830C3
:1004700090464318002508884F88069ADB1E90B1E5
:10048000C01C80B2904212D9801AB04200DB3046C4
:1004900085B298182A46414613F08AFE701B86B230
:1004A000A844002005E0FF1CBFB2E41EEAE7101AD2
:1004B00080B28119B94206D820443246414613F031
:1004C00077FEA81985B22846F0E5401D704710B5A3
:1004D000044600F12801C288808820F400431944B2
:1004E000904206D0A28922B9228A12B9A28A9042E9
:1004F00001D1002010BD0888498831B1201D00F0CD
:1005000064F800202082012010BD637F62880833D8
:10051000184481B2201DFFF783FCF2E70021C1815E
:1005200001774182C1758175704703881380C28944
:1005300042B1C28822F4004300F128021A440A6042
:10054000C08970470020704710B50446808AA0F526
:100550007F41FF3900D0FFDFE088A082E08900B151
:100560000120A07510BD4FF6FF71818200218175B9
:10057000704710B50446808AA0F57F41FF3900D14D
:10058000FFDFA07D28B9A088A18A884201D1002080
:1005900010BD012010BD8188828A914201D1807DE9
:1005A00008B1002070470120704720F4004221F478
:1005B00000439A4207D100F4004001F40041884210
:1005C00001D0012070470020704730B504460088F4
:1005D0000D4620F40040A84200D2FFDF21884FF4EE
:1005E000004088432843208030BD70B50C0005468C
:1005F00009D0082C00D2FFDF1DB1A1B2286800F09D
:1006000044F8201D70BD0DB100202860002070BD91
:100610000021026803E093881268194489B2002A15
:10062000F9D100F032B870B500260D46044608290D
:1006300000D2FFDF206808B91EE0044620688188E8
:10064000A94202D001680029F7D181880646A94253
:1006500001D100680DE005F1080293B20022994231
:1006600009D32844491B0260818021680968216000
:100670000160206000E00026304670BD00230B6062
:100680008A8002680A600160704700234360021D8F
:10069000018102607047F0B50F4601884088154619
:1006A0000C181E46AC4200D3641B3044A84200D94B
:1006B000FFDFA019A84200D9FFDF3819F0BD2DE9EE
:1006C000F041884606460188408815460C181F46AA
:1006D000AC4200D3641B3844A84200D9FFDFE019C4
:1006E000A84200D9FFDF70883844708008EB04000E
:1006F000BDE8F0812DE9F041054600881E46174609
:10070000841B8846BC4200D33C442C80688830441B
:10071000B84200D9FFDFA019B84200D9FFDF6888CE
:100720003044688008EB0400E2E72DE9F0410688D8
:100730001D460446701980B2174688462080B8428C
:1007400001D3C01B20806088A84200D2FFDF70194F
:10075000B84200D9FFDF6088401B608008EB0600CC
:10076000C6E730B50D460188CC18944200D3A41AD0
:100770004088984200D8FFDF281930BD2DE9F041AC
:10078000C84D04469046A8780E46A04200D8FFDF28
:1007900005EB8607B86A50F8240000B1FFDFB8689F
:1007A000002816D0304600F044F90146B868FFF73B
:1007B0003AFF05000CD0B86A082E40F8245000D348
:1007C000FFDFB9484246294650F826302046984770
:1007D0002846BDE8F0812DE9F8431E468C19914664
:1007E0000F460546FF2C00D9FFDFB14500D9FFDFDA
:1007F000E4B200954DB300208046E81C20F00300D1
:10080000A84200D0FFDF4946DFF89892684689F891
:10081000001089F8017089F8024089F8034089F8CE
:10082000044089F8054089F8066089F80770414658
:1008300000F008F9002142460F464B460098C01CC4
:1008400020F00300009012B10EE00120D4E703EB8A
:100850008106B062002005E0D6F828C04CF8207070
:10086000401CC0B2A042F7D30098491C00EB8400A2
:10087000C9B200900829E1D3401BBDE8F88310B548
:10088000044603F071FD08B1102010BD2078854AA0
:10089000618802EB800092780EE0836A53F8213081
:1008A00043B14A1C6280A180806A50F82100A06098
:1008B000002010BD491C89B28A42EED86180052013
:1008C00010BD70B505460C46084603F04DFD08B155
:1008D000102070BD082D01D3072070BD25700020A9
:1008E000608070BD0EB56946FFF7EBFF00B1FFDF1A
:1008F0006846FFF7C4FF08B100200EBD01200EBD01
:1009000010B50446082800D3FFDF6648005D10BD1F
:100910003EB5054600246946FFF7D3FF18B1FFDF57
:1009200001E0641CE4B26846FFF7A9FF0028F8D094
:100930002846FFF7E5FF001BC0B23EBD5949897844
:10094000814201D9C0B27047FF2070472DE9F041C4
:10095000544B062903D007291CD19D7900E00025BE
:1009600000244FF6FF7603EB810713F801C00AE07D
:100970006319D7F828E09BB25EF823E0BEF1000FC0
:1009800004D0641CA4B2A445F2D8334603801846B0
:10099000B34201D100201CE7BDE8F041EEE6A0F52E
:1009A0007F43FF3B01D0082901D300207047E5E6D3
:1009B000A0F57F42FF3A0BD0082909D2394A937833
:1009C000834205D902EB8101896A51F82000704702
:1009D000002070472DE9F04104460D46A4F57F4103
:1009E00043F20200FF3902D0082D01D30720F0E6C0
:1009F0002C494FF000088A78A242F8D901EB85060D
:100A0000B26A52F82470002FF1D0274839462030BE
:100A100050F8252020469047B16A284641F82480A6
:100A200000F007F802463946B068FFF727FE0020BD
:100A3000CFE61D49403131F810004FF6FC71C01C63
:100A4000084070472DE9F843164E884605460024B5
:100A50002868C01C20F0030028602046FFF7E9FF4B
:100A6000315D4843B8F1000F01D0002200E02A6850
:100A70000146009232B100274FEA0D00FFF7B5FDA5
:100A80001FB106E001270020F8E706EB8401009A79
:100A90008A602968641C0844E4B22860082CD7D313
:100AA000EBE60000500600204C47020070B50E46F1
:100AB0001D46114600F0D4F804462946304600F0A1
:100AC000D8F82044001D70BD2DE9F04190460D4638
:100AD00004004FF0000610D00027E01C20F00300B7
:100AE000A04200D0FFDFDDB141460020FFF77DFDD1
:100AF0000C3000EB850617B112E00127EDE7614FDE
:100B000004F10C00A9003C602572606000EB8500D8
:100B10002060606813F0EDFB41463868FFF765FD23
:100B20003046BDE8F0812DE9FF4F564C804681B03C
:100B300020689A46934600B9FFDF2068027A424552
:100B400003D9416851F8280020B143F2020005B0F2
:100B5000BDE8F08F5146029800F082F886B2584600
:100B60000E9900F086F885B27019001D87B22068D2
:100B7000A14639460068FFF756FD04001FD0678084
:100B800025802946201D0E9D07465A4601230095C3
:100B9000FFF768F92088314638440123029ACDF8DE
:100BA00000A0FFF75FF92088C1193846FFF78AF9DE
:100BB000D9F800004168002041F82840C7E7042028
:100BC000C5E770B52F4C0546206800B9FFDF2068E7
:100BD000017AA9420ED9426852F8251051B100237A
:100BE00042F825304A880068FFF748FD2168002058
:100BF0000A7A08E043F2020070BD4B6853F82030D7
:100C000033B9401CC0B28242F7D80868FFF700FD34
:100C1000002070BD70B51B4E05460024306800B939
:100C2000FFDF3068017AA94204D9406850F82500F6
:100C300000B1041D204670BD70B5124E054600245B
:100C4000306800B9FFDF3068017AA94206D94068F0
:100C500050F8251011B131F8040B4418204670BD2E
:100C600010B50A460121FFF7F6F8C01C20F003007A
:100C700010BD10B50A460121FFF7EDF8C01C20F0A9
:100C8000030010BD7000002070B50446C2F11005CD
:100C9000281913F08DFA15F0FF0108D0491EC9B2CA
:100CA000802060542046BDE8704013F000BB70BD4A
:100CB00030B505E05B1EDBB2CC5CD55C6C40C45447
:100CC000002BF7D130BD10B5002409E00B78521E7F
:100CD00044EA430300F8013B11F8013BD2B2DC09BE
:100CE000002AF3D110BD2DE9F04389B01E46DDE99D
:100CF000107990460D00044622D002460846F94974
:100D0000FDF77CFC102221463846FFF7DCFFE07B34
:100D1000000606D5F34A3946102310320846FFF77D
:100D2000C7FF102239464846FFF7CDFFF87B000683
:100D300006D5EC4A4946102310320846FFF7B8FFA3
:100D40001021204613F0B3FA0DE0103EB6B208EBC6
:100D50000601102322466846FFF7AAFF22462846CE
:100D60006946FDF74BFC102EEFD818D0F2B2414681
:100D70006846FFF789FF10234A46694604A8FFF733
:100D800097FF1023224604A96846FFF791FF2246E9
:100D900028466946FDF732FC09B0BDE8F083102310
:100DA0003A464146EAE770B59CB01E4605461346F2
:100DB00020980C468DF80800202219460DF10900F4
:100DC00013F0F6F9202221460DF1290013F0F0F975
:100DD00017A913A8CDE90001412302AA31462846EC
:100DE000FFF781FF1CB070BD2DE9FF4F9FB014AE1F
:100DF000DDE92D5410AFBB49CDE900762023203129
:100E00001AA8FFF770FF4FF000088DF808804FF028
:100E100001098DF8099054F8010FCDF80A00A08857
:100E2000ADF80E0014F8010C1022C0F340008DF84C
:100E3000100055F8010FCDF81100A888ADF8150085
:100E400015F8010C2C99C0F340008DF8170006A886
:100E5000824613F0ADF90AA883461022229913F0B6
:100E6000A7F9A0483523083802AA40688DF83C80CD
:100E7000CDE900760E901AA91F98FFF734FF8DF880
:100E800008808DF809902068CDF80A00A088ADF898
:100E90000E0014F8010C1022C0F340008DF8100071
:100EA0002868CDF81100A888ADF8150015F8010CD8
:100EB0002C99C0F340008DF81700504613F078F9D4
:100EC00058461022229913F073F9864835230838C2
:100ED00002AA40688DF83C90CDE900760E901AA9E0
:100EE0002098FFF700FF23B0BDE8F08FF0B59BB06E
:100EF0000C460546DDE922101E461746DDE9203284
:100F0000D0F801C0CDF808C0B0F805C0ADF80CC0ED
:100F10000078C0F340008DF80E00D1F80100CDF844
:100F20000F00B1F80500ADF8130008781946C0F3BA
:100F300040008DF815001088ADF8160090788DF8F7
:100F400018000DF11900102213F032F90DF12900EB
:100F50001022314613F02CF90DF1390010223946D8
:100F600013F026F917A913A8CDE90001412302AA1D
:100F700021462846FFF7B7FE1BB0F0BDF0B5A3B081
:100F800017460D4604461E46102202A8289913F063
:100F90000FF906A82022394613F00AF90EA82022DC
:100FA000294613F005F91EA91AA8CDE9000150231E
:100FB00002AA314616A8FFF796FE1698206023B0C5
:100FC000F0BDF0B589B00446DDE90E070D4639786D
:100FD000109EC1F340018DF8001031789446C1F3A2
:100FE00040018DF801101968CDF802109988ADF80C
:100FF000061099798DF808100168CDF809108188DC
:10100000ADF80D1080798DF80F0010236A46614607
:1010100004A8FFF74DFE2246284604A9FDF7EEFA84
:10102000D6F801000090B6F80500ADF80400D7F836
:101030000100CDF80600B7F80500ADF80A00002061
:10104000039010236A46214604A8FFF731FE22468A
:10105000284604A9FDF7D2FA09B0F0BD1FB51C68F7
:1010600000945B68019313680293526803920246EE
:1010700008466946FDF7C2FA1FBD10B588B00446A0
:10108000106804905068059000200690079008466C
:101090006A4604A9FDF7B2FABDF80000208008B046
:1010A00010BD1FB51288ADF800201A88ADF80220D7
:1010B0000022019202920392024608466946FDF719
:1010C0009DFA1FBD7FB5074B14460546083B9A1C89
:1010D0006846FFF7E6FF224669462846FFF7CDFF40
:1010E0007FBD0000A447020070B5044600780E469C
:1010F000012813D0052802D0092813D10EE0A068DA
:1011000061690578042003F0BDF8052D0AD0782325
:1011100000220420616903F00BF803E004206169F8
:1011200003F0B0F831462046BDE8704001F086B8C3
:1011300010B500F12D02C3799478411D64F00304C9
:101140002340C371DB070DD04B79547923404B7199
:101150000B79127913400B718278C9788A4200D9D1
:10116000817010BD00224A710A71F5E741780129AA
:1011700000D00C21017070472DE9F04F93B04FF073
:10118000000B0C690D468DF820B0097801260C2063
:1011900017464FF00D084FF0110A4FF008091B29B0
:1011A00075D2DFE811F01B00C30206031E035D03C6
:1011B0007003A203B703F803190461049304A004A5
:1011C000EC042A05340552055D05EE0531063406AA
:1011D00063067F06F9061D07E606EB0614B12078C4
:1011E0001D282AD0D5F808805FEA08004FD00120DA
:1011F0008DF82000686A02220D908DF824200A20C4
:101200008DF82500A8690A90A8880028EED098F8E3
:10121000001091B10F2910D27ED2DFE801F07D13CA
:1012200049DEFEFDFCFBFAF938089CF8F7000228BD
:101230002DD124B120780C2801D00026EFE38DF8C1
:101240002020CBE10420696A03F01CF8A888072855
:10125000EED1204600F0EDFF022809D0204600F034
:10126000E8FF032807D9204600F0E3FF072802D251
:101270000120207004E0002CB8D020780128D7D1BC
:1012800098F80400C11F0A2902D30A2061E0C4E1D2
:10129000A070D8F80010E162B8F80410218698F820
:1012A000060084F83200012028700320207044E0FA
:1012B0000728BDD1002C99D020780D28B8D198F8F6
:1012C000031094F82F20C1F3C000C2F3C0021042F3
:1012D00001D0062000E00720890707D198F8051003
:1012E0000142D2D198F806100142CED194F83120B3
:1012F00098F8051020EA02021142C6D194F8322073
:1013000098F8061090430142BFD198F80400C11F1D
:101310000A29BAD2617D00E006E281427ED8D8F87F
:1013200000106160B8F80410218198F80600A072DE
:10133000012028700E20207003208DF82000686A9C
:101340000D9004F12D000990601D0A900F300B9054
:1013500022E12875FDE3412891D1204600F069FF84
:10136000042802D1E078C00704D1204600F061FFD4
:101370000F2884D1A88CD5F80C8080B24FF0400B98
:10138000E669FFF747FC324641465B464E46CDF8DC
:101390000090FFF732F80B208DF82000686A0D905E
:1013A000E0690990002108A8FFF79EFE2078042834
:1013B00006D0A07D58B1012809D003280AD049E3FE
:1013C00005202070032028708DF82060CDE184F87E
:1013D00000A032E712202070E9E11128BCD120469C
:1013E00000F027FF042802D1E078C00719D020467A
:1013F00000F01FFF062805D1E078C00711D1A07DBD
:1014000002280ED0204600F014FF08E0CAE081E078
:101410006FE14EE121E101E1E7E017E0ADE11128E4
:101420009AD1102208F1010104F13C0012F0C0FE33
:10143000607801287ED012202070E078C00760D04C
:10144000A07D0028C8D00128C6D05AE0112890D12C
:10145000204600F0EEFE082804D0204600F0E9FE09
:10146000132886D104F16C00102208F10101064610
:1014700012F09EFE207808280DD014202070E1780C
:10148000C8070DD0A07D02280AD06278022A04D0B5
:101490000328A1D035E00920F0E708B1012837D1B1
:1014A000C80713D0A07D02281DD000200090D4E9E9
:1014B000062133460EA8FFF776FC10220EA904F190
:1014C0003C0012F049FEC8B1042042E7D4E90912F9
:1014D000201D8DE8070004F12C0332460EA8616B35
:1014E000FFF76FFDE9E7606BC1F34401491E006837
:1014F000C84000F0010040F08000D7E720780928BC
:1015000006D185F800908DF8209033E32870ECE345
:101510000920FBE711289AD1204600F08AFE0A280C
:1015200002D1E078C00704D1204600F082FE1528E1
:101530008DD100E08DE104F13C00102208F10101A1
:10154000064612F035FE20780A2816D016202070A4
:10155000D4E90932606B611D8DE80F0004F15C0372
:1015600004F16C0247310EA8FFF7C0FC10220EA94F
:10157000304612F0F1FD18B1F5E20B20207071E257
:101580002046FFF7D5FDA078216A0A18C0F11001A6
:10159000104612F08CFE23E3394608A8FFF7A4FD9D
:1015A00006463BE20228B6D1204600F042FE04285F
:1015B00004D3204600F03DFE082809D3204600F061
:1015C00038FE0E2829D3204600F033FE122824D2FC
:1015D000A07D02289FD10E208DF82000686A0D9012
:1015E00098F801008DF82400F0E3022893D12046FA
:1015F00000F01FFE002810D0204600F01AFE01283F
:10160000F9D0204600F015FE0C28F4D004208DF807
:10161000240098F801008DF825005EE21128FCD125
:10162000002CFAD020781728F7D16178606A022957
:1016300011D0002101EB4101182606EBC101102257
:10164000405808F1010112F0B3FD0420696A00F06E
:10165000E3FD2670F1E50121ECE70B28DDD1002C3C
:10166000DBD020781828D8D16078616A02281CD095
:101670005FF0000000EB4002102000EBC2000958B0
:10168000B8F8010008806078616A02280FD0002055
:1016900000EB4002142000EBC2000958404650F80D
:1016A000032F0A604068486039E00120E2E701202A
:1016B000EEE71128B1D1002CAFD020781928ACD199
:1016C0006178606A022912D05FF0000101EB4101EC
:1016D0001C2202EBC1011022405808F1010112F056
:1016E00067FD0420696A00F097FD1A20B6E0012129
:1016F000ECE7082891D1002C8FD020781A288CD1C3
:10170000606A98F80120017862F347010170616A0C
:10171000D8F8022041F8012FB8F80600888004208C
:10172000696A00F079FD8EE2072012E63878012818
:1017300094D1182204F11400796812F07EFDE0794A
:10174000C10894F82F0001EAD001E07861F30000AD
:10175000E070217D002974D12178032909D0C007C8
:1017600025D0032028708DF82090686A0D904120C4
:1017700004E3607DA178884201D90620E9E50226CC
:101780002671E179204621F0E001E171617A21F0D2
:10179000F0016172A17A21F0F001A172FFF7C8FC9B
:1017A0002E708DF82090686A0D900720E6E20420E4
:1017B000ACE6387805289DD18DF82000686A0D9038
:1017C000B8680A900720ADF824000A988DF830B068
:1017D0006168016021898180A17A81710420207073
:1017E000F4E23978052985D18DF82010696A0D91C8
:1017F000391D09AE0EC986E80E004121ADF824104E
:101800008DF830B01070A88CD7F80C8080B24026CC
:10181000A769FFF711FA41463A463346C846CDF864
:101820000090FEF71EFE002108A8FFF75DFCE0789F
:1018300020F03E00801CE0702078052802D00F20A8
:101840000CE049E1A07D20B1012802D0032802D09C
:1018500002E10720BFE584F80080EEE42070ECE4AC
:10186000102104F15C0002F034FA606BB0BBA07D83
:1018700018B1012801D00520FDE006202870F748A6
:101880006063A063BEE23878022894D1387908B149
:101890002875B3E3A07D022802D0032805D022E0FA
:1018A000B8680028F5D060631CE06078012806D095
:1018B000A07994F82E10012805D0E84806E0A17917
:1018C00094F82E00F7E7B8680028E2D06063E0786B
:1018D000C00701D0012902D0E04803E003E0F86826
:1018E0000028D6D0A063062010E68DF82090696A03
:1018F0000D91E1784846C90709D06178022903D1E2
:10190000A17D29B1012903D0A17D032900D00720A1
:10191000287031E138780528BBD1207807281ED0FF
:1019200084F800A005208DF82000686A0D90B86842
:101930000A90ADF824A08DF830B003210170E17851
:10194000CA070FD0A27D022A1AD000210091D4E943
:10195000061204F15C03401CFFF725FA67E384F8E4
:101960000090DFE7D4E90923211D8DE80E0004F182
:101970002C0304F15C02401C616BFFF722FB56E371
:10198000626BC1F34401491E1268CA4002F00101B2
:1019900041F08001DAE738780528BDD18DF82000C4
:1019A000686A0D90B8680A90ADF824A08DF830B040
:1019B000042100F8011B102204F15C0112F0F8FB75
:1019C000002108A8FFF790FB2078092801D01320F8
:1019D00044E70A2020709BE5E078C10742D0A17D52
:1019E000012902D0022927D038E0617808A801290E
:1019F00016D004F16C010091D4E9061204F15C03E5
:101A0000001DFFF7BBFA0A20287003268DF82080FE
:101A1000686A0D90002108A8FFF766FBDDE2C3E2CB
:101A200004F15C010091D4E9062104F16C03001D6E
:101A3000FFF7A4FA0026E9E7C0F3440114290DD208
:101A40004FF0006101EBB0104FEAB060E0706078D9
:101A5000012801D01020BEE40620FFE660780128AE
:101A60003FF4B7AC0A2051E5E178C90708D0A17D61
:101A7000012903D10B20287004202FE028702DE0CD
:101A80000E2028706078616B012817D004F15C0388
:101A900004F16C020EA8FFF7E1FA2046FFF748FBBD
:101AA000A0780EAEC0F11001304412F000FC062008
:101AB0008DF82000686A09960D909AE004F16C0395
:101AC00004F15C020EA8FFF7C9FAE9E739780229A8
:101AD00003D139790029D1D029758FE28DF8200002
:101AE000686A0D9058E538780728F6D1D4E90921BD
:101AF0006078012808D004F16C00CDE90002029161
:101B000005D104F16C0304E004F15C00F5E704F195
:101B10005C0304F14C007A680646216AFFF764F919
:101B20006078012821D1A078216A0A18C0F110013B
:101B3000104612F0BCFBD4E90923606B04F12D01BF
:101B40008DE80F0004F15C0304F16C0231460EA82D
:101B500000E055E2FFF7CAF910220EA904F13C009B
:101B600012F0FAFA08B10B20AFE485F8008000BF4C
:101B70008DF82090686A0D908DF824A00CE53878D7
:101B80000528AAD18DF82000686A0D90B8680A90DF
:101B9000ADF824A08DF830B080F80080617801297C
:101BA0001AD0D4E9093204F12D01A66B03920096F4
:101BB000CDE9011304F16C0304F15C0204F14C0162
:101BC000401CFFF793F9002108A8FFF78DFA607811
:101BD000012805D0152041E6D4E90923611DE4E779
:101BE0000E20287006208DF82000686ACDF824B0F9
:101BF0000D90A0788DF82800CEE438780328C0D165
:101C0000E079C00770D00F202870072066E7387889
:101C100004286BD11422391D04F1140012F00DFBBD
:101C2000616A208CA1F80900616AA078C871E17925
:101C3000626A01F003011172616A627A0A73616A71
:101C4000A07A81F82400162060E485F800A08DF8C1
:101C50002090696A50460D9190E00000A447020070
:101C60003878052842D1B868A8616178606A02298D
:101C700001D0012100E0002101EB4101142606EB17
:101C8000C1014058082102F024F86178606A0229F5
:101C900001D0012100E0002101EB410106EBC1016F
:101CA000425802A8E169FFF70DFA6078626A0228DB
:101CB00001D0012000E0002000EB4001102000EBEB
:101CC000C1000223105802A90932FEF7F1FF626A2F
:101CD000FD4B0EA80932A169FFF7E3F96178606A4C
:101CE000022904D0012103E042E18BE0BDE00021A4
:101CF00001EB4101182606EBC101A27840580EA95C
:101D000012F056FA6178606A022901D0012100E0E0
:101D1000002101EB410106EBC1014058A1780844C4
:101D2000C1F1100112F0C3FA05208DF82000686A95
:101D30000D90A8690A90ADF824A08DF830B0062166
:101D400001706278616A022A01D0012200E000225B
:101D500002EB420206EBC202401C8958102212F02C
:101D600027FA002108A8FFF7BFF91220C5F818B01C
:101D700028708DF82090686A0D900B208DF8240053
:101D80000AE43878052870D18DF82000686A0D9033
:101D9000B8680A900B20ADF824000A98072101705A
:101DA0006178626A022901D0012100E0002101EB83
:101DB0004103102101EBC30151580988A0F801101B
:101DC0006178626A022902D0012101E02FE100213D
:101DD00001EB4103142101EBC30151580A6840F89B
:101DE000032F4968416059E01920287001208DF8BF
:101DF000300077E6162028708DF830B0002108A852
:101E0000FFF772F9032617E114202870B0E638783E
:101E100005282AD18DF82000686A0D90B8680A90CC
:101E2000ADF824A08DF830B080F800906278616A37
:101E30004E46022A01D0012200E0002202EB4202BB
:101E40001C2303EBC202401C8958102212F0B0F987
:101E5000002108A8FFF748F9152028708DF82060A8
:101E6000686A0D908DF824603CE680E0387805289B
:101E70007DD18DF82000686A0D90B8680A90ADF8A1
:101E800024900921017061690978490841706169EC
:101E900051F8012FC0F802208988C18020781C28C1
:101EA000A8D1A1E7E078C00702D04FF0060C01E00E
:101EB0004FF0070C607802280AD04FF0000000BFF6
:101EC00000EB040101F1090105D04FF0010004E02D
:101ED0004FF00100F4E74FF000000B78204413EAC4
:101EE0000C030B7010F8092F02EA0C02027004D1E7
:101EF0004FF01B0C84F800C0D2B394F801C0BCF1C1
:101F0000010F00D09BB990F800C0E0465FEACC7C9E
:101F100004D028F001060670102606E05FEA887CEF
:101F200005D528F00206067013262E70032694F8B5
:101F300001C0BCF1020F00D092B991F800C05FEA75
:101F4000CC7804D02CF001060E70172106E05FEA71
:101F50008C7805D52CF002060E7019212170002610
:101F60000078D0BBCAB3C3BB1C20207035E012E0A0
:101F700002E03878062841D11A2019E42078012897
:101F80003CD00C283AD02046FFF7F0F809208DF815
:101F90002000686A0D9031E03878052805D00620C9
:101FA000387003261820287046E005218DF820108F
:101FB000686A0D90B8680A900220ADF824000120EC
:101FC0008DF830000A980170297D4170394608A8C3
:101FD000FFF78AF8064618202870012E0ED02BE055
:101FE00001208DF82000686A0D9003208DF82400F0
:101FF000287D8DF8250085F814B012E0287D80B189
:102000001D202070172028708DF82090686A0D9090
:1020100002208DF82400394608A8FFF765F8064627
:102020000AE00CB1FE2020709DF8200020B10021B4
:1020300008A8FFF759F810E413B03046BDE8F08F58
:102040002DE9F04387B00C464E6900218DF804104D
:1020500001202578034602274FF007094FF0050CB1
:1020600085B1012D53D0022D39D1FE2030708DF86D
:102070000030606A059003208DF80400207E8DF802
:10208000050063E02179012925D002292DD00329FB
:1020900028D0042923D1B17D022920D131780D1F08
:1020A000042D04D30A3D032D01D31D2917D1218905
:1020B000022914D38DF80470237020899DF8041030
:1020C00088421BD2082001E09C4702008DF80000E6
:1020D000606A059057E070780128EBD0052007B0C2
:1020E000BDE8F0831D203070E4E771780229F5D156
:1020F00031780C29F3D18DF80490DDE7083402F82B
:1021000004CB94E80B0082E80B000320E7E7157886
:10211000052DE4D18DF800C0656A05959568029596
:102120008DF8101094F80480B8F1010F13D0B8F1B5
:10213000020F2DD0B8F1030F1CD0B8F1040FCED18F
:10214000ADF804700E202870207E6870002168466B
:10215000FEF7CAFF0CE0ADF804700B202870207E5B
:10216000002100F01F0068706846FEF7BDFF377061
:102170000020B4E7ADF804708DF8103085F800C089
:10218000207E6870277011466846FEF7ADFFA6E70F
:10219000ADF804902B70207F6870607F00F0010024
:1021A000A870A07F00F01F00E870E27F2A71C007CE
:1021B0001CD094F8200000F00700687194F821000A
:1021C00000F00700A87100216846FEF78DFF28681F
:1021D000F062A8883086A87986F83200A069407835
:1021E00070752879B0700D203070C1E7A9716971E0
:1021F000E9E700B587B004280CD101208DF8000074
:102200008DF80400002005918DF805000146684610
:10221000FEF76AFF07B000BD70B50C46054602F038
:1022200031F821462846BDE870407823002201F0AD
:102230007FBF08B1007870470C20704770B50C0064
:1022400005784FF000010CD021702146F3F701F81A
:1022500069482178405D884201D1032070BD022089
:1022600070BDF2F7F6FF002070BD0279012A05D09B
:1022700000220A704B78012B02D003E00420704743
:102280000A758A6102799300521C0271C1500320C1
:102290007047F0B587B00F4605460124287905EB55
